:020000040800F2
:1000000000000120F53F0008892700088B27000821
:100010008D2700088F2700089127000800000000A6
:10002000000000000000000000000000932700080E
:10003000952700080000000097270008992700086E
:1000400045400008454000089D270008454000083D
:100050004540000845400008A9270008AF270008D0
:100060004540000845400008E127000845400008D9
:10007000B5270008B7270008B9270008C5270008DA
:10008000D1270008DD27000845400008454000084A
:100090000000000045400008E32700084540000834
:1000A000454000084540000845400008454000081C
:1000B000454000084540000845400008454000080C
:1000C00045400008454000084540000845400008FC
:1000D00045400008ED27000845400008454000085D
:1000E00045400008E9270008F927000845400008B6
:1000F00045400008000000000000000045400008E6
:100100004540000845400008052800084540000813
:1001100045400008454000084540000845400008AB
:10012000454000084540000845400008454000089B
:080130004540000845400008AD
:1001380010B5054C237833B9044B13B10448AFF319
:1001480000800123237010BD0C0600200000000071
:100158003819010808B5034B1BB103490348AFF32D
:10016800008008BD000000001006002038190108B2
:1001780014214160704714207047406A704700009E
:10018800790100087F01000883010008990100082F
:1001980010B5044604F1100000F05CFCC4F8F80047
:1001A8000148C4F87C0110BD88010008F8B5E6B024
:1001B80004460D4616461F460A4906A800F0CAFE20
:1001C80070996F9A05910492009733466E996D9ACB
:1001D800039102922A466C990191214600F060F839
:1001E80067B0F0BD94010008F8B5E6B004460D46C6
:1001F80016461F46094906A800F0ACFE6F996E9A8C
:100208000491039200976D996C9A0291019233467A
:100218002A46214600F087F867B0F0BD940100082F
:1002280038B500281CBF01680029184A23D1184B8B
:100238001C684FF6F0710C404CF24025AC421FBFD1
:100248001B6819404CF27024A14212D1114D296843
:1002580079B911490B68C3F30B03B3F58A6F1FBF54
:100268000968C1F30B0140F28343994204BF01219D
:10027800117028B905E0094B994204BF012111709A
:100288004068BDE8324001F09FBE00BF280600204C
:1002980000ED00E0002004E00010005C000037489A
:1002A8002DE9F04104460D46216816464A681F4666
:1002B80090478046B8F5403F2ED122680A99936846
:1002C800204698478046B8F5403F25D12368089ACC
:1002D8000799D3F80CC02046E0478046B8F5403F60
:1002E8001AD12368069A39461F692046B8478046BE
:1002F800B8F5403F10D1236829465D69324620464B
:10030800A8478046B8F5403F06D123680B9A09995B
:100318009D692046A847804621680A68204690477C
:100328004046BDE8F0812DE9F04104460D462168BC
:1003380016464A681F4690478046B8F5403F2ED17A
:1003480022680A999368204698478046B8F5403F46
:1003580025D12368089A0799D3F80CC02046E047AE
:100368008046B8F5403F1AD12368069A39461F6976
:100378002046B8478046B8F5403F10D12368294643
:100388005D6932462046A8478046B8F5403F06D109
:1003980023680999DD6900222046A847804621681C
:1003A8000A68204690474046BDE8F0814FF4403047
:1003B80070470000F0B50C4685B0114600281A4673
:1003C8001CBF0568002D0B4B11D082B104B971B95F
:1003D8000D9860B10F9E0E9F0A9B0290049603979A
:1003E8000B980C9E009001962046A8470346184695
:1003F80005B0F0BD020003002DE9F04F0646D0B06D
:100408000868F56DD6F860E0726EB76EF36E00BAE4
:1004180000906C46486800BA60600DF14008886832
:1004280000BAA060C86800BAE060086900BA206134
:10043800486900BA6061886900BAA061C86900BAF1
:10044800E061086A00BA2062486A00BA6062886A95
:1004580000BAA062C86A00BAE062086B00BA2063FA
:10046800486B00BA6063886B00BAA063C86B00BAB7
:10047800E063402058F80C1C58F820CC58F838ACE9
:100488008CEA010158F840CC8AEA01018CEA01099A
:100498004FEAF979401E48F8049BEBD187EA02003D
:1004A80000EA0E00784010EBF5610098DFF824C4EC
:1004B80041186144C81882EABE032B404FEAF06134
:1004C80053405918636859186144CF194FEAB50366
:1004D80083EABE01014081EABE0111EBF765A1681C
:1004E8004D196544A91883EAB0023A404FEAF1650C
:1004F8005A405519E26855194FEAB70282EAB0071F
:1005080065440F4005EBBE0E97EAB00717EBFE6592
:1005180027697D194FEAB10782EA0701654401EAB4
:100528000E01EB18514011EBF36561694D194FEA63
:10053800BE0187EA010E65440EEA030E15EBB00012
:100548008EEA070E0EEBF065D4F818E075446544A2
:10055800AA1881EAB30505404FEAF26E4D40AE4451
:10056800E569AE44E64477444FEAB00080EAB30E4A
:100578000EEA020E8EEAB30E0EEBF765D4F820E011
:1005880075446544691880EAB2053D404FEAF16E4A
:100598004540AE44656AAE44E6440EEBB3034FEA09
:1005A800B70787EAB20E0EEA010E8EEAB20E0EEB1C
:1005B800F365D4F828E075446544281887EAB1053E
:1005C8001D404FEAF06E7D40AE44E56AAE44E64415
:1005D8000EEBB2024FEAB30383EAB10E0EEA000E45
:1005E8008EEAB10E0EEBF265D4F830E0754465443E
:1005F800EF1983EAB00515404FEAF76E5D40AE4447
:10060800656BAE44E6440EEBB1014FEAB20282EAF2
:10061800B00E0EEA070E8EEAB00E0EEBF165D4F8B6
:1006280038E075446544EB1882EAB7050D404FEA97
:10063800F36E5540AE44E56BAE44E6440EEBB000B5
:100648004FEAB10181EAB70E0EEA030E8EEAB70E41
:100658000EEBF065D4F840E07544654481EAB30ECA
:10066800AA180EEA000E4FEAF2658EEA010E7544EA
:10067800DDF844E04FEAB000754480EAB30E654403
:100688000EEA020E15EBB7078EEAB30E0EEBF7650E
:10069800DDF848E04FEAB202754480EA020E65448C
:1006A8000EEA070E69188EEA000E0EEBF165DDF80A
:1006B8004CE07544654405EBB3034FEAB70E1427C5
:1006C8000DF1500CDFF810528EEA010B82EA0B0B89
:1006D8000BEBF36A5CF804BBDA44AA44504483EA9F
:1006E800B10B4FEAF06A8EEA0B0BDA445CF804BBF4
:1006F800DA44AA44524480EAB30B4FEAF26A8BEA1E
:10070800B10BDA445CF804BBDA444FEAB000AA44FF
:1007180080EA020BD6448BEAB30B0BEBFE6A5CF85B
:1007280004BBDA444FEAB202AA4482EA0E0B0AEB8F
:10073800B10180EA0B0B0BEBF16A5CF804BBDA44FD
:100748007F1DAA44282F0AEBB3034FEABE0EBBD382
:100758003C2F61D3502F4DD204EB870CC7F15407BF
:100768005E4CA7FB04A504465D4FA8088EEA010A63
:1007780082EA0A0A5CF804BB0AEBF3655D447D195A
:100788002C1983EAB10A4FEAF4658EEA0A0A55443D
:100798005CF804AB5CF804BB55447D19AA1884EADC
:1007A800B30A4FEAF2658AEAB10A55445D444FEA52
:1007B800B4047D1984EA020AAE448AEAB30A0AEB51
:1007C800FE655CF804AB55444FEAB2027D1982EA33
:1007D8000E0A15EBB10184EA0A0A5CF804BB0AEBBD
:1007E800F1655D447D1915EBB303401E4FEABE0E5B
:1007F800BCD12046F46D1B19F365336EC9183166F8
:10080800716E71447166B36ED218B266F16E40189B
:10081800F06650B0BDE8F08F4EEA010B0EEA010A0F
:100828000BEA020B4BEA0A0A0AEBF36554F827A015
:10083800DFF8B0C0554443EAB10B654403EAB10A96
:100848000BEA0E0B28184BEA0A0A7F1C0AEBF06524
:1008580054F827A0554440EAB30B654400EAB30AAC
:100868000BEAB10BAA184BEA0A0A7F1C0AEBF265DD
:1008780054F827A055444FEAB00040EA020B6544FB
:1008880000EA020A0BEAB30BAE444BEA0A0A7F1CE1
:100898000AEBFE6554F827A055444FEAB20242EA33
:1008A8000E0B654402EA0E0A0BEA000B15EBB101C8
:1008B8004BEA0A0A7F1C0AEBF16554F827A0554455
:1008C8007F1C65443C2F05EBB3034FEABE0EA3D350
:1008D80040E700BF9979825AA1EBD96ECDCCCCCC38
:1008E800D6C162CADCBC1B8F00B581B00168074A5B
:1008F800914200D110B9064801B000BD7C2110F02A
:100908007FFF4FF4003001B000BD00BFFC090008B4
:10091800030002002DE9F0410B4A92E8F85188B033
:10092800694681E8F8510268084B9A4200D118B923
:10093800074808B0BDE8F0811422083000F04FFBEA
:1009480008B0BDE8F08100BFDC090008FC09000818
:1009580003000200152904D20268044B9A4200D110
:1009680008B903487047083000F048BBFC09000884
:100978000300020010B481B013460268074CA2427B
:1009880000D118B901B010BC0548704701B000F19A
:10099800240210BC083000F035BB00BFFC09000879
:1009A8000300020010B481B013460268074CA2424B
:1009B80000D118B901B010BC054870470A4601B00B
:1009C80000F1240110BC083000F070BBFC090008DD
:1009D800030002000123456789ABCDEFFEDCBA981E
:1009E80076543210F0E1D2C300000000000000008D
:1009F80000000000F10800081D0900085D09000852
:100A08007D090008AD09000801040008790F0008F5
:100A1800C50F0008810F0008F0B5A3B004460B48C5
:100A280002900D4616461F46094B0822402104A88D
:100A380000F0D1FA28980190009733462A462146BB
:100A480002A800F01BF823B0F0BD00BFFC090008A5
:100A5800100A000810B5040008BF002408D0054893
:100A6800054B20600822402104F1080000F0B3FA89
:100A7800204610BDFC090008100A00082DE9F041C5
:100A880004460E46216817464A681D469047804628
:100A9800B8F5003F19D1226806999368204698470F
:100AA8008046B8F5003F10D123683146DE683A46E3
:100AB8002046B0478046B8F5003F06D12368079A1C
:100AC80029461D692046A847804621680A682046AD
:100AD80090474046BDE8F08110B500F033FA4FF476
:100AE800403400280EBF034C4FF4C07110F088FE4C
:100AF800204610BD0200030010B5044600F022FA9B
:100B080008B9054810BD0021A160D0F87C21116802
:100B180088474FF4403010BD0200030070B504460A
:100B28000D4600F00FFA064E40B1D0F87C0141683E
:100B38008847A84224BF65604FF44036304670BDF0
:100B4800020003002DE9FF4715000C4600D02CB128
:100B5800064600F0F7F95FEA000801D16448C3E0EF
:100B6800D8F8F80001684A689047B0F5003F17D1F7
:100B7800D8F87C118A68404690478146B9F1810FC0
:100B880080F09E80A94508F1FC0A17D2D8F8F80031
:100B98000368D3F80CC02A462146E047B0F5003F69
:100BA80040F08E80D8F8F8000368D3F810C06A4681
:100BB8005146E047B0F5003F76D10AE0002004E056
:100BC800215C0AF800100098401C00900098A84288
:100BD800F6D34FF0000C4749474A484B01AC009800
:100BE800844558D2D3E9007001ADC5E9007010788A
:100BF80000281ABF042086464FF0000E085854F803
:100C08000E5028443E4D05600127D0F800E087606B
:100C1800019D4F681AF80C007D408EEA050585F0A5
:100C2800040E65680F687D4085F0FC05754485F005
:100C3800A30568400AF80C000CF1010CCFE7D3E9D2
:100C4800004501A8C0E9004510782E4D002814BFC2
:100C58004FF0040E4FF0000E01A8744651F80EE054
:100C68000459A6440127CEF80050DEF80040CEF81B
:100C780008704D68019F40687D406C400D68684071
:100C880084F0040480F0FC00041984F057040AF886
:100C98000C400CF1010CCC45D1D3D8F8F800016810
:100CA8004A689047B0F5003F0AD1D8F8F8000368C1
:100CB800D3F80C804A465146C047B0F5003F01D0F2
:100CC800114811E0002006E05AF8201081F06A313E
:100CD8004AF82010401CB0EB990FF5D3B06840F0EB
:100CE8000100B0604FF4403004B0BDE8F08700BFA9
:100CF80002000300A419010828060020240F000898
:100D0800ADBE4ED70DBE75A10100030038B50C4627
:100D1800017A1546CA0702D500F014F908B908483F
:100D280032BDD0F8F80003682146DC682A46A0479F
:100D3800B0F5003F01D0034832BD4FF4403032BD1A
:100D480002000300010003002DE9F84191B00546B7
:100D58000E461746402101A810F052FD297AC8070F
:100D680004D5284600F0EEF8040002D1DFF8A4808C
:100D78004BE0D4F8F800DFF8A0800368D3F810C07F
:100D88006A4601A9E047B0F5003F3ED1D4F8F80023
:100D980001684A689047B0F5003F36D1D4F87C1115
:100DA8008A6820469047D4F8F830024618461B68EF
:100DB800D3F80CC004F1FC01E047B0F5003F24D1A2
:100DC800D4F87C0141688847D4F8F83002461846C0
:100DD8001B68D3F80CC001A9E047B0F5003F14D157
:100DE800D4F8F8000268696893689847B0F5003F3E
:100DF8000BD1D4F8F80003681C693A463146A0477D
:100E0800B0F5003F08BF4FF44038404612B0BDE887
:100E1800F08100BF02000300010003002DE9F84142
:100E2800A5B0074688461646402115A810F0E8FCEC
:100E380000220492402105A810F0E2FC387AC1078C
:100E48005ED5384600F07EF8050059D0D5F8F80090
:100E58002D4C0368D3F810C06A4605A9E047B0F5E1
:100E6800003F3CD1D5F8F80001684A689047B0F5D2
:100E7800003F34D1D5F87C118A6828469047D5F8C8
:100E8800F830024618461B68D3F80CC005F1FC017F
:100E9800E047B0F5003F22D1D5F87C01416888478A
:100EA800D5F8F830024618461B68D3F80CC005A9D7
:100EB800E047B0F5003F12D1D5F8F800026879682C
:100EC80093689847B0F5003F09D1D5F8F800036852
:100ED8001D6904AA15A9A847B0F5003F01D020460E
:100EE8000FE00A4B0A490B4A0396029101924046C9
:100EF8001C68049B009415AA796800F0E5F900E0E5
:100F0800054826B0BDE8F08101000300AC190108CE
:100F1800936E030026C703000200030004B001011A
:100F280000170145E10A0008010B0008250B00081D
:100F3800B50300084D0B0008150D0008510D0008F9
:100F4800250E00080168024A914218BF0020704728
:100F58002C0F000810B5040008BF002404D0034873
:100F68002060204609688847204610BD2C0F0008DD
:100F780020225C3010F042BCF0B58468A30800223F
:100F880004F0030407E000F15C0555F8226035BA67
:100F980041F82250521C9A42F5D300220BE000F18E
:100FA8005C0502EB830755F82360D500C5F11805E9
:100FB800EE40CE55521CA242F1D3F0BD30B5C46804
:100FC80003690022E31AD5188C5C0544521C082AD0
:100FD8002C77F8D330BD0360C1600261704738B523
:100FE800044615460022626023685A68904700202C
:100FF8006061A061A5604FF4003032BD81604FF49C
:10100800003070472DE9F84304462079D4F80C8065
:10101800450748BF244845D466691D46A8F1010024
:1010280000EAD60306EBC506B6EBC50F666102D229
:10103800A669761CA6611746A66906EB5576A661D1
:101048000E46E918884225D2A8EB03094A463146DC
:10105800F81810F0D3FB2268136839460FE04246AF
:10106800384610F0CBFB23681A683946204690476B
:1010780007E0311811F00300F1D122681368204607
:101088009847484600EB0809A9F10101A942F0D3A5
:10109800002300E000202A1A3118F81810F0AEFBDF
:1010A8004FF40030BDE8F283040002002DE9FC4F44
:1010B800024685B0D0681369DFF86CC1DFF86C812F
:1010C800A0EB030A506840F004005060002703A812
:1010D80002900DF10C0ED8E9003403A8544DC0E974
:1010E80000342878534D00280CBF00230423994668
:1010F8005CF803305EF80940234401261D601C6833
:101108009E60DCF80430039DDCF80090DEF8046093
:101118005D406540484C654089EA0606474C664094
:101128007519474C6540D8E9006B03AC0028C4E941
:10113800006B0EBF002404200424029E5CF800000B
:10114800345920183F4C04600126046886600398CF
:10115800029E43406340384C7068634089EA00004F
:10116800364C6040034438484340280018BF0120EB
:101178005B1E9B41042F2CBFC0B2D80F02F1140391
:1011880053F8200007F00303C3F10303DB00D84042
:101198000DF807007F1C082F9DD315460C466A6979
:1011A800AB69E868D20842EA4372401E00EA0207C7
:1011B800002302409B420AD8524508D28020E055BD
:1011C8007F1C574516D2AAEB0701E01910E08020D2
:1011D800E05500E0E355E8687F1C8742FAD32A68A7
:1011E800136828469847BAF1000F03D051462046A5
:1011F80010F006FB2A68069E059F936869462846F4
:1012080098472A68D2F8009021462846C8472B6894
:10121800DA683946284690470EB1A86830604FF41E
:10122800003007B0BDE8F08FA41901085412000877
:10123800280600205FC5109304850012FC68017A17
:10124800C0F524FF24AF33D426AF698B04B0010165
:1012580000170145F8B501240094002300240DE08F
:10126800009D065D0F5D7E40F643761CF60F86F006
:10127800010635400095641C009DEB189442EFD39D
:101288001846F2BDF8B5002301240094002A11E0A5
:10129800009C85188F1815F8016C17F8015C6E40D2
:1012A800F643761CF60F86F0010634400094009C45
:1012B800E318521EECD11846F2BD00005D1200087A
:1012C8008D120008010000002DE9F84F1D46DDF8D9
:1012D80028900B9F0D9C4FF0FF3300930E469246CB
:1012E800D9F800B0804632465146D847834664B3A1
:1012F800D9F8043032465146404698476FEA0B0207
:10130800521C42EA0B0200996FEAD2735B1C194027
:10131800C2430091521C024300996FEAD2735B1CCE
:101328001940009186F05531484087EA000181F064
:101338005531216080F05531C943491C0843009A52
:101348006FEAD070401C82430092D9F80800012847
:1013580009D17540E943491C0D4300986FEAD572DD
:10136800521C90430AE0F11C85EA9102D243521CB8
:10137800154300986FEAD5735B1C984386F0AA362C
:10138800009086EA0B0686F0AA33F243DB430C98FA
:10139800C2F3C0725B1C42EAD3720099D243521C5A
:1013A80091430091774000998843009987F0AA37C4
:1013B8000F403843BDE8F28F034613F8012B002A8B
:1013C800FBD1181A0138704781F0004102E000BFD4
:1013D80083F0004330B54FEA41044FEA430594EAED
:1013E800050F08BF90EA020F1FBF54EA000C55EA28
:1013F800020C7FEA645C7FEA655C00F0E2804FEAF9
:101408005454D4EB5555B8BF6D420CDD2C4480EADA
:10141800020281EA030382EA000083EA010180EA0A
:10142800020281EA0303362D88BF30BD11F0004F58
:101438004FEA01314FF4801C4CEA113102D040428E
:1014480061EB410113F0004F4FEA03334CEA1333C9
:1014580002D0524263EB430394EA050F00F0A780E1
:10146800A4F10104D5F1200E0DDB02FA0EFC22FADC
:1014780005F2801841F1000103FA0EF2801843FAD0
:1014880005F359410EE0A5F120050EF1200E012AC1
:1014980003FA0EFC28BF4CF0020C43FA05F3C018FF
:1014A80051EBE37101F0004507D54FF0000EDCF178
:1014B800000C7EEB00006EEB0101B1F5801F1BD321
:1014C800B1F5001F0CD349085FEA30004FEA3C0C25
:1014D80004F101044FEA445212F5800F80F09A801B
:1014E800BCF1004F08BF5FEA500C50F1000041EB1F
:1014F800045141EA050130BD5FEA4C0C404141EB23
:101508000101013C28BFB1F5801FE9D291F0000F1D
:1015180004BF01460020B1FA81F308BF2033A3F1CC
:101528000B03B3F120020CDA0C3208DD02F1140CC3
:10153800C2F10C0201FA0CF021FA02F10CE002F1FE
:101548001402D8BFC2F1200C01FA02F120FA0CFCF7
:10155800DCBF41EA0C019040E41AA2BF01EB045140
:10156800294330BD6FEA04041F3C1CDA0C340EDC3E
:1015780004F11404C4F1200220FA04F001FA02F381
:1015880040EA030021FA04F345EA030130BDC4F13F
:101598000C04C4F1200220FA02F001FA04F340EA34
:1015A8000300294630BD21FA04F0294630BD94F0E5
:1015B800000F83F4801306BF81F480110134013DCC
:1015C8004EE77FEA645C18BF7FEA655C29D094EA3D
:1015D800050F08BF90EA020F05D054EA000C04BFBB
:1015E8001946104630BD91EA030F1EBF00210020A6
:1015F80030BD5FEA545C05D14000494128BF41F045
:10160800004130BD14F580043CBF01F5801130BDA8
:1016180001F0004545F0FE4141F470014FF0000033
:1016280030BD7FEA645C1ABF194610467FEA655CE4
:101638001CBF0B46024650EA013406BF52EA033586
:1016480091EA030F41F4002130BD00BF90F0000F74
:1016580004BF0021704730B54FF4806404F13204B0
:101668004FF000054FF0000150E700BF90F0000F69
:1016780004BF0021704730B54FF4806404F1320490
:1016880010F0004548BF40424FF000013EE700BF60
:1016980042004FEAE2014FEA31014FEA02701FBFF0
:1016A80012F07F4393F07F4F81F06051704732F022
:1016B8007F4208BF704793F07F4F04BF41F4002179
:1016C800704730B54FF4607401F0004521F00041D7
:1016D8001CE700BF50EA010208BF704730B54FF061
:1016E80000050AE050EA010208BF704730B511F062
:1016F800004502D5404261EB41014FF4806404F19A
:1017080032045FEA915C3FF4D8AE4FF003025FEA1F
:10171800DC0C18BF03325FEADC0C18BF033202EBA3
:10172800DC02C2F1200300FA03FC20FA02F001FAFD
:1017380003FE40EA0E0021FA02F11444BDE600BFA0
:101748004FF0FF3C06E000BF4FF0010C02E000BF85
:101758004FF0010C4DF804CD4FEA410C7FEA6C5C68
:101768004FEA430C18BF7FEA6C5C1BD001B050EA0B
:10177800410C0CBF52EA430C91EA030F02BF90EAF6
:10178800020F0020704710F1000F91EA030F58BFB5
:10179800994208BF90422CBFD8176FEAE37040F017
:1017A800010070474FEA410C7FEA6C5C02D150EAB5
:1017B800013C07D14FEA430C7FEA6C5CD6D152EA70
:1017C800033CD3D05DF8040B704700BF8446104635
:1017D80062468C461946634600E000BF01B5FFF734
:1017E800B7FF002848BF10F1000F01BD4DF808ED04
:1017F800FFF7F4FF0CBF012000205DF808FB00BFD5
:101808004DF808EDFFF7EAFF34BF012000205DF82E
:1018180008FB00BF4DF808EDFFF7E0FF94BF01207B
:1018280000205DF808FB00BF4DF808EDFFF7CEFF7C
:1018380094BF012000205DF808FB00BF4DF808EDBB
:10184800FFF7C4FF34BF012000205DF808FB00BF8C
:101858004FEA410212F5001215D211D56FF47873D0
:10186800B3EB625212D94FEAC12343F0004343EA73
:10187800505311F0004F23FA02F018BF404270474E
:101888004FF00000704750EA013005D111F00040D8
:1018980008BF6FF0004070474FF00000704700BF6E
:1018A80080F0004002E000BF81F0004142001FBF0D
:1018B8005FEA410392EA030F7FEA226C7FEA236C16
:1018C8006AD04FEA1262D2EB1363C1BFD21841400B
:1018D80048404140B8BF5B42192B88BF704710F0A1
:1018E800004F40F4000020F07F4018BF404211F044
:1018F800004F41F4000121F07F4118BF494292EAAC
:10190800030F3FD0A2F1010241FA03FC10EB0C00D7
:10191800C3F1200301FA03F100F0004302D5494264
:1019280060EB4000B0F5000F13D3B0F1807F06D311
:1019380040084FEA310102F10102FE2A51D2B1F109
:10194800004F40EBC25008BF20F0010040EA0300FE
:101958007047490040EB0000013A28BFB0F5000F7E
:10196800EDD2B0FA80FCACF1080CB2EB0C0200FA34
:101978000CF0AABF00EBC25052421843BCBFD04083
:101988001843704792F0000F81F4000106BF80F4FD
:1019980000000132013BB5E74FEA41037FEA226CC0
:1019A80018BF7FEA236C21D092EA030F04D092F08B
:1019B800000F08BF0846704790EA010F1CBF0020BF
:1019C800704712F07F4F04D1400028BF40F000401C
:1019D800704712F100723CBF00F50000704700F03C
:1019E800004343F0FE4040F4000070477FEA226263
:1019F80016BF08467FEA23630146420206BF5FEA34
:101A0800412390EA010F40F4800070474FF0000333
:101A180004E000BF10F0004348BF40425FEA000CFA
:101A280008BF704743F0964301464FF000001CE0A2
:101A380050EA010208BF70474FF000030AE000BFF8
:101A480050EA010208BF704711F0004302D5404236
:101A580061EB41015FEA010C02BF844601460020A8
:101A680043F0B64308BFA3F18053A3F50003BCFAC3
:101A78008CF2083AA3EBC25310DB01FA02FC634470
:101A880000FA02FCC2F12002BCF1004F20FA02F277
:101A980043EB020008BF20F00100704702F120026A
:101AA80001FA02FCC2F1200250EA4C0021FA02F2CB
:101AB80043EB020008BF20EADC7070474FEA40029F
:101AC800B2F1FE4F0FD34FF09E03B3EB12620DD964
:101AD8004FEA002343F0004310F0004F23FA02F0CE
:101AE80018BF404270474FF00000704712F1610F75
:101AF80001D1420205D110F0004008BF6FF000404C
:101B080070474FF00000704753B94AB9002908BF21
:101B180000281CBF4FF0FF314FF0FF3000F070B9C4
:101B2800ADF1080C6DE904CE00F006F8DDF804E02C
:101B3800DDE9022304B070472DE9F047089E0D4601
:101B480004460F46002B4AD18A42944665D9B2FA18
:101B580082F343B102FA03FCC3F120029F4020FA4A
:101B680002F217439C404FEA1C4E1FFA8CF5B7FB54
:101B7800FEF1220C0EFB117742EA074201FB05F049
:101B880090420AD91CEB020201F1FF3780F01B8159
:101B9800904240F2188102396244121AA4B2B2FB90
:101BA800FEF00EFB102244EA024400FB05F5A542B4
:101BB8000AD91CEB040400F1FF3280F00681A5422B
:101BC80040F203816444023840EA0140641B00216A
:101BD8001EB1DC400023C6E90043BDE8F0878B4214
:101BE80008D9002E00F0EC800021C6E9000508465F
:101BF800BDE8F087B3FA83F1002949D1AB4202D39B
:101C0800824200F2F780841A65EB0302012017462E
:101C1800002EE2D0C6E90047DFE702B9FFDEB2FADC
:101C280082F3002B40F08F808A1A4FEA1C471FFA74
:101C38008CFE0121B2FBF7F507FB1520220C42EAC6
:101C480000420EFB05F0904208D91CEB020205F198
:101C5800FF3802D2904200F2CA804546121AA4B256
:101C6800B2FBF7F007FB102244EA02440EFB00FE29
:101C7800A64508D91CEB040400F1FF3202D2A645A0
:101C880000F2BA801046A4EB0E0440EA05409FE734
:101C9800C1F120078B4022FA07FC4CEA030C05FA35
:101CA80001F420FA07F3FD40234300FA01F94FEA53
:101CB8001C401FFA8CFEB5FBF0F81C0C00FB1855F5
:101CC80044EA054408FB0EF5A54202FA01F20BD9D5
:101CD8001CEB040408F1FF3A80F08780A54240F22B
:101CE8008480A8F102086444641B9DB2B4FBF0F33D
:101CF80000FB134445EA044403FB0EFEA64508D93D
:101D08001CEB040403F1FF306BD2A64569D9023BF2
:101D1800644443EA0840A0FB0283A4EB0E049C42FF
:101D2800C6461D4655D352D056B1B9EB0E0364EBE7
:101D3800050404FA07F7CB40CC401F43C6E90074FA
:101D48000021BDE8F087C3F1200102FA03FC20FA64
:101D580001F225FA01F19D402A434FEA1C471FFA78
:101D68008CFEB1FBF7F007FB1015110C41EA054199
:101D780000FB0EF58D4204FA03F408D91CEB0101AF
:101D880000F1FF382FD28D422DD902386144491B0A
:101D980092B2B1FBF7F507FB151142EA014205FBC8
:101DA8000EF1914208D91CEB020205F1FF3816D258
:101DB800914214D9023D6244521A45EA004139E77A
:101DC8003146304609E73946E7E61046FCE6C145A4
:101DD800AAD2B8EB020E63EB0C050138A4E745461E
:101DE800EAE7034695E74046D1E7D0467CE7023D5F
:101DF800624433E708460BE76444023843E700BF10
:101E0800704700BF1348144A08B54FF00043C0E9B3
:101E180000230422002342610122C2614FF4805151
:101E280007220383C0E90233C0E90933C0E90C1271
:101E38000361837680F8203080F82C30826380F844
:101E48003C30C36402F094FD18B1BDE8084000F0CE
:101E5800F3BB08BD2C060020002401400268084B93
:101E68009A4282B00AD14FF0B0431A6E42F400721F
:101E78001A661B6E03F400730193019B02B070474E
:101E8800002401400268054B9A4201BF4FF0B0425E
:101E9800136E23F400731366704700BF00240140DB
:101EA80030B585B000240546CDE901440394FFF719
:101EB800A9FF144803F0F4F808B100F0BDFB11487D
:101EC800039401A9CDE9015402F0B0FE08B100F075
:101ED800B3FB0C4803F00EF808B100F0ADFB4FF06F
:101EE800FF31084802F044FE064803F0BBF80548F5
:101EF80002F098FE0446034803F05EF8204605B059
:101F080030BD00BF2C060020014B024A1A60704702
:101F18002C0600200024014008B50948FFF7C0FF3F
:101F280068B1084BB3F8AA304FF6FF72934216BF58
:101F380040F6E442044B5343B3FBF0F398B208BDB8
:101F4800002000B40075FF1FD8084C0013B500230B
:101F5800ADF80630FFF7E0FF04461948FFF7A0FF89
:101F6800184BB3F8C820B3F8A8108A4204FB00F055
:101F780018D040F6E443B0FBF3F364205B1A434304
:101F8800521A93FBF2F31E331BB2ADF80630BDF8BC
:101F980006305BB21B02ADF80630BDF8060000B291
:101FA80002B010BD4FF47A7240F6FF73B0FBF3F342
:101FB8005343A3F53923A3F50C6340F6C412E0E7B5
:101FC800001000B00075FF1F4FF0B04382B09A6A4E
:101FD80022F480529A629A6C42F480529A649B6C02
:101FE80003F480530193019B002002B070474FF027
:101FF800B04382B09A6C02439A649B6C034001938D
:10200800019B02B0704708B50420FFF7F0FF0120DC
:10201800FFF7EDFF0220FFF7EAFF002211460B2031
:1020280003F0DCF80B2003F00BF9002211460C201A
:1020380003F0D4F80C2003F003F9002211460D2018
:1020480003F0CCF80D2003F0FBF8002211460E2017
:1020580003F0C4F80E2003F0F3F8002211460F2015
:1020680003F0BCF80F2003F0EBF800221146102013
:1020780003F0B4F8102003F0E3F800221146112011
:1020880003F0ACF8112003F0DBF8002236201146EB
:1020980003F0A4F8BDE80840362003F0D1B80000EA
:1020A80008B503F015FB10B16FF0040008BD064B2E
:1020B8009A6942F040429A614CF2FA321A6103F08E
:1020C80019FB0028F2D0EFE700400058F0B585B0C2
:1020D80000230C4600930646A8B3FFF7E1FF054628
:1020E80070BB03F0F5FA88BB1A481B4A0223019318
:1020F800D0F8E01506F1784302EA8121B3FBF1F745
:1021080001FB1733DB0A0293D0F8E00504F17841AC
:102118000139314402EA8022B1FBF2F002FB1011CE
:10212800C3EBD1230133694601A8039303F062FB93
:1021380020B102280CBF01256FF0010503F0DAFA7F
:10214800284605B0F0BD6FF00505F9E76FF0040506
:10215800F6E700BF0070FF1F00FCFF03014B18608B
:1021680000207047900600202DE9F04F89B0B0F1AB
:10217800006F06460F460092C0F0C580DFF89881D0
:10218800664DD8F8E03505EA832303F10063013B87
:10219800984200F2B880002800F0B880002900F0CA
:1021A800B58040EA02035B0740F0B080FFF778FF94
:1021B8000446A0BB03F08CFA002840F0AA80D8F8A7
:1021C800E01506F1784205EA8121B2FBF1F301FB43
:1021D8001322009B03F17843013B3344B3FBF1F036
:1021E80001FB1033DB0A01334FEAD22AA3EBD222D8
:1021F800012A039388BFC6F30A050AF58038C6F199
:10220800080398BF009D069388BFC5F500654FEA8F
:10221800C828B346039B9A4505D303F06BFA2046BA
:1022280009B0BDE8F08FA6F10803069A1A44954252
:1022380019D804950197CDF814B04FF00009059B03
:1022480009EB0301049B99453ED3009BAB442F4403
:102258005D1BB5F5006F28BF4FF400650AF1010A50
:1022680008F50068D6E753F8081F5A68B2F1FF3F2F
:1022780008BFB1F1FF3FD8D0294B186810B96FF0EB
:102288000504CAE7B8F1000F04D04FF400624146D4
:102298000EF050FEDFF88890D9F80030CBF30A0032
:1022A80039461844AAB20EF045FE4FF40061404684
:1022B800FFF70CFF08BBD9F8003001934FF4006317
:1022C800CDF814800493B8E7019B07914B4402931F
:1022D8000120D3E9002303F047FA88B90799019B45
:1022E800D1E9000259F80310029B5B689A4208BFC3
:1022F800884205D109F10809A1E76FF001048CE7CC
:102308006FF0030489E74FF0FF3488E76FF00504A6
:1023180085E76FF0040482E70070FF1F00FCFF03ED
:1023280090060020B1F1006F70B511D30B4BD3F8B4
:10233800E0650B4B03EA862303F10063013B9942F6
:1023480006D840B139B192B20EF0F4FD002070BD4C
:102358004FF0FF30FBE76FF00500F8E70070FF1F54
:1023680000FCFF03B0F1006F10B40DD3084BD3F895
:10237800E045084B03EA842303F10063013B9842DC
:1023880002D810BCFFF7A2BE4FF0FF3010BC704758
:102398000070FF1F00FCFF034FF0B04382B0DA6CFF
:1023A8000243DA64DB6C03400193019B02B070477F
:1023B80030B5012087B00024CDE90444FFF7ECFFD5
:1023C8000220FFF7E9FF0420FFF7E6FF01250222BC
:1023D8000DEB00014FF404134FF09040CDE90123B9
:1023E800039503F055FA4FF4441301A94FF09040B8
:1023F800CDE90235019503F04BFA04230DEB0301F7
:102408000C48CDE90135CDE9034403F041FA2246F1
:102418002146062002F0E2FE062002F011FF2246C5
:102428002146072002F0DAFE072002F009FF07B074
:1024380030BD00BF0004004808B51248124A134BCB
:10244800C0E9002300230122C0E90232C0E90433B5
:10245800C0E90633036203F0B5FC08B100F0ECF8FC
:102468000848002103F02EFE08B100F0E5F8054801
:10247800002103F04DFE18B1BDE8084000F0DCB8BB
:1024880008BD00BF54070020005800405D3E3020C2
:1024980070B596B005461422002103A80FF082F902
:1024A8003822002108A80FF07DF92A68304B9A429B
:1024B8005BD18023089308A84FF440230E9304F0BF
:1024C80083FB08B100F0B8F84FF0B0444FF4C050A7
:1024D800E36C43F00103E364E36C03F0010302934C
:1024E800029B12230026CDE903030323CDE90563EC
:1024F8004FF09040042303A9079303F0C9F9A36D93
:10250800DFF870C043F48003A365A36D1A4C03F48D
:1025180080030193019B26620D23C4E900C3204672
:102528008023C4E90266C4E90436C4E9066602F0F9
:10253800E7FE08B100F080F8104AEC63A562104C81
:102548000E23C4E900231021002380222046C4E979
:102558000213C4E90423C4E90633236202F0D0FE5F
:1025680008B100F069F8AC63A56216B070BD00BF91
:1025780000580040440002409406002058000240E1
:10258800F406002000B59BB04822002108A80FF0EF
:1025980009F91822002102A80FF004F903F0DEFD62
:1025A8004FF0B0420120D2F8903023F01803C2F85F
:1025B8009030D2F8003423F4C06343F40073C2F8B7
:1025C8000034D2F8003403F4C0630193019B242340
:1025D800089381230B930023CDE91003B02208A8A8
:1025E800CDE9122303F032FF08B172B6FEE74F239C
:1025F800CDE90230CDE90400CDE90600022102A8A8
:1026080004F0BEF908B172B6FEE71BB05DF804FB32
:1026180008B502F05BF9FFF7B5FFFFF7C9FEFFF752
:10262800F2FCFFF709FF00F0B1FD40F6B83000F00A
:102638003FFA00F0B2FDFCE772B6FEE700B58DB0D8
:102648002C22002101A80FF0ADF81748174B0360A2
:102658001F2383604FF080420023C0E90433C0E9A0
:10266800072383614FF48073436204F033FC08B19D
:10267800FFF7E2FF0C4804F059FD08B1FFF7DCFF53
:102688004FF0005300220793074808924FF48073D5
:1026980001A9029206920B9304F07CFC08B1FFF7A3
:1026A800CBFF0DB05DF804FBA80700200028004010
:1026B80010B5044690B03822002102A80FF072F835
:1026C8002268194B9A422CD14FF48033029302A806
:1026D8004FF480730F9304F077FA08B1FFF7ACFF5B
:1026E8004FF0B0430220D3F8902042F40042C3F8E0
:1026F80090209A6D42F480629A659B6D002203F4E3
:10270800806311460193019B02F068FD022002F0EC
:1027180097FD00222A20114602F060FD2A2002F0CF
:102728008FFD10B010BD00BF0028004070470000AA
:1027380008B502F0E1F8044B0120C3F88800BDE8B1
:10274800084003F063BD00BF0004005802F0DBB886
:1027580008B502F0D8F800F059FCFFF729FEFFF79A
:1027680052FCBDE80840FFF767BE08B502F0C4F8A0
:10277800BDE808400121002003F0F8BC704770470D
:10278800FEE7FEE7FEE7FEE7FEE7704770477047A3
:1027980070470000014804F0EFBC00BFA807002004
:1027A800012003F0A1B9022003F09EB970477047D9
:1027B800014802F01FBF00BF94060020014802F044
:1027C80019BF00BF80080020014802F013BF00BFF6
:1027D80020080020FFF7F2BF7047202003F084B9DB
:1027E80070470000014805F08BB800BFE0080020E2
:1027F800014804F0F3BA00BFA8070020014804F01C
:10280800E6BE00BF0C0800202DE9F04389B08046E1
:102818000020109E0790894615461F46FDF700FDCB
:10282800F0B9104CCDE90090CDE9020407AB0E4891
:102838000593142304933A46434629460068FDF756
:10284800B9FD2346324604F1140153F8044B42F80B
:10285800044B8B42F9D1079B337509B0BDE8F0836F
:102868000120FAE7E0070020A01901081FB50E4C67
:1028780000233C2202A8CDE902336275237500F0DB
:10288800B9F8042303AA009412210848FFF7BCFFF3
:102898000749142220460EF075FFB0FA80F35B0951
:1028A800637504B010BD00BFF4070020C819010803
:1028B800920B0020054808B50823036004F0A2FC29
:1028C80018B1BDE80840FFF7B7BE08BD0C080020E6
:1028D8004FF0B04307B55A6E42F001025A665B6E7C
:1028E800002203F00103019311463220019B02F0FC
:1028F80075FC322003B05DF804EB02F0A1BC0000C7
:102908000CB407B5054A05AB102101930EF01CFE67
:1029180003B05DF804EB02B0704700BFDA19010894
:1029280030B585B0044602A80D460EF039FCBDF955
:102938000C30064A00931021029B2046FFF7E0FF67
:102948002046FEF739FD288005B030BDDA190108A8
:102958004FF0B04210B5936823F4004393600EF033
:10296800A7FC0E4B01241C7000F0B6F80EF070F9AD
:102978000B480EF087F90B4B4FF400421A612046C2
:102988000EF086F9FFF7C0FA00F012F90EF07CFAA3
:1029980021462046BDE810400EF096BA18080020DF
:1029A80029290008004000580EF0A4BA08B5FFF71E
:1029B800B3FA40F6B83398420CD8B0F5E16F0BD3B0
:1029C800FE23A0F5E16058434FF49663B0FBF3F0A3
:1029D800C0B208BDFE20FCE70020FAE77FB56846D4
:1029E80000F0CAF80198FFF769F800B207B05DF87F
:1029F80004FB0000194A38B5D2F88035591C044642
:102A080019D101F087FF054601F090FF054401F058
:102A180087FF2B0EE3712B0CA3712B0A6371030E36
:102A2800E370C0F30742C0F307232571C0B2A27058
:102A38006370207038BD190AC3718171190C1B0E9F
:102A480041710371D2F88435C370D2F88405C0F39C
:102A58000722C0F30743000EE9E700BF0070FF1F1D
:102A680038B5094BD3F8803503600133054609D1E1
:102A780001F050FF044601F053FF444001F056FFB7
:102A880044402C6038BD00BF0070FF1F01210220A8
:102A98000EF004BA002102200EF000BA00207047A0
:102AA800024B187808B100F0BBB87047180800202E
:102AB80082B00190019802B000F04EB94FF0B043D7
:102AC80082B0DA6C42F00202DA64DB6C03F00203D3
:102AD8000193019B02B070472DE9F043254C87B064
:102AE80001F02AFF01F030FF01F036FF0123002535
:102AF80002934FF48059032301A9204604934FF40D
:102B0800005803950595FFF7D9FFFFF7D7FFFFF7A3
:102B1800D5FFFFF7D3FFCDF8049002F0B9FE01A965
:102B280020464FF40067CDF8048002F0B1FE01A9F9
:102B380020464FF40046019702F0AAFE01A920465C
:102B4800019602F0A5FE2A464946204602F0C6FF35
:102B58002A464146204602F0C1FF2A463946204609
:102B680002F0BCFF2A463146204602F0B7FF07B004
:102B7800BDE8F0830004004810B50446FFF7E6F905
:102B8800074BA36040F30F20FEF744FF054B064AAE
:102B98002360064B6060C4E90323002010BD00BF1A
:102BA8000000484200007A440D093E00AB030500CE
:102BB80000207047014B1868704700BF1C080020B0
:102BC8000320704708B501464FF47A72002380024B
:102BD800890DFEF799FF08BD4FF47A73A0FB030334
:102BE800800A40EA83507047034B98689A6890427D
:102BF800FBD1C043704700BF0028004008B5FFF76D
:102C0800F3FF014B186008BD1C08002008B5FFF74A
:102C1800EBFF024B1B68C01A08BD00BF1C08002050
:102C2800024B187808B1FFF7DFBF7047190800207A
:102C380010B5074B074C0122DA654FF48071204626
:102C480004F092F84FF0FF332363002010BD00BF5B
:102C580000280040A807002002460021014804F08F
:102C68009CBA00BFA807002002460121014804F0D1
:102C780094BA00BFA807002010B58CB02C22002100
:102C8800044601A80EF08EFDFFF7D2FF0C4B0D484D
:102C98001B681C440023089306934FF00053E44339
:102CA800079301224FF4807301A902940B9304F057
:102CB80071F908B1FFF7C0FC00200CB010BD00BFCF
:102CC8001C080020A807002038B50546FFF78CFF30
:102CD80002210446074804F067FAC4F309024FF4D6
:102CE8007A71A2FB0121920AA30A2A8043EA805042
:102CF80038BD00BFA80700200148002104F054BADD
:102D0800A80700200148012104F04EBAA8070020B6
:102D1800F8B50F4D2E78CEB90E4C4FF0FF3727631C
:102D2800FFF78CFCFFF784FF4FF48071204604F016
:102D38001BF82046276304F0DBF9324620460221BF
:102D480004F02BFAFFF75AFF01232B700020F8BD7F
:102D580019080020A8070020014610B54FF47A7220
:102D680000238002890DFEF7CFFE0146FFF73CFFE6
:102D78000446FFF739FF031B8B4200D310BD00BF89
:102D8800F7E70EF09DBB000010B5064C0221204667
:102D980004F00AFA0221421C2046BDE8104004F063
:102DA800FCB900BFA80700201648174A08B54FF419
:102DB800E133C0E9002300230C22C0E90233C0E953
:102DC8000523C0E90733C0E90933036105F079FB3E
:102DD80008B1FFF731FC0B48002105F0EEFC08B103
:102DE800FFF72AFC0748002105F007FD08B1FFF7A7
:102DF80023FC044805F0C1FC18B1BDE80840FFF702
:102E08001BBC08BDE00800200044004070B596B027
:102E180005461422002103A80EF0C4FC3822002124
:102E280008A80EF0BFFC2A68334B9A4261D10223EE
:102E3800089308A8314B0A9303F0C6FE08B1FFF7C0
:102E4800FBFB4FF0B0430C219A6D2D4C42F400323D
:102E58009A659A6D02F400320292029ADA6C42F094
:102E68000102DA64DB6C03F001030193019B022386
:102E78000026CDE903130323CDE905634FF0904005
:102E8800072303A9079302F003FD1E4826621423B3
:102E9800C4E900031023C4E9023620468023C4E9AC
:102EA8000436C4E9066602F02BFA08B1FFF7C4FB42
:102EB800154AEC67A562154C1323C4E90023204684
:102EC80000238022C4E90233C4E90423C4E9063399
:102ED800236202F015FA08B1FFF7AEFB2520C5F80A
:102EE800804000220221A56202F078F9252002F034
:102EF800A7F916B070BD00BF0044004004000C00E4
:102F080080080020800002406C0002402008002059
:102F180002680E4B9A4210B5044616D14FF0B042E3
:102F28000C21936D23F4003393654FF0904002F029
:102F38005BFDE06F02F058FAD4F8800002F054FA12
:102F4800BDE81040252002F089B910BD00440040BA
:102F580008B50A460146024804F036FC002008BDC0
:102F6800E008002013B5114B114C18604FF4001302
:102F7800009302AB13E90600204605F0A2FB236884
:102F8800DA69D103FCD4DA695202FCD59A68084898
:102F980042F480029A6005F0DAFB064904480122EF
:102FA80005F048FB002002B010BD00BF74090020E6
:102FB800E00800207C09002008B5074B1860FFF7DF
:102FC80022F8FFF7F1FE054AD2F8803043F000639B
:102FD800C2F88030002008BD780900200008005899
:102FE80008B54FF0B04308489A6B42F400329A6330
:102FF8009A6B22F400329A63FFF78AFF0F2002F0DF
:103008002DF9002008BD00BFE008002008B50748DA
:1030180005F057FA08B1FFF70FFB054802F070F901
:1030280018B1BDE80840FFF707BB08BDE00800205D
:10303800800800200268044B9A4203D1034B002009
:103048001B681847704700BF0044004078090020FB
:1030580002680B4B9A4210B504460FD1094B1B6806
:103068002BB1D0F8902012B9074801219847204683
:103078000549BDE81040012205F0DCBA10BD00BFCB
:1030880000440040740900207C09002010B50A4C57
:1030980023780BB9E37C6BB1FFF7E8FB0038074BEB
:1030A80018BF0120400018701B78022B02BF0023B4
:1030B8002370E37410BD00BF920B00208509002027
:1030C80038B5114C2378EBB9E37CDBB90F4D2B688D
:1030D800012B07D92B68042B04D80D4A04210120A1
:1030E80000F0DAF92B68042B0CD9FFF7BFFB003886
:1030F800084B18BF0120400018701B78022B04BF32
:103108000023237038BD00BF920B002080090020E7
:10311800341A01088509002010B5084C0122042141
:10312800204602F0DBFC0A20FFF7C2FC2046002202
:10313800BDE81040042102F0D1BC00BF00040048E3
:1031480070477047022808B50ED801221021074899
:1031580002F0C4FC3220FFF7ABFCBDE8084003488E
:103168000022102102F0BABC08BD00BF00040048CC
:1031780070470000034B1B788370034B01221A70C1
:10318800704700BF84090020910B002008B5FFF7A5
:10319800DFFBBDE8084000F005BB4FF0FF300DF045
:1031A8000DBF704770470000014BD870704700BFD3
:1031B8005C000020014B1874704700BF5C000020C1
:1031C80020B1037813B102480EF028B9704700BF48
:1031D800C80A002008B5022000210DF0B7FEBDE89E
:1031E800084001480EF01AB9E00A00200021012029
:1031F8000DF0ACBE10B5094C60B1206008480EF067
:10320800BFF8216806480EF043F9BDE810400448AD
:103218000EF004B942F210732360EFE77400002047
:10322800E00A002038B504460D4607484FF400610F
:10323800FFF798F830B92A4621460348BDE83840D8
:10324800FEF792BF38BD00BF00F003080A460149E7
:10325800FFF768B800F0030838B50C480EF090F88E
:1032680005F024FF60B90A4C0A480125257005F0CD
:10327800C1FD2078294605F0EBFB04480EF0CEF896
:10328800BDE8384004480EF0C9B800BFE00A002085
:10329800000000205C000020B00A002005F0A4BF58
:1032A80030B585B0FFF782FB354D0446FEF734FE96
:1032B80001A8FFF75FFF33496A68097804232B7078
:1032C8001170696800224A7069688B706B68012107
:1032D800D9706B6820B200EB400000EB4010FE2470
:1032E800B0FBF4F018716B685971274B18780028F7
:1032F80034D01A704FF0904005236C682B7002F0A0
:10330800E7FBA0710723214A214C1278012A88BFC4
:1033180000236B70637A33B105F03CFB012802D1BE
:1033280020460EF02DF81B4B1548D978002205F0E1
:103338001DFC063022D105F027FB044616480EF086
:103348001FF8164B14481968A14238BF21460EF0E1
:103358009FF811480EF062F805B030BD104B1149C6
:103368001A780AB90A783AB100220A701A706B689A
:103378009DF806209A71C5E70623C4E70024DDE717
:1033880004000020780A0020100B00208509002086
:103398007C0A00205C000020E00A00207400002065
:1033A800A70B0020910B002008B5104B012200212B
:1033B80002201A700DF0CAFD0D480EF02FF80D4BC3
:1033C8001B788BB10C4B1A7872B9DB7C63B90B4B49
:1033D8001A68042A9EBF1A6801321A600021BDE8E3
:1033E800084010200DF0B2BD08BD00BF100B002032
:1033F800F80A0020AC0A0020920B00208009002067
:10340800044B1B78022B03D1002108200DF09EBD30
:10341800704700BF0000002008B505F050FE80B9D5
:1034280005F0B8FA01280CD1BFF34F8F0549064BB8
:10343800CA6802F4E0621343CB60BFF34F8F00BF4A
:10344800FDE708BD00ED00E00400FA05704770478D
:103458007047704770470000022808B501460FD032
:10346800202810D0012811D14FF0904002F030FBF5
:10347800074B002118700220BDE808400DF066BD1A
:1034880000210820F8E7034B01221A7008BD00BF8D
:1034980084090020B80B002070B505460C46164676
:1034A80005F046FB0346002834D000241A480DF0E6
:1034B80067FF1A4B18481968A14238BF21460DF01A
:1034C800E7FFBDE8704014480DF0A8BF4A68F05CFB
:1034D800D0540133DAB29442F8D8114B0D701B78EE
:1034E800012B88BF00244C700E4C637A33B105F071
:1034F80051FA012802D120460DF042FF0A4B0B4831
:10350800D978002205F032FB0630CED105F03CFA1E
:103518000446CBE70549DDE7E00A002074000020F7
:10352800850900207C0A00205C000020040000209F
:10353800044B1B7823B9044A05210120FFF7ACBFCF
:10354800704700BF85090020391A010810B500240A
:1035580090B03C22214601A800940EF023F92C4B90
:103568002022DA7219788DF8001059788DF8011038
:1035780099788DF80210D9788DF8031019798DF89B
:10358800041059798DF8051099798DF80610D979B4
:103598008DF80710197A8DF80810597A8DF80910E6
:1035A800997A8DF80A108DF80B2021460DF10B023F
:1035B80058180131007B02F8010F1C29F8D193F843
:1035C80028208DF8282093F829208DF8292093F8B1
:1035D8002A208DF82A2093F82B208DF82B200DF126
:1035E8002B0100229818013290F82C0001F8010FE5
:1035F800142AF7D107484FF40061FEF7B3FE20B94B
:10360800044840226946FEF7AFFD10B010BD00BF68
:103618007800002000F80308014940220DF08ABC18
:1036280000F8030838B51E4C207963794D2BC0B2D9
:103638002BD1C0EB001080000A284FF47A7338BFF2
:103648000A205843174D184B18602B782BB3EB7C86
:103658001BB3FFF7CFFDA379E3794D2B03D0E379B3
:10366800482B18BFE379237A104ADBB21370637AC8
:103678000F4ADBB213700023E21892F82C20D2B262
:10368800EA540133142BF7D138BD6379482B0ABFAC
:103698004FF4616363795843CEE742F21070D8E77C
:1036A80078000020920B002074000020A60B002058
:1036B8008509002010B590B000213C2201A8009196
:1036C8000EF070F84022344968460DF033FC9DF83E
:1036D80000203AB99DF80100042803D19DF8021092
:1036E80001290ED0FFF732FF2C48142200210DF0DB
:1036F8002BFC4FF47A70FFF7DBF9FFF793FF10B05C
:1037080010BD274B1A70587099709DF80310D97026
:103718009DF8041019719DF8051059719DF806104F
:1037280099719DF80710D9719DF8081019729DF8C4
:10373800091059729DF80A1099729DF80B1001F042
:103748003F01D972D87AD1B288421BD89DF8282077
:1037580083F828209DF8292083F829209DF82A201D
:1037680083F82A209DF82B2083F82B200DF12B01BC
:1037780000229818013211F8014F80F82C40142AC1
:10378800F7D1BAE701F140006844194410F8340C45
:1037980008730132D6E700BF00F80308920B002037
:1037A800780000201FB5002403A92046039405F0E3
:1037B80069FC03A9012005F065FC384B38480094E2
:1037C80022464FF4FA710DF07DFD364B36480094D1
:1037D80022464FF4FA710DF075FD344B34480094CD
:1037E80001224FF4FA710DF06DFD2046FEF7B6FC8C
:1037F80008B1FEF721FF2F4B009400224FF4FA6125
:103808002D480DF05FFD2D4A002101200DF05AFCD6
:103818002B4A002102200DF055FC2A4A00210420E1
:103828000DF050FC284A002108200DF04BFC00F058
:1038380061FB2649264805F0E7FB264805F0DAFA39
:103848001B480DF0EBFD244B0021187805F000F91A
:1038580022490094224B0968224800220DF032FDCB
:1038680020480DF0DBFDFFF725FF1F4A002110203F
:103878000DF028FC1D4A00214FF480700DF022FC49
:103888001B4B1C4819681C4B009400220DF01AFDB4
:1038980018480DF0C3FD04B010BD00BF593400082E
:1038A800C80A00205B340008940A00205534000838
:1038B8007C0A002009340008B00A00205589000855
:1038C800A9320008A532000861320008000003018F
:1038D800100000205C000020000000207400002080
:1038E800DD310008E00A0020C93000082131000855
:1038F8000C000020F80A0020B133000810B5044677
:10390800E8B190F90630D3B90D480DF039FDE279E8
:103918000C4B0D4C1A70FFF7CDFE2368236023680B
:103928000BB90A4B23600A480DF02AFD21680848A4
:103938000DF0AEFDBDE8104005480DF06FBD10BD9F
:103948007C0A0020AC0A00200C000020A0860100A0
:10395800F80A002010B50024A2B07C22214603A852
:1039680002940DF01FFF53238DF808304FF4827333
:10397800ADF80A3001238DF80C30ADF80440FFF79C
:1039880015F8FE23B0FBF3F000EB400000EB40100D
:103998008DF80D0001A800F053FBA0B958238DF84D
:1039A8000E3007243022802108480DF0FBFE224605
:1039B80002A906480DF027FF044A21460120FFF717
:1039C8006BFD22B010BD0624ECE700BF110B0020F0
:1039D80070B50378592B90B0044640F0C081052992
:1039E80059D84378443B162B55D8DFE813F011011A
:1039F80054000101540009015400540054005400BB
:103A080073005400EC005400540054007701540033
:103A180054008F0054005400540017008578482D36
:103A280011D1A64A14210120FFF736FD41F2883052
:103A3800FFF73EF840F6B830FFF73AF810B0BDE8A7
:103A48007040FFF7E9BC532D0ED1302280219C48ED
:103A58000DF0A8FEFFF77EFF41F28830FFF728F847
:103A6800974A1521012066E0432D16D100246846A7
:103A78008DF8004005F022F9914A4C231370042375
:103A880093709DF80030547001204133D070137149
:103A98000521FFF701FD10B070BD442DFBD1884C06
:103AA8002C228021201D0DF07DFE002325706370DF
:103AB80001250423A370E5702571FEF777FFFE2327
:103AC800B0FBF3F000EB400000EB401060712246C1
:103AD8000621C7E78378303BDBB2092BDBD879496D
:103AE800794A0B700B78DBB25372754A59231370FD
:103AF8004D2353700B783033937003210120FFF767
:103B0800CBFC10B0BDE87040FFF720BD8578482D8C
:103B180016D16B4A562313700023537004239370F5
:103B280003231371172353710B230120937102236D
:103B3800D070D371082110B0BDE87040FFF7ACBC5D
:103B4800432DA8D15E4C00213C2201A800910DF024
:103B580029FE6846FFF760FD2422802104F10C004D
:103B68000DF020FE9DF8003063709DF80130A370C1
:103B78009DF80230E3709DF8033023719DF80430FE
:103B880063719DF80530A3719DF80630E3719DF8C7
:103B9800073023729DF80830257063729DF80B502A
:103BA8009DF80930A3729DF80A30E3722A4603A9EA
:103BB800257304F10D000DF026FE05F10D012246D6
:103BC800C9B2012065E7807839280CD83038C0B2EE
:103BD800FFF7B6FA3A4A2378137063785370A378DC
:103BE800937003213EE710B0BDE87040FFF7A0BC1A
:103BF80080783928F7D83038C0B2FFF7A2FAE9E759
:103C080080783928EFD83038C0B2FFF79BFAE1E75F
:103C18008378303BDAB2092AE5D8C0783038C2B2A6
:103C2800092AE0D82179A1F14802D2B20B2ADAD8C0
:103C3800264D45FA02F2D207D5D40A224D2902FBB5
:103C4800030036D13C2358434FF47A735843204B32
:103C58001860204B1860FFF7CDFA194A23781370C3
:103C680063785370A3789370E378D37023791371D2
:103C780005210120FFF710FC134B00221A700422C3
:103C88005A7001229A70DA70A278303A02EB8201F7
:103C9800E278303A02EB4102D2B21A7122795A71B3
:103CA8000D4A1278D2B21A72064A1278D2B25A72F1
:103CB80027E74829C8D14FF46163C4E73F1A0108D0
:103CC800110B00208509002078000020DEF7FFFF97
:103CD800740000200C000020A60B00208678A6F1B6
:103CE8003003092B3FF67FAFC078A0F13003092BD2
:103CF8003FF679AF2179A1F14802D2B20B2A3FF6FB
:103D080072AF5A4B134113F001057FF46CAF584A58
:103D18005923137053235370D07011719670052175
:103D28000120FFF7B9FB534904230D704B700123A1
:103D38008B70CB70A378303B03EB8302E378303B86
:103D480003EB4203DBB28B712379CB714A4B1B78AF
:103D5800DBB20B72494B1B78DBB24B72D1E6502BAE
:103D680048D102297FF697AE4378303B012B3FF6C6
:103D780092AE8378312B7FF48EAE0B2904D8FFF7EF
:103D8800D7FB00213A4A6DE63A4D0234002214F876
:103D9800013FA918303B0132DBB20C2A0B73F6D174
:103DA800FFF7E6F9324B502204211A70997000226D
:103DB80001215A70D97003F8041FA9180132097B30
:103DC8000C2A01F1300103F8011FF6D100232B70F2
:103DD80004236B700123AB70EB70274B1B78DBB2AD
:103DE8002B72264B1B78DBB26B72EA72FFF7AEFBC5
:103DF8001121C7E7412B7FF44EAE4378432B7FF464
:103E08004AAE16297FF447AE1D4D421C002312F816
:103E1800011FE9540133142BF9D1FFF737F9194B76
:103E28005B7D012B19D113490023EA5CC8180133C3
:103E3800D2B2142B80F82C20F7D1104B00221A7024
:103E48001B78DBB24B72FFF781FB094A631E1534FE
:103E5800A34206D1064A162104E6084B02221A702C
:103E6800F3E713F8011F02F8011BF1E7DEF7FFFF84
:103E7800110B002078000020A60B002085090020E7
:103E8800920B0020F407002038B504460D4661B3B4
:103E980016480DF0C3FA2B783BB334B36068237827
:103EA80018B3032B0CD0042B17D0022B1DD161782B
:103EB80001291AD00B0618D4BDE83840FFF788BD91
:103EC8006378012B11D10078012802D0022800D094
:103ED80058B9BDE8384004F071BD6378012B04D1AE
:103EE8000378034A03F00103137038BD940A0020D5
:103EF800780A0020034B0022C3E902220122C3E909
:103F080000227047A80B002000487047A80B00202B
:103F18004FF0B04382B0DA6C0243DA64DB6C0340E2
:103F28000193019B02B070472DE9F04186B000244F
:103F38000220154D0594FFF7EBFF0420FFF7E8FF7B
:103F4800124F03944FF4807601230DEB0001CDE965
:103F580001632846032304934FF4005801F098FCAA
:103F680001A93846CDF8048001F092FC224641466A
:103F7800384601F0B3FD28462246314601F0AEFD31
:103F8800204606B0BDE8F08100040048000800485B
:103F9800032810B50ED8012810D868B902460B4876
:103FA8004FF4807101F09AFD002209484FF4005146
:103FB80001F094FD002010BD0122F0E70022034823
:103FC8004FF4807101F08AFD0122EEE700040048F9
:103FD8000008004802207047002070470120704701
:103FE80000280CBF0F201620704700000D4885469A
:103FF80000F06AFC0C480D490D4A002302E0D45831
:10400800C4500433C4188C42F9D30A4A0A4C00231A
:1040180001E013600432A242FBD30DF0CBFBFEF7A4
:10402800F7FAFEE700000120000000200C0600203F
:10403800C02401080C060020FC2A0020FEE7704777
:1040480010B5044600F008F810F0FF001CBFEE237E
:104058002370AA23637010BD2DE9F34700242D4E69
:104068002D4D346021462046FFF7E9FF2146012007
:10407800FFF7E5FF21460220FFF7E1FF274F4FF04A
:104088005208A146012195F8640185F86081C5F8B8
:104098006891FFF7D4FF0320FEF70AFD0DF1060231
:1040A800C021284600F0CAFB78BBBDF806204EF6B2
:1040B800AA639A4229D14FEA440A0AF1540A5FFADC
:1040C8008AFA5146284600F02BF8F0B90DF106029D
:1040D800C021284685F860A100F0B0FB284600F012
:1040E80063F990B9326801231A4432603A68C5F816
:1040F8006831A34013433B600134032C05F5C875B0
:10410800C0D1306802B0BDE8F0870021E0B2FFF707
:1041180096FFF1E7C00B0020B8000020BC0B002080
:104128004A088A2100F03CBB00F09BBA13B5002373
:104138000C460DF1070201218DF8073000F052FB03
:1041480078B99DF80730C3F300122270C3F3C00298
:10415800A270C3F380026270C3F38012DB09E270BD
:10416800237102B010BD37B50D460DF10202F821DA
:10417800044600F063FB70B901AA0421204600F050
:104188007DFB40B9BDF802201AB1019BB3FBF2F3E5
:104198002B602B68A36103B030BD37B50D460DF118
:1041A80006022021044600F049FB28B9BDF8063074
:1041B80023B9236A2B60207703B030BDDB002B6066
:1041C800236201232377F7E70529F8B504460E464D
:1041D800154635D862B100EB810301215A6B0023E3
:1041E800701E042807D8DFE800F00E171A1D2400F7
:1041F80011460123F4E784F828103444E5B984F81B
:104208002850002007E0C2F34F224421204600F046
:10421800D7FA0028F1D0F8BD84F82A10EDE784F821
:104228002B10EAE75B00FE226021204600F0EFFA3F
:10423800EFE71B01EF22F7E7012384F82830E0E7D6
:104248006FF00300E7E770B54318044693F82800B9
:104258000E46154618B904EB8106726370BD052930
:104268001BD8DFE801F0030912141616626304EB89
:10427800860400206563F1E7C2F34F2244212046FB
:1042880000F09EFA0028E9D1F1E7E263EFE7226443
:10429800EDE7C2F34F226421F1E76FF00300DDE799
:1042A80037B50446154605292CD8DFE801F0030781
:1042B80017191B1B436B2B60002021E00DF1060230
:1042C800442100F0BBFAD8B9BDF8062053029AB1D0
:1042D8002B60A363012384F8293011E0C36BEAE75C
:1042E800036CE8E70DF10602642100F0A7FA38B97B
:1042F800BDF806305B02DEE7A36B2B6084F829006B
:1043080003B030BD6FF00300FAE737B50D460DF185
:1043180007020121044600F065FA38B99DF8073014
:1043280084F83031DB092B7084F84C3003B030BD91
:104338002DE9F843037C0C4601F8083B0546FFF7D6
:1043480012FF40BB207304F110012846FFF725FF38
:1043580008BB04F11401284600F0D4F8D8B904F1D8
:10436800240705F1270904F1170806463A46B1B2B1
:104378002846FFF795FF70B9013619F8013F08F88C
:10438800013F062E07F10407F0D104F13C0128464D
:10439800FFF7BBFF08B1BDE8F883211D2846BDE83B
:1043A800F84300F078B90000F0B50022054693B054
:1043B800882100F0F5F94FF47A72A5F852214FF4EC
:1043C800C872A5F854214C4AC5F8582100234B4A15
:1043D80085F8F030C5F8D4202B6202A92846FFF7EB
:1043E800A7FF044670B9ADF8080002AE0FCE05F17C
:1043F80010070FC70FCE0FC70FCE0FC796E80F00D5
:1044080087E80F003E4BC5F834314FF4FA730126A4
:10441800A5F838314FF42063A5F83C3132468021A5
:1044280085F85061284600F0BBF932460746FF215F
:10443800284600F0B5F9002211460743284600F047
:10444800AFF93C4364B204430DF1070291212846B9
:1044580000F0C8F964B29DF8073085F83A31044392
:1044680032460021284600F09BF964B2044300223A
:10447800FF21284600F094F964B204430022802109
:10448800284600F08DF964B2204340B2002488BB6E
:10449800A1B2012228460134FFF796FE062CF6D178
:1044A80040BB04466885024604212846FFF78CFE77
:1044B80000BB024605212846FFF786FED0B94FF417
:1044C80090136B634FF4804201212846FFF7BBFE2F
:1044D80080B94FF40C13FF22C5E90F3085F830215D
:1044E8000121284600F05CF9012385F8323108B92A
:1044F80085F8154113B0F0BD856B0100A470090063
:104508006400840313B50C460DF10602282100F05F
:1045180095F978B9BDF80620C2F30B0312F4006FC1
:1045280018BFA3F580534FF0FA0214BF13FB02F330
:104538005343236002B010BDC3B2000A03FA00F06F
:1045480001307047064B5A434FF47A7002F5FA72FD
:10455800B2FBF0F24A4302F5FA72B2FBF0F0704790
:10456800002F3A002DE9FF4102294FF000050746C8
:1045780016468DF80350ADF804501CD80DF1020210
:104588002946FFF7D1FD044630B90DF10302462153
:10459800384600F027F904469DF80300FFF7CCFFE2
:1045A80081B29DF802203846FFF7CCFF30602046E4
:1045B80004B0BDE8F081032918D10DF102022946A3
:1045C800FFF7B2FD0446002846D101460DF102026C
:1045D8003846FFF7A9FD044628B901AA51213846F3
:1045E80000F02CF90446BDF80400D7E7042935D1BA
:1045F80002A9FFF79BFD9DF80B30ABB10DF102024C
:1046080029463846FFF790FD044658B901AA5121BA
:10461800384600F013F90446BDF80400FFF78CFF94
:1046280085B214B1002015E01D460DF102020121EA
:104638003846FFF779FD04460028F3D10DF106024C
:104648007121384600F0FAF80446BDF80600FFF775
:1046580073FF80B2401BA3E72846A7E728462C46ED
:10466800A4E713B5144629B1012910D06FF003004F
:1046780002B010BD0DF10702502100F0B3F8002878
:10468800F6D19DF8073001335B002370F0E70DF198
:1046980007027021F1E770B54FF4FA6286B0002383
:1046A800CDE9022340F636330B600C4604A90646D2
:1046B800FFF73CFD0546002836D19DF811209DF8EE
:1046C800103013439DF81220134319D002AA022177
:1046D8003046FFF747FF002840D19DF810302BB136
:1046E800029B03F24E222368134423609DF8123084
:1046F800EBB1029B03F2B222236803EB420323606F
:104708009DF81330EBB99DF814305BB101AA042170
:104718003046FFF727FF019B03F226222368134444
:104728002360D8B923687361284606B070BD9DF828
:104738001130002BE4D0029B03F525722368134443
:10474800DDE703AA03213046FFF70CFF039B03F5BF
:1047580025722368134423600028D4D00546E3E774
:1047680007B502F10A03009393B20A4690F8601164
:10477800D0F85C0101F078FB03B05DF804FB13B5D9
:1047880002F10A0390F860410093D0F85C0193B2FB
:104798000A4644F0010101F0FDFB02B010BD000023
:1047A80008B5064B19705A7019460222FFF7D8FF50
:1047B800002814BF6FF01300002008BDC40B0020B0
:1047C80008B5074B1970110A59709A7019460322D7
:1047D800FFF7C6FF002814BF6FF01300002008BDC4
:1047E800C40B002037B515468DF8071001220DF1CE
:1047F80007010446FFF7B4FF28B9012229462046DD
:10480800FFF7BDFF08B16FF0130003B030BDF7B577
:1048180015460DF1070206460F461C46FFF7E2FF54
:1048280050B99DF807301D4044EA05023946304624
:104838008DF80720FFF7B4FF03B0F0BD73B5144639
:104848008DF8071001220DF107010646FFF788FFD2
:1048580018B16FF0130002B070BD074D022229464F
:104868003046FFF78CFF0028F3D12A786B7803EBEA
:1048780002232380EFE700BFC40B002073B5144662
:104888008DF8071001220DF107010646FFF768FFB2
:1048980018B16FF0130002B070BD0A4D042229460A
:1048A8003046FFF76CFF0028F3D16B782A781B0499
:1048B80003EB0263EA781344AA7803EB022323602C
:1048C800E9E700BFC40B00207047000010B50320C3
:1048D80000F072FC01F0AAFD064B18600F20FEF7ED
:1048E800DDF8044618B9FDF74AFF204610BD01243B
:1048F800FBE700BF680500204FF0E022136923F0B2
:104908000203136170474FF0E022136943F002037A
:1049180013617047014BD3F8900570470070FF1F73
:10492800014BD3F8940570470070FF1F014BD3F873
:10493800980570470070FF1F024A536823F001036F
:1049480053607047002004E0024A536823F00203D2
:1049580053607047002004E0024A536823F00403C0
:1049680053607047002004E08068C0F380007047FF
:10497800F7B5002301930446002800F0E980856D0F
:1049880025B9FDF76BFAE56584F8545023689A68F1
:10499800D00040F1A1809A68D10000F1B480A26DE6
:1049A80042F01002A265E26D42F00102E2650125C3
:1049B8001846FFF7D9FFA26D02F01002024340F03B
:1049C800C980A26D206922F4817242F00202A265B8
:1049D8009A68D2075DD4226BA67E94F82CC0003A60
:1049E80018BF01221703D4E902120A43217E42EAC2
:1049F8008132617E42EAC13242EA4632002842EA06
:104A08004C02B4BF20F000414FF400113A430A436E
:104A180094F82010012903D1002E76D142F4803277
:104A2800616A21B1A66A01F4E07131430A43D96889
:104A3800E66C21F4FE3121F4FF711143D96094F83A
:104A48003C206168012A01F0404C4CEA060609D175
:104A5800D4E910273A433243A66C324342EA0C02A7
:104A680042F001061F693E4A3A4032431A6121F07A
:104A78000042B2F1804F0CD0B1F1004F09D0394E4D
:104A8800D6F8082701F4701122F470120A43C6F808
:104A980008275A69666BA16B22F0070232435A61F4
:104AA8005A6922F0700242EA01125A61002835D18F
:104AB8009A6A62F00F029A625B6903F007039E42EA
:104AC8003CD10023E365A36D23F0030343F0010306
:104AD800A365284603B0F0BD9A68234922F0104226
:104AE80022F0170242F080529A60204A1268B2FB04
:104AF800F1F2013252000192019A002A3FF44BAFC1
:104B0800019A013AF7E7002552E7A16D41F020012B
:104B1800A165E16D41F00101E16581E7B0F5001F94
:104B2800CAD19A6AE269013A92006FF00F0102F065
:104B38001C0201FA02F2216E0A43BCE7A36D23F0BE
:104B4800120343F01003A365E36D43F00103E3652B
:104B58000125BEE7A36D43F01003A365F8E700BF86
:104B680002FCFF1F00200140400D030068050020E3
:104B7800F8B54569082D04460E460AD00368DB6877
:104B8800D80705D5A36D43F02003A3650120F8BD20
:104B98000425FDF785FF074623681A682A4221D0B5
:104BA800A26D42F40072A265DA6812F4406F14D163
:104BB800A27E92B91A6812070FD51846FFF7D4FEDD
:104BC80028BB5A6822F00C025A60A26D22F4807247
:104BD80022F0010242F00102A265207E00BB0C22F5
:104BE8001A60D4E7711CD8D0FDF75AFFC01BB04239
:104BF80001D8002ED0D123681B682B40CCD1A26DE0
:104C080084F8543042F00402A2650320BFE7A26D85
:104C180042F02002A265E26D42F00102E265DCE7A3
:104C28000020B4E70368186C70470000F7B500234C
:104C3800019390F85430012B044600F0C5800568B4
:104C48000669012380F854302846FFF78DFE0028B6
:104C580040F0B480D1E90020022826F0040300F0D7
:104C68008280B3F1004FC2F3110E13D1AB6A43EA4D
:104C78000E03AB628B68686903EA022323F07C4366
:104C880023F0FF0320EA02210B43002A6B6126DB95
:104C9800002055E0236E00F01F074FF00F0C0CFAB0
:104CA80007FC6FEA0C0623EA0C0CBEF1000F11D1C9
:104CB800C2F38463BB4043EA0C0323668008E369BC
:104CC80001309842D6D8A86AC2F38363BB40064035
:104CD8003343CEE792FAA2F3B3FA83F3EAE73B4908
:104CE8003B48D1F80837824203F0E07519D11B021E
:104CF800CED4D1F8083723F0E0732B4343F40003F4
:104D0800C1F80837334B1A68334BB2FBF3F20C2364
:104D180002FB03330193019B002BB9D0019B013B9C
:104D2800F8E72E48824210D113F08070B0D1D1F844
:104D3800083723F0E0732B4343F08073C1F808373A
:104D4800002384F8543003B0F0BD254882429FD137
:104D580013F480009CD1D1F8083723F0E0732B437B
:104D680043F48003EAE7B3F1004F01BFAB6AC2F333
:104D780011018B43AB62002A8ADA15481349824233
:104D8800D1F8083709D1D1F8082703F0A07322F029
:104D9800E0721343C1F808377AE71048824204D119
:104DA800D1F8082703F44003F1E70D4882427FF465
:104DB8006FAFD1F8082703F0C073E8E7A26D42F09F
:104DC8002002A2651846BBE70220BCE7002001408C
:104DD800001000B068050020400D0300004000B836
:104DE800002000B4026838B504461046FFF7BCFD41
:104DF80008B9002038BD9368990707D4936823F051
:104E0800004323F0170343F010039360FDF748FEB7
:104E1800054623689B685B07EBD5FDF741FE401B01
:104E28000228F6D923689B685A07F2D5A36D43F088
:104E38001003A365E36D43F00103E3650120D9E79F
:104E480073B50023026801939368DD07044602D511
:104E5800002002B070BD9168214B194209D0A36DA2
:104E680043F01003A365E36D43F00103E3650120FC
:104E7800EFE7936823F0004323F0170343F001039F
:104E88009360184BD3F8083718021CD4637E012BA3
:104E9800DED0FDF705FE144E054622681368DB07D1
:104EA800D6D49368D9075FBF9368334043F00103B2
:104EB8009360FDF7F5FD401B0228EED923681B68B7
:104EC800DA07EAD4CBE7094B094A1B68B3FBF2F3CC
:104ED80001330193019B002BD8D0019B013BF8E7DC
:104EE8001700008000200140E8FFFF7F68050020D0
:104EF800400D030038B504460068FFF735FD054648
:104F080020BB94F85430012B20D0012384F854306E
:104F18002046FFF795FFB0B9A36D226823F47063AC
:104F280023F0010343F48073A3651C23E065136039
:104F380084F85400936823F0004323F0170343F0E8
:104F48000403936038BD84F85450FBE70220F9E766
:104F5800026838B5936891680446C80701D40020F0
:104F680038BD9907FBD4936803F00503012B19D1C9
:104F7800936823F0004323F0170343F00203936080
:104F880003231360FDF78CFD054623689B68DB0748
:104F9800E5D5FDF785FD401B0228F6D923689B68F7
:104FA800DA07F2D5A36D43F01003A365E36D43F070
:104FB8000103E3650120D3E770B5044600284BD010
:104FC800836D43F002038365FFF70CFF054668B95C
:104FD8002046FFF7BDFF054608B90123A3652268EF
:104FE800936823F0104323F01703936023685A68EB
:104FF80022F4677222F003025A6040F29F321A606C
:10500800D968164A0A40DA601A6922F040421A61E1
:105018005A6922F007025A611A6A02F0F0221A62EB
:105028005A6A02F0F0225A62DA6A02F0F022DA6270
:105038009A6A0B4A00269E62D2F8083723F0FE735C
:10504800C2F808372046FCF71DFFE6652666A66508
:1050580084F85460284670BD0125FBE700023E83B2
:105068000020014010B590F85430012B044615D0AB
:10507800012380F85430FFF7B5FE58B92046FFF7F2
:1050880067FF38B9A36D23F4807323F0010343F05D
:105098000103A365002384F8543010BD0220FCE707
:1050A800F7B50023019390F85430012B04467FD0C4
:1050B800012380F85430FFF74BFF23689A6812F0F9
:1050C8000102054607D0A36D43F01003A365002332
:1050D80084F854302DE0A16D364F21F4817141F0F0
:1050E8000201A165DE68D96826F4FF4626F07C0631
:1050F80021F40041360421F00301360CD960082060
:105108009968394041F0004199609968002913DA9B
:105118000199013101910199B1F52E3FF5D3A36DA4
:1051280023F0120343F01003A365002384F85430DE
:105138000125284603B0F0BDD3F8B410013801F0BA
:105148007F010A44DCD199681A48014041F0010105
:105158009960D3F8B41021F07F0141EAD202C3F874
:10516800B4209A68024042F002029A60FDF798FC67
:10517800074623689A68D20708D4DA683243DA60A7
:10518800A36D23F0030343F001039FE7FDF788FCB9
:10519800C01B0228EDD923689B68D907E9D5A36D00
:1051A80043F01003A365E36D43F00103E365BFE734
:1051B8000225BEE7E8FFFF7F0749CA6822F4E062DC
:1051C8000302120403F4E063120C134343F0BF63B9
:1051D80043F40033CB60704700ED00E0164B30B568
:1051E800DC68C4F30224C4F10703251D042B28BF7F
:1051F8000423062D4FF0FF358CBF033C002405FA2D
:1052080003F321EA0303A54022EA0502A34000288C
:1052180043EA0203ACBF00F16040084A4FEA0313B7
:10522800B8BF00F00F00DBB2AABF00F5614013540D
:1052380080F8003330BD00BF00ED00E014ED00E061
:10524800002807DB044A4109012300F01F008340BE
:1052580042F82130704700BF00E100E000280CDB75
:105268004309064900F01F0020330122824041F81B
:105278002320BFF34F8FBFF36F8F704700E100E02B
:1052880070B5D0E913456560446D14B1D0E9164591
:105298006560D0E9105404F01C060124B4406C6029
:1052A800046863608368102B0BBFA260A160E16093
:1052B800E26070BD0268416CD3B210B5083B14249B
:1052C800B3FBF4F30B4CA24288BF0B4A21F0030155
:1052D80099BF01F1804202F5023252180733826405
:1052E800064AC26403F01F03012202FA03F30365AE
:1052F80010BD00BF070402401C080240800802409D
:1053080038B500285ED002682F4B9A424FF014013E
:105318004CD82E4B1344B3FBF1F32D499B00C0E945
:105328001013022380F825301368056923F4FF431E
:1053380023F070031360D0E9024323432B434569EC
:1053480011682B4385692B43C5692B43056A2B4399
:105358000B431360FFF7AEFFB4F5804F04BF002383
:1053680043604268816C02F07F030B60D0E913143C
:10537800013A032A4C6020D8164A174981651A4415
:10538800013B9200012103F0030301FA03F300211A
:105398004265C3651160114A536400230122C36347
:1053A80080F8243080F82520184638BD0C4B13446B
:1053B800B3FBF1F30B499B00B1E70023C0E91533B8
:1053C800C365EAE70120F0E707040240F8FFFDBFE4
:1053D800000002403F8200104009024000090240DC
:1053E800F8FBFDBF0004024038B5002841D0026830
:1053F800136823F0010313601F4B9A424FF0140106
:1054080030D81E4B1344B3FBF1F31D499B00C0E990
:105418001013012403F01C0304FA03F3002515609C
:105428004B60FFF747FF836C41681D60D0E913327A
:105438005A604A1E032A06D8124B0B449B0094401C
:105448001D60114B5C640023C363C0E91533C0E9D8
:105458000B33C0E90D33C36580F8253080F824305C
:10546800184638BD094B1344B3FBF1F308499B00B8
:10547800CDE70120F5E700BF07040240F8FFFDBFB4
:10548800000002403F82001000090240F8FBFDBF07
:105498000004024070B590F82450012D04463BD01A
:1054A80090F825600125AE4280F824504FF00006A0
:1054B8002CD1022580F825500568C6632E6826F091
:1054C80001062E60FFF7DCFE036BBBB12B6843F0CF
:1054D8000E032B60A36C1A68D20342BF1A6842F409
:1054E80080721A60636D1BB11A6842F480721A6088
:1054F8002B6843F001032B60002070BD2B6823F05C
:1055080004032B602B6843F00A03E2E78023C3639C
:1055180080F824602846F0E70220EEE7034640B111
:1055280090F82520022A06D00422C263002280F8BF
:105538002420012070470268806C116821F00E0158
:105548001160016821F480710160116821F0010186
:105558001160D3E9100202F01C0101228A40426066
:10556800D3E9132151605A6D32B1116821F4807169
:105578001160D3E9162151600122002083F825200B
:1055880083F82400704710B590F82530022B03D01B
:105598000423C363012010BD03681A6822F00E02B9
:1055A8001A601A6822F001021A60826C136823F4E8
:1055B80080731360D0E9101303F01C020123934099
:1055C8004B60D0E913325A60436D33B11A6822F444
:1055D80080721A60D0E916325A60012380F82530AB
:1055E800836B002480F8244013B198472046D2E703
:1055F8001846D0E770B4426C046C036826681D68CE
:1056080002F01C020421914031420FD015F0040F22
:105618000CD01A6892065EBF1A6822F004021A605B
:10562800036B6160002B33D070BC18470221914096
:10563800314217D015F0020F14D01A68940606D418
:105648001A6822F00A021A60012280F82520114AFD
:1056580093428CBF104B114B5960002380F82430C3
:10566800C36ADFE708219140314211D029070FD5DD
:10567800196821F00E011960012303FA02F2626031
:10568800C36380F82530002380F82430436BC9E7D2
:1056980070BC7047800002400004024000000240D5
:1056A8000A4A536943F4802330B55361EFF31084F9
:1056B80072B60023CD58C5500433B3F5807FF9D1B5
:1056C8001369DB03FCD484F3108830BD0040005814
:1056D800064B5A69002ABFBF054A9A6002F1883210
:1056E8009A60BABF5869C00F002070470040005840
:1056F80023016745044B5A6942F000425A615869D0
:10570800C043C00F704700BF0040005870B5054641
:10571800FDF7C6F9124E04463369D90313D4336929
:10572800DA0744BF012232614CF2FA32134011D138
:105738000B4E306910F480200BD0FDF7B1F9001B37
:10574800A842F6D304E0FDF7ABF9001BA842E3D367
:10575800032070BD024A1361024A01205360F8E732
:1057680000400058040C00202DE9F041184D9846DF
:105778002B78012B06460C46174626D001232B70A2
:105788004FF47A7000236B60FFF7C0FFA0B9012EB9
:1057980016D1104A536943F0010353612760BFF3E0
:1057A8006F8FC4F804804FF47A70FFF7AFFF094A8F
:1057B800536923EA0603536100232B70BDE8F08187
:1057C80039462046FFF76CFFEDE70220F6E700BFF9
:1057D800040C002000400058054A536923F47E73E6
:1057E80043EAC00040F4803040F002005061704746
:1057F800004000582DE9F041234F3B78012B054626
:1058080088463FD001233B704FF47A7000237B60B9
:10581800FFF77CFF044688B92B68042B13D11B4A79
:10582800536943F4803343F0040353614FF47A70AF
:10583800FFF76CFF0446154B1A681B6800233B7082
:105848002046BDE8F0814FF0FF33C8F800306E689D
:10585800D5E901321344B3420AD93046FFF7BCFFF9
:105868004FF47A70FFF752FF50B1C8F80060044651
:10587800064A536923F47E7323F002035361DAE77F
:105888000136E5E70224DBE7040C0020004000585D
:105898002DE9F04F524C00234FF00F090A6832FAF5
:1058A80003F501D1BDE8F08F012505FA03F818EAE0
:1058B800020200F08E804E68032706F003054FEAC7
:1058C800430E07FA0EFC6F1E012F6FEA0C0C32D83C
:1058D800876807EA0C0ACF6807FA0EF747EA0A074B
:1058E8008760476827EA0808C6F300179F4047EA19
:1058F80008074760C76807EA0C088F6807FA0EF7B9
:1059080047EA0807022DC76017D14FEAD30800EB12
:10591800880803F0070AD8F820704FEA8A0A09FABB
:105928000AFB27EA0B0B0F6907FA0AF747EA0B0786
:10593800C8F8207001E0032DDCD1076805FA0EF5E0
:1059480007EA0C073D4316F4403F056041D023F0B9
:10595800030707F1804707F5803703F0030CBD689C
:105968004FEA8C0C4FF0070E0EFA0CFEB0F1904F78
:1059780025EA0E0E2FD01B4DA8422ED005F58065C6
:10598800A8420CBF0225072505FA0CF545EA0E05C5
:10599800BD602568D74316F4801F0CBF3D401543F2
:1059A8002560656816F4001F0CBF3D40154365600F
:1059B800D4F8805016F4803F0CBF3D401543C4F81E
:1059C8008050D4F88450B60354BF3D401543C4F802
:1059D8008450013362E70025D6E70125D4E700BFEC
:1059E8000008005800040048374A2DE9F04F00230A
:1059F8004FF0010A4FF0070B4FF00F0931FA03F48B
:105A080001D1BDE8F08F0AFA03FC1CEA010654D064
:105A180023F0030404F1804404F5803403F0030701
:105A2800A568BF000BFA07F8B0F1904F08EA050E19
:105A380045D0264DA84244D005F58065A8420CBF44
:105A480002250725BD40754517D1D2F8805025EAB3
:105A58000605C2F88050D2F8845025EA0605C2F837
:105A68008450156825EA06051560556825EA060577
:105A78005560A56825EA0805A560056803265C0049
:105A880006FA04F423FA06F6254300EB86060560B9
:105A980003F00705376AAD0009FA05F527EA050797
:105AA8003762856825EA04058560456825EA0C059E
:105AB8004560C56825EA0404C46001339EE70025F3
:105AC800C0E70125BEE700BF0008005800040048F1
:105AD8000369194214BF0120002070470AB181618F
:105AE8007047816270470000044AD168014208B5D6
:105AF80002D0D060FDF7B0FC08BD00BF0008005818
:105B080003689A69910744BF00229A629A69D2078A
:105B18005EBF9A6942F001029A61704730B5039DF1
:105B280004682B4343EA0243064A6068C1F309014B
:105B38000B4342EA555223F0004320EA0200034394
:105B4800636030BDFF63FF0303682DE9F0419C6982
:105B580014F0100405460F4616466FD01022002494
:105B6800DA61A0462B689A69900661D4B8F1000FF3
:105B780035D044F0040401202E68B369D90541BF2B
:105B88004FF48072F26144F0010401205A0541BFCC
:105B98004FF4806244F00804F26101209B054FD560
:105BA8004FF4007344F00204F3612846FFF7A8FF9E
:105BB800736823F0FF7323F48B3323F4FF7323F00C
:105BC800010373606B6C23436B64202385F84130B9
:105BD800002385F8423085F84030012032E07A1CF5
:105BE800C1D0FCF75DFF801BB84201D8002FB9D1A6
:105BF8002B68596895F8422098690004D2B20AD5F2
:105C0800490408D4202A06D05A6842F480425A60CF
:105C1800FCF746FF06462B689B699B06A2D4FCF757
:105C28003FFF801B1928F6D920244FF0010899E777
:105C3800B8F1000F9DD12022DA619AE720469BE750
:105C48000028B2D1BDE8F08170B504460D4616466D
:105C580023689B699B0701D5002070BD3246294601
:105C68002046FFF771FFA0B96A1CF1D0FCF718FFB6
:105C7800801BA84201D8002DEAD1636C43F02003B1
:105C88006364202384F84130002384F8423084F888
:105C980040300120E1E770B504460D4616462368FA
:105CA8009B695B070ED4324629462046FFF74CFF16
:105CB80038BB23689A69910625D59A69520703D596
:105CC800228D0AB1002070BD9A6912F010021CBF23
:105CD8001022DA614FF0200118BF04226264D961F2
:105CE8005A6822F0FF7222F48B3222F4FF7222F0FB
:105CF80001025A60002384F8411084F8423084F885
:105D080040300120DFE7FCF7CBFE801BA84201D81A
:105D1800002DC4D1636C43F020036364202384F80E
:105D280041300023EBE72DE9F041069F0446884601
:105D380016461D462268936938EA03030CBF0123FF
:105D48000023B34201D0002015E06B1CF3D0FCF710
:105D5800A7FEC01BA84201D8002DEBD1636C43F00D
:105D680020036364202384F84130002384F8423000
:105D780084F840300120BDE8F08170B504460D4636
:105D8800164623689B699B0601D5002070BD3246E4
:105D980029462046FFF7D8FE90B9FCF781FE801B04
:105DA800A84201D8002DECD1636C43F02003636452
:105DB800202384F84130002384F8423084F84030AE
:105DC8000120E3E710B5044600284AD090F8413096
:105DD80003F0FF021BB980F84020FCF759FB24238D
:105DE80084F8413023681A6822F001021A60626858
:105DF80022F070621A619A6822F400429A60D4E92B
:105E08000221012924D142F400429A605A6842F0E2
:105E1800007242F400425A60DA6822F40042DA6002
:105E2800D4E904210A43A16942EA0122DA60D4E9EB
:105E380007210A431A601A6842F001021A6000201A
:105E48002023606484F84130206384F8420010BD48
:105E580042F4044202299A6004BF4FF400625A6077
:105E6800D4E70120F3E700002DE9F347984690F8BE
:105E780041300A9F202B04460E46914640F086800A
:105E880090F84030012B00F081804FF0010A80F833
:105E980040A0FCF705FE19230546009052464FF432
:105EA80000412046FFF73FFF18B1012002B0BDE8CE
:105EB800F087212384F84130102384F8423060644D
:105EC800A4F82A80638DC4F824909BB2FF2B6063EA
:105ED8002F4B26D9FF22228500934FF0807331463D
:105EE8002046FFF71BFE638D9BB22A4639462046A3
:105EF800FBB9FFF742FF0028D7D123682021D961D9
:105F08005A6822F0FF7222F48B3222F4FF7222F0D8
:105F180001025A6084F8411084F8400084F8420075
:105F2800C4E7628D009392B222854FF00073D2B21B
:105F3800D5E7FFF789FE0028B7D1636A226813F80E
:105F4800011B91626362638D228D013B9BB2638565
:105F5800638D013A92B29BB22285002BC3D0002AEE
:105F6800C1D100953B4680212046FFF7DCFE002882
:105F78009BD1638D9BB2FF2B03D9FF222285009012
:105F8800ABE7628D009092B22285CEE702208DE7C2
:105F9800002000802DE9F347984690F841300A9F89
:105FA800202B04460E46914640F0878090F84030FA
:105FB800012B00F082804FF0010A80F840A0FCF726
:105FC8006FFD19230546009052464FF400412046C4
:105FD800FFF7A9FE18B1012002B0BDE8F08722231F
:105FE80084F84130102384F842306064A4F82A8091
:105FF800638DC4F824909BB2FF2B6063304B26D985
:10600800FF22228500934FF0807331462046FFF728
:1060180085FD638D9BB22A4639462046FBB9FFF7BA
:10602800ACFE0028D7D123682021D9615A6822F014
:10603800FF7222F48B3222F4FF7222F001025A60BE
:1060480084F8411084F8400084F84200C4E7628D67
:10605800009392B222854FF00073D2B2D5E7FFF7D2
:106068001AFE0028B7D123685A6A636A1A70636AED
:10607800228D01336362638D013B9BB26385638D1F
:10608800013A92B29BB22285002BC2D0002AC0D11D
:1060980000953B4680212046FFF745FE00289AD10F
:1060A800638D9BB2FF2B03D9FF2222850090AAE7BC
:1060B800628D009092B22285CDE702208CE700BF66
:1060C8000024008010B590F84120202A0346D4B25D
:1060D8001CD190F84020012A18D0242280F84120B1
:1060E8000268106820F001001060106820F48050E9
:1060F80010601068014311601168002041F001012F
:10610800116083F8414083F8400010BD0220FCE78D
:1061180010B590F84120202A0346D4B21BD190F83C
:106128004020012A17D0242280F8412002681068F4
:1061380020F001001060106820F4706040EA01212E
:1061480011601168002041F00101116083F841409D
:1061580083F8400010BD0220FCE70000024A1368E3
:1061680043F4807313607047000400580D4B10B55A
:106178005B690C4628B99A0507D500F027F820B1C5
:1061880010BD9B0501D400F019F8074A1369012CCA
:1061980023F00403136101D130BFF1E740BF20BFF2
:1061A80020BFEDE70004005800ED00E0024B18683E
:1061B80000F4C060704700BF00040058024A13682A
:1061C80043F4804313607047000400580C4A136876
:1061D80023F4804313600B4B1B6832214B430A495D
:1061E800B3FBF1F35169890500D533B9536913F449
:1061F800007F14BF032000207047013BF2E700BF77
:10620800000400586805002040420F000B4A13683C
:1062180023F0070343F002031360094B1A690128AE
:1062280042F004021A6105D130BF1A6922F0040253
:106238001A61704740BF20BF20BFF6E7000400582E
:1062480000ED00E04FF0B0431868C0F340407047DD
:106258004FF0B0431868C0F3400070474FF0B042A9
:10626800536823F47F4343EA0023536070474FF099
:10627800B0431868C0F34060704700007FB54FF026
:10628800B0432C4AD3F80831C0F3031003F00F03CE
:1062980052F82040284A52F82330B4FBF3F4FFF7B1
:1062A80085FF264B054693E80700B5F5007F04AB4C
:1062B80003E9070010D0224B9C4218D303F5B7031B
:1062C80003F67F539C4229D903F5741303F5106331
:1062D8009C4225D802230BE01A4B9C4207D91A4B43
:1062E8009C421BD903F5370303F5D853F0E7002385
:1062F80004AA02EB830353F80C4C144D2B6823F0CB
:10630800070323432B60FCF7CBFB06462B6803F0FF
:1063180007039C4206D1002004B070BD0123E7E7C3
:106328000024EAE7FCF7BCFB801B0228EED9032017
:10633800F2E700BFB41A0108541A010850190108FD
:10634800C0CF6A00BFEA21013F93340200400058E1
:106358004FF0B04310B59A68D96812F00C0205D016
:106368000C2A4AD101F00303012B50D14FF0B04160
:106378002B480B6813F0080306D00B6813F00803CA
:1063880037D1D1F8941007E00C68240756BFD1F82C
:1063980094300968C3F3032350F82330002A0CBF54
:1063A800184600204FF0B0418A6802F00C020C2A0F
:1063B8001ED1CA6802F00302022A2ED0032A06D18F
:1063C8000B68184A13F4801F174B18BF13464FF079
:1063D800B042D068D168D268C0F306205843C1F3F0
:1063E80002130133B0FBF3F0530F0133B0FBF3F0AA
:1063F80010BD0B68C3F30313CEE7042A0AD0082A9A
:1064080005D11B6813F4801304D10748CAE7002399
:106418001846C7E703480023C4E7024BD7E700BF85
:10642800B41A01080024F4000048E80108B5FFF791
:106438008FFF4FF0B043044A9B68C3F3031352F82D
:106448002330B0FBF3F008BD541A01082DE9F041E0
:106458000446002853D04FF0B0439D68DE680368B7
:106468009B0605F00C0506F0030668D5026A1DB107
:106478000C2D46D1012E44D1002A40D04FF0B04314
:10648800A16A1A68170756BFD3F894301B681B090E
:1064980003F0F00399421FD90846FFF7EFFE0028E2
:1064A8002DD14FF0B042136843F00803136013680E
:1064B800A16A23F0F0030B431360606AFFF7CEFE76
:1064C800FFF7B4FFAB4B1860AB4B1868FCF7E6FA64
:1064D800002834D0BDE8F0814FF0B042136843F093
:1064E80008031360136823F0F0030B431360606A1A
:1064F800FFF7B4FE0846FFF7C1FE0028E0D00120F0
:10650800E8E74FF0B043002A54D01A6842F001027D
:106518001A60FCF7C5FA0746FFF79AFE002842D032
:106528004FF0B042136843F0080313601368A16A80
:1065380023F0F0030B431360606AFFF78FFE2368B4
:10654800D80748D42368990700F18C8023681E0770
:1065580040F1FA80A3694FF0B046002B00F0E180CB
:10656800D6F89430E16903F01002914200F0C4803B
:1065780003F00302022AC2D0D80740F1B380D6F84C
:10658800943023F00103C6F89430FCF789FA0746E3
:10659800D6F89430990740F1A580FCF781FAC31B1F
:1065A800112BF5D904E0FCF77BFAC01B0228B3D9FC
:1065B80003208FE71A6822F001021A60FCF770FACC
:1065C8000746FFF745FE0028B9D0FCF769FAC01B5B
:1065D8000228F6D9ECE7082D03D00C2D05D1032E9F
:1065E80003D16368002BADD189E74FF0B043A168B0
:1065F8001A6822F480120A431A606268B2F5803F72
:1066080010D11A6842F480321A60FCF749FA07463A
:10661800FFF718FE002895D1FCF742FAC01B642842
:10662800F6D9C5E7B2F5041F04D11A6842F400127E
:106638001A60E6E7196821F480311960196821F4B5
:1066480000111960002AE0D1FCF72AFA0746FFF783
:10665800F9FD00283FF476AFFCF722FAC01B642846
:10666800F5D9A5E7042D236903D00C2D0ED1022EF0
:106678000CD1002B3FF443AF4FF0B042616953682F
:1066880023F0FE4343EA016353605FE74FF0B046EF
:10669800BBB1336843F480733360FCF701FA0746F3
:1066A80033685A0507D57368626923F0FE4343EAE5
:1066B800026373604AE7FCF7F3F9C31B022BEFD9B7
:1066C80076E7336823F480733360FCF7E9F907460B
:1066D80033685B057FF53AAFFCF7E2F9C31B022B81
:1066E800F6D965E74FF0B042E169D2F8943023F06B
:1066F80010030B43C2F894304FF0B047D7F89430EA
:1067080043F00103C7F89430FCF7CAF90646D7F8F6
:1067180094309A0718D4FCF7C3F9831B112BF6D9C8
:1067280046E7D6F8943023F00103C6F89430FCF716
:10673800B7F90746D6F894309B0705D5FCF7B0F9AA
:10674800C31B112BF6D933E72368580754D50B4FD1
:106758003B68D90514D4FFF701FDFCF7A1F90646FB
:106768003B68DA050CD4FCF79BF9831B022BF7D99D
:106778001EE700BF680500206C05002000040058D3
:10678800E3684FF0B046002B58D023F08003052B68
:1067980002BFD6F8903043F00403C6F890304FF0AB
:1067A800B046FCF77DF9D6F8903043F00103074670
:1067B800C6F8903041F28838D6F890309B0705D457
:1067C800FCF76EF9C31B4345F6D9F1E6E36823F0FD
:1067D8000403812B1BD1FCF763F9D6F8903043F002
:1067E8008003C6F8903007464FF0B04641F288382B
:1067F800D6F89030180504D5E06A00284AD1002060
:1068080068E6FCF74DF9C01B4045F1D9D0E6FCF726
:1068180047F9D6F8903023F08003C6F89030074641
:106828004FF0B04641F28838D6F890301905E3D5D4
:10683800FCF736F9C01B4045F6D9B9E6FCF730F944
:10684800D6F8903023F080030746C6F8903041F21E
:106858008838D6F890301A0516D4FCF721F9D6F8FE
:10686800903023F00103C6F8903007464FF0B04847
:1068780041F28836D8F890309B07BDD5FCF710F95F
:10688800C31BB342F6D993E6FCF70AF9C01B40458F
:10689800DFD98DE60C2D4ED04FF0B04302281A6890
:1068A80022F080721A6033D1FCF7FAF80546FFF738
:1068B800DEFC38BBD4E90C314FF0B0420B43D06852
:1068C8002D4901400B43E16B0B43216C0B43616C79
:1068D8000B43A16B43EA0123D360136843F0807331
:1068E8001360D36843F08053D360FCF7D9F80446AB
:1068F800FFF7BDFC002882D1FCF7D2F8001B0A285C
:10690800F6D955E6FCF7CCF8401B0A28CFD94FE654
:10691800FCF7C6F80446FFF7AAFC30B94FF0B042BE
:10692800164BD1680B40D360D4E5FCF7B9F8001BCF
:106938000A28F0D93CE601283FF4CCAD4FF0B0432B
:10694800226BDB6803F0030191427FF4D8AD616BE1
:1069580003F070028A427FF4D2ADA16B03F4FE42C9
:10696800B2EB012F7FF4CBAD626C03F0604393422E
:106978003FF445AFC3E500BF8C80C111FCFFFEEEBC
:106988002DE9F0410D46044610B90120BDE8F0811B
:10699800684E336803F007038B4216D323689A07BF
:1069A80027D54FF0B047A268BB6823F0F003134324
:1069B800BB60FCF775F80646BB68DB0319D4FCF727
:1069C8006FF8831B022BF7D911E0336823F0070314
:1069D8000B433360FCF764F80746336803F007039A
:1069E800AB42DBD0FCF75CF8C01B0228F5D90320CA
:1069F800CCE72368580617D54FF0B0476269D7F837
:106A0800083123F00F0343EA1213C7F80831FCF7E3
:106A180047F80646D7F80831D90305D4FCF740F8FB
:106A2800831B022BF6D9E2E723685A0713D54FF0E8
:106A3800B047E268BB6823F4E0631343BB60FCF72C
:106A48002FF80646BB689B0305D4FCF729F8831B7F
:106A5800022BF7D9CBE72368180714D54FF0B047B6
:106A68002269BB6823F4605343EAC203BB60FCF7A6
:106A780017F80646BB68590305D4FCF711F8831BC1
:106A8800022BF7D9B3E72368DA070FD4294C236818
:106A980003F00703AB4239D8FFF7C8FC264B186050
:106AA800264BBDE8F0411868FBF7F8BF6268022A78
:106AB8001DD1FFF7C7FB00283FF467AF4FF0B04682
:106AC80041F28838B36823F003031343B360FBF73C
:106AD800E7FF0746B368626803F00C03B3EB820F65
:106AE800D4D0FBF7DDFFC01B4045F3D97FE7032A6D
:106AF80002D1FFF7BCFBDEE712B9FFF7A9FBDAE723
:106B08004FF0B0431B685B05D8D43EE7236823F0F9
:106B180007032B432360FBF7C3FF0646236803F0F4
:106B28000703AB42B8D0FBF7BBFF801B0228F5D99F
:106B38005DE700BF00400058680500206C05002094
:106B480008B5FFF773FC4FF0B043044A9B68C3F3E2
:106B5800022352F82330D84008BD00BF941A010818
:106B680008B5FFF763FC4FF0B043044A9B68C3F3D2
:106B7800C22352F82330D84008BD00BF941A010838
:106B88004FF0B043D3F89000C0F3400070474FF087
:106B9800B0410209D1F8883002F47F22000123EACB
:106BA800020300F47F200343C1F8883070474FF098
:106BB800B041020CD1F88830120423EA020343EAF8
:106BC8000040C1F88800704770B5066816F4803632
:106BD800044638D0FFF7C2FAFBF762FF614E05465C
:106BE8003368DB0529D54FF0B043616BD3F89020AB
:106BF80002F44072914214D0D3F89010D3F8902048
:106C080042F48032C3F89020D3F8902021F44070E9
:106C180022F480328D07C3F89020C3F8900000F169
:106C280090804FF0B042616BD2F8903023F44073FB
:106C38000B43C2F89030002605E0FBF731FF401BFC
:106C48000228CDD903262568E8070AD54FF0B041B8
:106C58006268D1F8883023EA124392B21343C1F82C
:106C68008830A9070AD54FF0B041A268D1F888301A
:106C780023EA124392B21343C1F88830AA0609D511
:106C88004FF0B0422169D2F8883023F440630B43B7
:106C9800C2F88830AB0502D5206AFFF788FF68057F
:106CA80002D5606AFFF783FF290502D5A06AFFF7BE
:106CB8007EFF6A0602D56069FFF769FF2B0602D5D9
:106CC800A069FFF764FFE80502D5E069FFF75FFFF9
:106CD800E90610D54FF0B042E168D2F8883023F4C5
:106CE80040730B43C2F88830B1F5807F02BFD36888
:106CF80043F08073D3602A040ED54FF0B042216B65
:106D0800D2F8883023F040430B43C2F8883019B9D1
:106D1800D36843F08073D3606B0410D54FF0B04252
:106D2800E16AD2F8883023F040530B43B1F1005F99
:106D3800C2F8883003D1D36843F48033D360304637
:106D480070BDFBF7ADFE41F288360546FFF718FF28
:106D580001283FF466AFFBF7A3FE401BB042F5D90C
:106D680070E700BF0004005830B590F82C30012BB4
:106D780002464FF0020022D0174B82F82D00CA2499
:106D8800012582F82C505C6253245C62B1F5807F47
:106D9800146B996914D121F488519961596C24F0C4
:106DA800010421F0004159641463DD650A4BFF2199
:106DB80059620020012382F82D3082F82C0030BD62
:106DC80021F408519961D96C24F0020421F00041A2
:106DD800D9641463D865E9E70028004070B50B4E04
:106DE800036B756D1D40EA07044603D50123F3655F
:106DF800FBF7C7FFAB0704D50223F365204600F075
:106E0800CBF9012384F82D3070BD00BF0028004065
:106E180038B50A4CE36823F02003E360FBF740FE33
:106E28000546E3689B0601D5002038BDFBF738FE10
:106E3800401BB0F57A7FF4D90320F6E7002800401C
:106E48002DE9F041114DEC6814F0400407461AD1C1
:106E5800EB6843F08003EB60FBF722FE4FF003087A
:106E68000646EB685B0601D4032C02D12046BDE838
:106E7800F081FBF715FE801BB0F57A7F84BF87F899
:106E88002D800324EDE70024F0E700BF0028004030
:106E980038B50F4CE36823F08003E360A3699B06D1
:106EA800054606D4FFF7B4FF10B1032085F82D007E
:106EB80038BDA36923F02003A361FFF7A9FF10B130
:106EC800032085F82D00A36943F02003A361EFE7B1
:106ED8000028004038B5044600284BD090F82D30E3
:106EE80003F0FF021BB980F82C20FBF7E1FB02231B
:106EF800214D84F82D30EB68DB0632D4CA236B624F
:106F080053236B622046FFF79BFF78BBAB6923F0E6
:106F18008E6323F04003AB6121696368AA690B4360
:106F28001343A2691343AB61D4E9022343EA024342
:106F38002B61D4E90931EA680B4322F4F852134370
:106F4800EB602046FFF7A4FF80B9D4E90713AA69CC
:106F58000B4322F06042134362691343AB61FF2382
:106F68006B62012384F82D30002002E0024BFF22DF
:106F78005A6238BD0120FCE7002800400023092898
:106F880003D840EA0310C0B270470A380133C0B2D0
:106F9800F5E700002DE9F04790F82C30012B054665
:106FA8004FF0020069D0012385F82C304E4B85F84C
:106FB8002D00DE6806F44076B6F5807F78D04C69FF
:106FC800087891F8019091F802A091F82470002AAD
:106FD80055D19B6913F0400308BFCB70FFF7CEFF74
:106FE80080464846FFF7CAFF02465046FFF7C6FFED
:106FF80081463846FFF7C2FF0B6ACF78234343EA3E
:10700800875343EA090343EA084343EA022343EA6E
:107018000063354ACA205062532050628C6A8869DE
:10702800B4F5807F946945D124F48854946101248F
:10703800D465B6F5807F09BFCB69136403435364F5
:1070480018BF5064284B4A681A672A6B42F001023D
:107058002A639A6942F488529A61244AD2F88030A5
:1070680043F40033C2F880301F4BFF225A620020DD
:10707800012385F82D3085F82C00BDE8F087B4F1A0
:10708800803F07D0B4F5000F04D09B6913F040038C
:1070980008BFCB700B6ACA781C4344EA0A0444EA66
:1070A800004343EA092343EA825343EA0763B0E70C
:1070B8000023AEE724F4085494610224D465B6F59D
:1070C800807F09BFCB6993640343D36418BFD0643E
:1070D800054B4A685A672A6B42F002022A639A698A
:1070E80042F40852B8E700BF0028004000080058E2
:1070F80090F82C20012A03464FF0020012D00A4AC9
:1071080083F82D00CA21516253215162916941F0DF
:1071180020019161FF2151620020012283F82D2076
:1071280083F82C00704700BF0028004090F82C20FE
:10713800012A03464FF0020019D00D4A83F82D00AA
:10714800CA2151625321516291690A4841F0800174
:107158009161D0F8801041F48021C0F88010FF219F
:1071680051620020012283F82D2083F82C007047FB
:107178000028004000080058064B5A6D520610B50A
:10718800044603D54022DA65FBF7FEFD012384F8A7
:107198002D3010BD002800407047890001F1804162
:1071A80001F531410A607047890001F1804101F51C
:1071B8003141086870470000034AD2F8903043F420
:1071C8000043C2F89030704700040058034AD2F8D0
:1071D800903023F40043C2F8903070470004005800
:1071E800074B1A6822F040021A6040F441704FF4CD
:1071F800B85218605A601A6842F040021A60704724
:107208000000015837B5054600284ED0837903F0B1
:10721800FF046BB1032C0BD0254B4FF400629A612D
:107228002868FFF7DDFF002401232B71AC602FE0F5
:1072380000236B712846FBF74BFB1E4AD2F89030AF
:1072480043F48053C2F89030002CE5D102234FF06C
:10725800B042AB71D2F8943023F40043C2F89430B2
:10726800154B1B681C214B43DB0C64214B430193DA
:10727800019B93B90124AC60FFF79EFF0C4B9A6801
:1072880042F400629A604FF400629A61002CC7D001
:107298000123AB71204603B030BD019B013B019334
:1072A800D2F894305B04E3D4E6E70124F2E700BFA8
:1072B80000040058000800586805002037B5174D2D
:1072C8002B6802461C204343DB0C642043431448CC
:1072D8000193019B93B901209060114C21732B6895
:1072E8001C214B43DB0C64214B430193019B6BB97D
:1072F800012090600A4BDB6803B030BD019B013B65
:10730800019383689C07E4D50020E6E7019B013BD5
:107318000193A368DB07E9D5ECE700BF6805002007
:107328000000015837B5184D2B6802461C2043430E
:10733800DB0C6420434315480193019BA3B901204A
:107348009060124CFF2323732B681C256B43DB0CC6
:1073580064256B430193019B73B9012090600B4B2B
:10736800DB680B7003B030BD019B013B0193836860
:107378009C07E2D50020E4E7019B013B0193A36849
:10738800DB07E8D5EBE700BF6805002000000158DF
:107398000F4B13B51B680F4C182253431B0D642267
:1073A8005343014601936269019B02F0040223B929
:1073B80002238B60012002B010BD019B013B0193A9
:1073C800606910F00200F6D0002AECD11046F2E70E
:1073D800680500200004005807B50379012B0FD178
:1073E8000A4B1B68182253431B0C0193FFF7EEFE50
:1073F800019B013B0193019B002BF9D1FFF7DCFEB8
:1074080003B05DF804EBFFF7C3BF00BF68050020B9
:10741800F8B51E468379012B154604460F46DAB2A5
:107428002DD14379012B2AD0022342718371FFF7B2
:10743800D3FF0D212046FFF7C9FEFFF73FFF390AAA
:107448002046FFF73BFFF9B22046FFF737FF2E44EF
:10745800B5420ED12046FFF7AFFEFFF799FFA068AF
:1074680001230038A3714FF0000318BF0120637196
:10747800F8BD15F8011B2046FFF720FFE8E70220BA
:10748800F6E7F8B51E468379012B154604460F46E4
:10749800DAB22FD14379012B2CD04271FFF79CFF30
:1074A8001D212046FFF792FEFFF708FF390A204604
:1074B800FFF704FFF9B22046FFF700FF002120463E
:1074C800FFF7FCFE2E44B5420ED12046FFF774FEAE
:1074D800FFF75EFFA06801230038A3714FF0000397
:1074E80018BF01206371F8BD29462046FFF71AFF2F
:1074F8000135E8E70220F6E7F8B51F468379012B46
:10750800154604460E46DAB22CD14379012B29D010
:107518004271FFF761FF06F0EF03A3F184025342C3
:107528005341237131462046FFF750FEFFF7C6FE50
:107538002F44AF4210D1FFF73FFE842E02D02046E1
:10754800FFF726FFA06801230038A3714FF000035E
:1075580018BF01206371F8BD15F8011B2046FFF71D
:10756800ADFEE6E70220F6E7F8B51E468379012B63
:10757800154604460F46DAB227D14379012B24D0A9
:107588004271FFF729FF39462046FFF71FFEFFF734
:1075980095FE00212046FFF791FE2E44B5420ED1FC
:1075A8002046FFF709FEFFF7F3FEA0680123003825
:1075B800A3714FF0000318BF01206371F8BD29467D
:1075C8002046FFF7AFFE0135E8E70220F6E737B5BA
:1075D8000023ADF8043001AA022312210546FFF763
:1075E800C3FFBDF80440022364BA01AAA4B2194635
:1075F8002846FFF781FFE20702D5284609F02AFA54
:10760800A30702D5284609F02BFA600702D52846B9
:1076180009F050FA210702D5284609F051FAE20686
:1076280002D5284609F052FAA30602D5284609F0E1
:107638003BFA600602D5284609F018FA210606D555
:1076480014F4807118BF0121284609F015FAA20523
:1076580002D5284609F020FA630402D5284609F025
:107668003BFA03B030BDF8B51E468379012B1546A9
:1076780004460F46DAB227D14379012B24D0427150
:10768800FFF7AAFE0E212046FFF7A0FDFFF716FE22
:1076980039462046FFF712FE2E44B5420ED1204649
:1076A800FFF78AFDFFF774FEA06801230038A37175
:1076B8004FF0000318BF01206371F8BD15F8011BD6
:1076C8002046FFF7FBFDE8E70220F6E7F8B51E467F
:1076D8008379012B154604460F46DAB22BD143793C
:1076E800012B28D04271FFF777FE1E212046FFF7B5
:1076F8006DFDFFF7E3FD39462046FFF7DFFD00216A
:107708002046FFF7DBFD2E44B5420ED12046FFF799
:1077180053FDFFF73DFEA06801230038A3714FF029
:10772800000318BF01206371F8BD29462046FFF702
:10773800F9FD0135E8E70220F6E7026852E8003F64
:1077480023F0C00342E8003102680029F5D102F1B4
:10775800080353E8003F23F4000302F1080C4CE847
:1077680000310029F3D12023C0F888307047000089
:1077780010B5026852E8003F23F4907342E80031E4
:1077880002680029F5D10F4C02F1080353E8003FC5
:10779800234002F1080C4CE800310029F4D1C36EF3
:1077A800012B07D152E8003F23F0100342E80031D3
:1077B8000029F7D12023C0F88C300023C366436723
:1077C80010BD00BFFEFFFFEFF8B504461346D4F81E
:1077D8008850202D32D1F1B1EAB1E06FA4F85620DB
:1077E800A4F8542000262122C4F890602165C4F82A
:1077F8008820226888B1124FC762124F0763124F60
:107808002832C0E90D76FDF745FE30B11023C4F8E3
:107818009030C4F8885001200FE0236840221A6293
:10782800226802F1080353E8003F43F0800302F1A5
:10783800080141E800300028F3D1F8BD0220FCE738
:10784800557800089D780008A978000808B503460F
:10785800806A1B681B6813F0200317D1A0F8563004
:10786800026802F1080353E8003F23F0800308325E
:1078780042E8003102680029F2D152E8003F43F0A3
:10788800400342E800310029F7D108BDFBF7D2FBDD
:10789800FBE7704708B5806AFFF7FBFF08BD704734
:1078A800806A38B50468D0F88830D0F88C50A2685F
:1078B800120606D5212B04D10023A0F85630FFF775
:1078C8003CFFA3685B0606D5222D04D10023A0F84F
:1078D8005E30FFF74DFFD0F8903043F01003C0F84A
:1078E8009030FFF7DCFF38BD08B5806A0023A0F8A8
:1078F8005E30A0F85630FFF7D2FF08BD7047000091
:107908000368D9691A682DE9F04140F60F0631423B
:107918009D68044610D18E0640F1978002F020063B
:1079280005F080573E4300F09080436F002B00F035
:107938008580BDE8F0411847AB4EAC482E4010405A
:10794800304300F08280CF0709D5D00507D5012044
:107958001862D4F8900040F00100C4F890008F0736
:1079680009D5E80707D502201862D4F8900040F03E
:107978000400C4F890004F0709D5E80707D504208C
:107988001862D4F8900040F00200C4F890000F0785
:107998000BD502F02000304307D008201862D4F835
:1079A800900040F00800C4F890000E050AD5500178
:1079B80008D54FF400601862D4F8903043F02003E3
:1079C800C4F89030D4F89030002B37D08B0609D506
:1079D80002F0200205F080552A4303D0636F0BB1F3
:1079E800204698472668D4F89020B36802F0280209
:1079F80003F0400353EA0205204621D0FFF7B8FE02
:107A0800B3685F0617D5226802F1080353E8003F00
:107A180023F04003083242E800310029F3D1D4F8BA
:107A2800800040B1724B8363FDF7ADFD30B1D4F8EF
:107A38008000836B7DE72046FFF731FFBDE8F081CA
:107A4800FFF72DFFC4F89050F8E7E06E012840F0EA
:107A58008980CE0640F18680D00640F183801022CE
:107A68001A629A6851064BD5D4F8802011684A6882
:107A780092B2002AE2D0B4F85C009042DED9A4F8B1
:107A88005E200A6892062FD453E8002F22F48072F1
:107A980043E800210029F7D103F1080252E8002F3A
:107AA80022F0010203F1080040E800210029F3D187
:107AB80003F1080252E8002F22F0400203F1080007
:107AC80040E800210029F3D12022C4F88C20E16687
:107AD80053E8002F22F0100243E800210029F7D1D3
:107AE800D4F88000FDF71AFD02232367B4F85E304E
:107AF800B4F85C10C91A89B22046FFF7FFFE9DE76B
:107B0800B4F85E20B4F85E00B4F85C1080B292B2AB
:107B1800002893D0891A89B200298FD053E8002F02
:107B280022F4907243E800200028F7D1314D03F188
:107B3800080252E8002F2A4003F1080646E8002010
:107B48000028F4D12022C4F88C206067E06653E84E
:107B5800002F22F0100243E800200028F7D102236A
:107B68002367C9E7CF0209D56E0207D54FF4801203
:107B780020461A62BDE8F04100F0A0BD08060BD50A
:107B880002F0800005F40005284305D0A36F002B00
:107B98003FF454AF2046CCE64F0611D556060FD514
:107BA80053E8002F22F0400243E800210029F7D1D2
:107BB8002023C4F88830A1672046FBF73BFA3DE74D
:107BC8000D0206D5500004D52046BDE8F04100F06E
:107BD80077BDCB017FF532AF002ABFF62FAF204625
:107BE800BDE8F04100F06BBD010000102001000469
:107BF800F1780008FEFFFFEFD0F88C20B0F8601095
:107C0800222A08B5036855D15B6A826D0B40137050
:107C1800836D01338365B0F85E30013B9BB2A0F8F9
:107C28005E30B0F85E309BB2002B42D1026852E859
:107C3800003F23F4907342E8003103680029F5D12E
:107C480003F1080252E8002F22F0010203F1080CA8
:107C58004CE800210029F3D12022C0F88C20184AD2
:107C680041679342016705D1C26E012A0ED0FBF726
:107C7800EFF91EE05A681102F6D553E8002F22F0FA
:107C8800806243E800210029F7D1EDE70022C266AF
:107C980053E8002F22F0100243E800210029F7D111
:107CA800DA69B0F85C10D20644BF10221A62FFF7F6
:107CB80025FE08BD9A6942F008029A61F9E700BFFB
:107CC80000800040D0F88C20B0F86010222A08B557
:107CD800036852D15A6A1140826D22F8021B8265EC
:107CE800B0F85E20013A92B2A0F85E20B0F85E20AB
:107CF80092B2002A40D153E8002F22F4907243E850
:107D080000210029F7D103F1080252E8002F22F0E0
:107D1800010203F1080C4CE800210029F3D12022CC
:107D2800C0F88C20174A41679342016705D1C26E9B
:107D3800012A0ED0FBF78CF91EE05A681102F6D51D
:107D480053E8002F22F0806243E800210029F7D190
:107D5800EDE70022C26653E8002F22F0100243E844
:107D680000210029F7D1DA69B0F85C10D20644BFC7
:107D780010221A62FFF7C2FD08BD9A6942F0080294
:107D88009A61F9E7008000402DE9F74F0368B0F8E1
:107D98006080DF691A689D68D0F88C1001922229EA
:107DA800044640F0B480B0F86890DFF86CA1DFF8C2
:107DB8006CB10026B9F1000F01D0BB0621D4B4F88C
:107DC8005E309BB2D3B1B4F868209A4216D92268C3
:107DD80002F1080353E8003F23F08053083242E8D9
:107DE800003122680029F2D14D4B636752E8003F09
:107DF80043F0200342E800310029F7D103B0BDE881
:107E0800F08F2368A26D5B6A03EA08031370A36D01
:107E18000133A365B4F85E30013B9BB2A4F85E3031
:107E28002368DF6978072CD0F9070AD5019AD205AB
:107E380007D501211962D4F8901041F00101C4F866
:107E48009010B80709D5E90707D502211962D4F8B7
:107E5800901041F00401C4F890107A0709D5E8079A
:107E680007D504211962D4F8903043F00203C4F80E
:107E78009030D4F8903023B12046FFF710FDC4F8B5
:107E88009060B4F85E309BB2002B93D1216851E822
:107E9800003F23F4807341E8003023680028F5D1BF
:107EA80003F1080252E8001F01EA0A0142E8001043
:107EB8000028F5D120215B45C4F88C106067206745
:107EC8000AD05968090207D553E8001F21F08061DC
:107ED80043E800100028F7D1E16E012913D1E666C6
:107EE80053E8001F21F0100143E800100028F7D1E3
:107EF800D969CA0644BF102119622046B4F85C103B
:107F0800FFF7FCFC56E72046FBF7A2F852E79A6910
:107F180042F008029A6171E7FEFFFFEF008000401F
:107F2800017C00082DE9F74F0368B0F86080DF692D
:107F38001A689D68D0F88C1001922229044640F0F6
:107F4800B280B0F86890DFF868A1DFF868B1002661
:107F5800B9F1000F01D0BB0621D4B4F85E309BB252
:107F6800D3B1B4F868209A4216D9226802F10803FE
:107F780053E8003F23F08053083242E8003122687A
:107F88000029F2D14C4B636752E8003F43F02003CD
:107F980042E800310029F7D103B0BDE8F08F23682B
:107FA800A26D596A08EA010122F8021BA265B4F819
:107FB8005E20013A92B2A4F85E20DF6978072CD0DF
:107FC800F9070AD5019AD20507D501211962D4F813
:107FD800901041F00101C4F89010B80709D5E907DD
:107FE80007D502211962D4F8901041F00401C4F8B1
:107FF80090107A0709D5E80707D504211962D4F843
:10800800903043F00203C4F89030D4F8903023B194
:108018002046FFF744FCC4F89060B4F85E309BB289
:10802800002B95D1216851E8003F23F4807341E883
:10803800003023680028F5D103F1080252E8001F38
:1080480001EA0A0142E800100028F5D120215B4529
:10805800C4F88C10606720670AD05968090207D5F0
:1080680053E8001F21F0806143E800100028F7D191
:10807800E16E012913D1E66653E8001F21F01001D3
:1080880043E800100028F7D1D969CA0644BF102177
:1080980019622046B4F85C10FFF730FC58E7204618
:1080A800FAF7D6FF54E79A6942F008029A6173E733
:1080B800FEFFFFEF00800040CD7C000838B5044685
:1080C80003682169A2681D68C0690A4361690A4397
:1080D8007D49024329400A431A605A68E16822F43C
:1080E80040520A435A60794AA16993421CBF226AE6
:1080F80011439A6822F06E4222F430620A439A6071
:10810800DA6A616A22F00F020A43DA62704A93421D
:108118001CD14FF0B043D3F8883003F0030343F485
:108128004033A3F54033013B022B00F2C780694A74
:108138009B5CB0F5004F40F08980082B24D8DFE81D
:1081480003F061C08323802323236500624A93429E
:1081580009D14FF0B043614AD3F8883003F00C03DB
:1081680043F44023E4E7594A93420DD14FF0B0431A
:10817800D3F8883003F44063B3F5006F1AD005D8FC
:1081880053B1B3F5806F12D0012009E0B3F5406F09
:10819800FAD14FF400400EE0FEF7D2FC58B90020A7
:1081A8004FF00113A3660023C4E91D3338BDFEF761
:1081B800CFF8F3E74A4865684A4B626A05EB450120
:1081C80033F81220B0FBF2F39942DDD8B3EB053F48
:1081D800DAD800231946F9F797FC090241EA106139
:1081E8006B080002C0182A464FF0000341F1000155
:1081F800F9F78AFC3C4BA0F540729A42C4D8236830
:10820800D860CCE7FEF79CFC0028C8D06168354BE5
:10821800626A33F81220B0FBF2F24B0803EB420318
:108228004FF6EF72B3FBF1F3A3F110019142ABD813
:1082380023F00F02216892B2C3F342031343CB60C9
:10824800ADE7FEF785F8DFE72548DFE7082B9BD881
:1082580001A252F823F000BFA9820008B5820008E5
:10826800C182000891810008BB8200089181000842
:108278009181000891810008858200084FF4004030
:108288006368616A174A32F81120B0FBF2F000EB1C
:108298005300B0FBF3F04FF6EF73A0F11002ACE718
:1082A800FEF74EFC00283FF47AAFE9E7FEF758FCEA
:1082B800F8E7FEF74DF8F5E70948E1E7B0F5004FB4
:1082C800F4D1FEF74DFC9FE7F369FFCF0080004033
:1082D80000380140F41A010800440040F71AF50775
:1082E8000024F400041B0108FFFC0F00836ADA076E
:1082F80010B506D50168C46A4A6822F400322243E0
:108308004A609C0706D50168046B4A6822F48032EB
:1083180022434A60590706D50168446B4A6822F42B
:10832800802222434A601A0706D50168846B4A688E
:1083380022F4004222434A60DC0606D50168C46B79
:108348008A6822F4805222438A60990606D5016819
:10835800046C8A6822F4005222438A605A060FD5B8
:108368000168446C4A6822F480122243B4F5801FE5
:108378004A6005D14A68846C22F4C00222434A60EC
:108388001B0606D50268C16C536823F400230B430F
:10839800536010BD2DE9F041DDF8188004460E4603
:1083A80015461F462268D36936EA03030CBF01232A
:1083B8000023AB4201D0002027E0B8F1FF3FF2D004
:1083C800FAF76EFBC01B4045206802D8B8F1000FD1
:1083D8001DD150E8003F23F4D07340E80032002A52
:1083E800F7D100F1080353E8003F23F0010300F13F
:1083F800080141E80032002AF3D12023C4F888306C
:10840800C4F88C3084F884200320BDE8F081036828
:108418005A07C7D5C3691B05C4D54FF40063036267
:1084280050E8003F23F4D07340E80032002AF7D127
:1084380000F1080353E8003F23F0010300F10801AD
:1084480041E80032002AF3D12023C4F88830C4F868
:108458008C30C4F89030D5E773B504460026C0F8D0
:108468009060FAF71DFB23681B681A07054619D4A4
:1084780023681B685B070AD56FF07E4300930022D0
:108488002B464FF480012046FFF784FFB0B9002047
:108498002023C4F8883084F88400C4F88C30E0665F
:1084A80020670CE06FF07E430093324603464FF49A
:1084B80000112046FFF76EFF0028D9D0032002B034
:1084C80070BD10B5044650B3D0F888301BB980F899
:1084D8008430FAF79BFC22682423C4F88830136898
:1084E80023F0010313602046FFF7E8FD012816D0AA
:1084F800A36A13B12046FFF7F9FE23685A6822F4ED
:1085080090425A609A6822F02A029A601A6842F0E9
:10851800010220461A60BDE81040FFF79DBF012008
:1085280010BD000030B581658168A0F85C2000238B
:10853800B1F5805FA0F85E20436735D10369002B51
:1085480040F2FF1318BFFF23A0F860300023C0F8E3
:1085580090302223C0F88C30016801F1080353E8F9
:10856800003F43F00103083141E800340368002C60
:10857800F2D1456E84680169B5F1005F34D1B0F875
:108588006850954230D8B4F5805F1DD1254A264CF5
:10859800002918BF22464267C1B153E8002F42F4B0
:1085A800807243E80021F7E729B90369002B14BF5B
:1085B8007F23FF23C8E7B1F1805FC5D10369002B92
:1085C8000CBF7F233F23BFE7174AE4E703F1080204
:1085D80052E8002F42F0805203F1080040E80021E1
:1085E8000029F3D1002030BDB4F5805F0FD10F4AC8
:1085F8000F4C002918BF2246426751B153E8002F9B
:1086080042F4907243E800210029F7D1EAE7084ACA
:10861800F2E753E8002F42F0200243E80021002946
:10862800F7D1DFE72D7F0008917D0008CD7C000899
:10863800017C0008D0F88C30202B30B415D1B9B1AA
:10864800B2B100230468C3660A4B9C420AD063682F
:108658001B0207D554E8003F43F0806344E8003527
:10866800002DF7D130BCFFF75DBF022030BC70474A
:108678000120FBE700800040436E30B52BB9012391
:10868800A0F86A30A0F8683030BD0368094D9A68D0
:108698009968094C490FC2F342626B5C615CDB006C
:1086A800B3FBF1F3A0F86A30AB5CA25CDB00B3FB70
:1086B800F2F3E7E7241B01081C1B01087047704709
:1086C80070471FB504AB03E9060090F88430012B0E
:1086D80004463AD0012380F884302423C0F8883037
:1086E80003681A6822F001021A609A6822F440129C
:1086F8000A439A6071B95A68BDF80C009DF80E10CB
:1087080022F0100202435A605A6822F07F4242EA7D
:1087180001625A601A6842F001021A60FAF7C0F959
:108728006FF07E42034600924FF4800100222046FB
:10873800FFF730FE38B92023C4F88830002384F8C6
:10874800843004B010BD0320F8E70220F9E790F860
:108758008430012B0FD0012380F88430016851E860
:10876800002F42F0020241E80023002BF6D180F8E6
:108778008430184670470220704710B590F884304E
:10878800012B044617D02423C0F8883003681A68E0
:10879800196821F00101196042F000524FF00051B0
:1087A80041661A60FFF768FF2023C0F88830002070
:1087B80084F8840010BD0220FCE770B590F884307E
:1087C800012B044617D005682423C0F888302E688A
:1087D8002B6823F001032B60AB6823F06043194337
:1087E800A960FFF749FF20232E60C0F888300020D9
:1087F80084F8840070BD0220FCE770B590F88430DE
:10880800012B044617D005682423C0F888302E6849
:108818002B6823F001032B60AB6823F060631943D6
:10882800A960FFF729FF20232E60C0F888300020B8
:1088380084F8840070BD0220FCE7000038B5094DBB
:10884800002455F8043B33B90134E3B2052B64B274
:10885800F7D1002038BD002CF6D01B6998470028B6
:10886800F2D0F7E7340D00207FB50A2301A88DF870
:10887800043003F0D9F80038044B059A1A6018BF81
:108888000120404207B05DF804FB00BF2C0D00201A
:1088980070B504460B46144962784A700020A278E5
:1088A8000A7208701A884A729A788A72DB780B748E
:1088B8006368CB600D4B1B68DA6A2AB1237803F032
:1088C800FB030B2B00D09047094E002556F8043BBC
:1088D8001BB19B6A0BB1204698470135EBB2052BBB
:1088E8006DB2F3D170BD00BF88050020300D0020A7
:1088F800340D002070B504461148012303706378D5
:108908004370A3788372E368C360E37803762369CE
:108918004376237943720B4B1B689B6A03B19847D4
:10892800094E002556F8043B1BB1DB690BB1204604
:1089380098470135EBB2052B6DB2F3D170BD00BF7E
:108948009C050020300D0020340D002038B501F0C2
:1089580011FE0C4D052455F8043B5BB15B694BB126
:1089680055F8043C9B682BB1984718B155F8043C5E
:108978005B699847013C14F0FF04ECD1BDE838402E
:10898800FFF75CBF340D0020014B1868704700BF2B
:108998002C0D002000B58BB0012368468DF80030FF
:1089A80002F0BCFC38B99DF80400003818BF01205B
:1089B8000BB05DF804FB0020FAE7000030B58BB07F
:1089C800054601F0BBFD0446002839D1FFF7E2FF58
:1089D800012838D168468DF8004002F09FFC10B19C
:1089E8004FF0FF3004E09DF80430AB4202D1002084
:1089F8000BB030BD012DF3D0022D11D0002DF7D1D1
:108A0800002BF4D068468DF8045002F099FD002838
:108A1800E6D10E4B1B681B6B002BE8D09847E6E7A6
:108A2800002BDDD168468DF8045002F089FD00283E
:108A3800D6D1064B1B681B6B002BD8D02846EDE718
:108A48006FF00100D4E76FF00200D1E7300D00208D
:108A580070B5324C324B94F9042094F9055090B01B
:108A6800012602288DF804608DF809208DF80A5037
:108A78000AD18DF80800D871197202F09FFB01A87D
:108A880002F0D2FF10B070BD4FF480701A715D71A2
:108A9800D8801972234B8DF808601B7853BB1E23AE
:108AA80006A88DF81C208DF8183002F049FD1F2308
:108AB8008DF8183006A823798DF81C3002F040FD97
:108AC80021238DF8183006A863798DF81C3002F040
:108AD80037FD20238DF8183006A863798DF81C30EF
:108AE80002F02EFD28238DF8183006A80E4B0793A8
:108AF80002F026FD02F062FB012306A88DF818306B
:108B08008DF81C3002F01CFD084B1B685B6A0BB12A
:108B1800034898476078FFF751FFB3E7480D0020F6
:108B280070050020280D002000030001300D0020F2
:108B380008B501F003FD40B9FFF72CFF012806D066
:108B4800084B197AD879FFF783FF012008BD064B37
:108B58001B68DB6898470028F7D1BDE80840FFF795
:108B68006DBE00BF70050020340D00202DE9F041D6
:108B780086B005460C46164601F0E0FC002840F099
:108B88008D8001F0EDFC40B9FFF704FF012807D004
:108B9800444B197AD879FFF75BFF6FF002046DE058
:108BA800414F3B68DB68984730B13A682B781278B8
:108BB8009A4201D0002B6ED13C4FDFF8F4803C7212
:108BC800003C18BF012498F8043068788DF80440F8
:108BD80069468DF8123002F049FB002840D0002386
:108BE8008DF804300393ADF810306FF0060495E863
:108BF8000300304B83E8030098F80430BB72314619
:108C080001A803F009F82C4B059A1A6011283FD8DF
:108C180001A353F820F000BF7F8C0008A58C000842
:108C2800998C0008998C0008998C0008998C000888
:108C3800998C0008A38B0008998C0008998C00086F
:108C4800998C0008938C0008998C0008998C00086E
:108C5800A58C0008A58C0008A58C00088D8C000840
:108C68002B788DF808306B78ADF810306B6803936B
:108C78004FF0FF34BBE7E31D18BF0024204606B0C1
:108C8800BDE8F0816FF00404F8E76FF00504F5E73C
:108C98004FF0FF34F2E76FF00304EFE76FF00104E1
:108CA800ECE700BF70050020340D00209C05002073
:108CB800480D0020AC0500202C0D002010B50446FE
:108CC8008AB018B94FF0FF300AB010BD00236846CB
:108CD8008DF8003002F022FB0028F3D19DF8043013
:108CE8002370F1E7F0B587B000220B462A498DF8CA
:108CF800072001220A7042784A700446002A41D1AE
:108D080002790A721A884A729A788A72DB780B7426
:108D18000369CB60C378214D8DF80830037B8DF84B
:108D28000930836803932B68DB6A0BB102A8984764
:108D38002B689B6B13B1227E02B19847184E002511
:108D4800374656F8043B53B11A6A42B11A78E378A9
:108D58009A4219D156F8043C20461B6A98470135B7
:108D6800EBB2052B6DB2ECD10DF10700FFF7A6FFB2
:108D780063793BB10021012204A8ADF810100591D8
:108D8800FFF7F4FE07B0F0BD002DE8D13B68DB68C3
:108D980098470028DED1E2E788050020300D002042
:108DA800340D002010B504468AB018B94FF0FF30D2
:108DB8000AB010BD1F2368468DF8003002F0AEFAE5
:108DC8000028F3D1024A9DF9043023701371EFE7AC
:108DD800480D002000B58BB02223019068468DF81D
:108DE800003002F0ADFB003818BF012040420BB044
:108DF8005DF804FB70B5634C014618228EB020461E
:108E080005F09AFFFBF780F823784068012202FA00
:108E180003F1014004D15C4B084607F083FFFEE7ED
:108E28005A495B481A4602F011F818B14FF0FF3062
:108E38000EB070BD262304A88DF8103002F080FB18
:108E4800544E554D002870D1012333702B68DB69CF
:108E58000BB100209847262304A88DF8103002F0A3
:108E68005DFA059B93F84820227093F8182193F82F
:108E78001A316270A370454BD3E9020105F04EFE2A
:108E880005460028D2D1454E062304A88DF8103097
:108E980002F044FA059B736104A802F051FB022317
:108EA80004A88DF81030059602F038FA0836032326
:108EB80004A88DF81030059602F030FA0F2605F058
:108EC800F1FE012304A88DF814308DF8106002F02B
:108ED80037FB10230DEB03008DF810308DF814507C
:108EE80002F02EFB04238DF8103004A8A3788DF827
:108EF800143002F025FB39238DF8103004A863697B
:108F0800059302F01DFB02A920788DF8086003F094
:108F180051FF003818BF0120E0711420FFF75AFFF5
:108F2800E07903F003F8284682E727238DF810300C
:108F38002B681B6943B104A802F0F0F92B68059867
:108F48001B694FF4EE619847262304A88DF810306A
:108F580002F0F6FA50B9012304A88DF8103002F097
:108F6800DDF99DF81430002B7FF46EAF3378002BB9
:108F78007FF46CAF052204A88DF81020059302F049
:108F8800DFFA78E7480D00202C1B0108600D00204F
:108F9800780D0020280D0020300D0020100D002035
:108FA80037B500230D4601930446C0B900F0D0FA46
:108FB8000190019BC3B10E4A0E4942F824300E4A73
:108FC800DA620E4A1A630E4A5A630E4A12689269A6
:108FD8009A6128465B68F2229847002006E001A9BA
:108FE80000F0BCFA0028E4D04FF0FF3003B030BDE9
:108FF800340D00201C0C0020598A0008758B0008CD
:1090080071880008300D0020154B07B51860154B06
:10901800154A1A60154A5A60154A9A60154ADA6064
:10902800154B02681A6042685A6082689A60C26882
:10903800DA60124A01911A61114982695A61002065
:10904800FFF7AEFF48B901A800F086FA003818BF4C
:109058000120404203B05DF804FB4FF0FF30F9E710
:10906800300D0020780D0020FD880008ED8C0008E8
:109078000991000899880008600D00206DCD00084E
:109088007C05002051B118B1012804D00020704798
:10909800044B0B607047044B0B60F7E74FF0FF3051
:1090A800704700BF000300010300010108B502F08A
:1090B80059FF002814BF6FF00100002008BD08B553
:1090C80002F0A4F8002814BF6FF00100002008BDCA
:1090D80010B504468AB018B94FF0FF300AB010BD79
:1090E800202368468DF8003002F018F90028F3D1E3
:1090F800024A9DF9043023705371EFE7480D0020B0
:109108002DE9F0412F4D304F00232B7043786B70C1
:109118003B689B6A8AB004460BB128469847DFF83B
:10912800AC80002658F8043B1BB15B6A0BB12046A3
:1091380098470136F3B2052B76B2F3D12378052B85
:109148002FD00C2B35D0012B25D1214C0623684676
:109158008DF8003002F0E2F80199E07905F024FD7D
:1091680010B91C4B019A5A611B48FFF71BFE1B489C
:10917800FFF7AEFF6B788BB9A371194B5878FFF7DF
:109188001DFC3B685B6A0BB1114898476B7813B9B3
:10919800E07905F099FD0AB0BDE8F081FF23A371DD
:1091A800EFE7104B01225A74227A9A74627ADA74C1
:1091B800F1E76378002BEED00AB0BDE8F041FFF785
:1091C80053BB00BF9C050020300D0020340D00204B
:1091D80070050020100D0020740500207505002082
:1091E800480D00208805002030B58BB0FFF767FFD9
:1091F8000446F0B903F0BEFD831C1DD0F8B9134D29
:109208002B685B69DBB1262368468DF8003002F0D5
:1092180085F82B6801985B694FF4EE61984703F075
:10922800BBFD78B92CB9094B1B68DB690BB1012070
:10923800984720460BB030BD6FF00704EFE74FF0BA
:10924800FF34ECE74FF0FF34F3E700BF300D0020A8
:1092580030B5064D064C30B129B12860A160627165
:109268000123237030BD00232B60FAE7B40D0020E2
:10927800880D0020014B1878704700BF880D00202A
:10928800024B187800B15878704700BF880D00204D
:1092980070470000064B1A784AB15A783AB10278FA
:1092A800012A04D1027912B19A8901329A81704750
:1092B800880D0020074B1A7852B15A7842B10278CB
:1092C800052A05D1017A427AD973012098731A7454
:1092D800704700BF880D002013B51A4C23783BB3A4
:1092E80063782BB3A27BA36862B10022A273032226
:1092F800A27105221A70E27B5A70227C9A700122B0
:10930800A27004E0A278012A14D0042AF7D0E0223F
:109318008DF800200C48A27901938DF8012008F0FF
:109328007DF80A4B1B6B1BB1E17801226846984710
:1093380002B010BD0222A271A2895A70110A1970D6
:10934800E5E700BF880D00209C0D0020B80500202F
:10935800FFF7C2BF30B5794C23788DB0002B43D0CE
:10936800437B002B40D0657825B1837B13B9A38953
:109378000133A381C178E02936D1002D36D1027B93
:10938800042A31D18368187801282DD1587801280A
:109398002AD19878012827D1DB78012B24D1022003
:1093A8006380A071E56002A863708DF80C302171AC
:1093B8008DF80820257402F0C3F8284602F0B6FD9F
:1093C8005F4B1B685B6803B1984700225D4B0092B6
:1093D8004FF0FF315C4807F075FF41F288315A4879
:1093E80008F056F8FFF778FF0DB030BD83681A789B
:1093F800A2700A2AF8D8DFE802F0062124282A3DBC
:1094080044658D8F9900504807F0BAFF00236370B8
:10941800A3814B4C04238DF80830236802A81B78DD
:109428008DF80C3002F08CF82368587802F07EFD35
:1094380023689B68002BD7D09847D5E70223A371F0
:10944800D2E740F201136380CEE70123FBE7A5686A
:10945800037BA37104222A7062799A4228BF1A46B4
:1094680000230133D9B28A42BED98168C95C01316F
:10947800E954F6E705238DF8083002A802F0D4FA7B
:10948800B2E7314807F07CFF00236370A3812C4CBE
:1094980004238DF80830236802A81B788DF80C3057
:1094A80002F04EF82368587802F040FD23689B6864
:1094B80003B19847254BDB6A002B95D00121022088
:1094C800984791E7027B032A0DD106228DF80820E0
:1094D800B3F801305BBAADF80C3002A802F0A4FA78
:1094E8000123A37080E7072AF7D18DF80820B3F885
:1094F800012052BAADF80C201A79D978120242EA42
:10950800014259790A4364214A4304929B798DF8B0
:109518001430E2E70A23AEE700228DF808205B78D2
:109528008DF80C3002A802F00BF85DE70D228DF8DB
:1095380008205B788DF80C309FE700BF880D00206D
:10954800B40D0020599300089C0D0020B805002098
:1095580000487047B8050020002070474FF0FF30E2
:1095680070470000044B054A93F81831022B18BFC6
:10957800062382F880347047281500209C1C0020A0
:10958800034BD3F8483313B15B6903B118477047ED
:109598009C1C0020034A137843F002031370FFF762
:1095A800EFBF00BF981C00201FB50A4B8DF80900BB
:1095B80093F87C208DF80A2093F88C2093F84800C3
:1095C8000D3202A98DF8082003F0F4FBC0B205B0F3
:1095D8005DF804FB2815002010B50D4C04F57D70CE
:1095E80007F0CEFE94F8103413B1012384F80F3439
:1095F800084B93F81831022B02BF94F8813443F0DA
:10960800100384F88134BDE81040FFF7B9BF00BFEC
:109618009C1C00202815002010B50C4CD4F84033B1
:1096280043F08003C4F8403394F8103413B1002099
:10963800FFF7D2FF94F8813423F0120343F01203AA
:1096480084F88134BDE81040FFF78CBF9C1C0020D3
:109658002DE9F0412C4D95F81831022B07460E469E
:1096680002D02A4BDB6A984702F01BFD044628B15A
:10967800022002F00CFD002002F00EFD95F81831D2
:10968800012B17D102F00FFD804630B1002002F007
:10969800FFFC002002F001FD444602F006FD48B13F
:1096A800002002F0F6FC002002F0F8FCBDE8F041D2
:1096B800FFF758BF002CF9D1154C94F8802494F882
:1096C8001034B2B90BB184F83574384602F090FE04
:1096D800E86A07F01BFED4F8B4339842E6D30D4885
:1096E80007F04EFE94F8813443F0100384F8813477
:1096F800DCE70BB184F83564304602F079FE95F862
:109708001831022BEED1D1E72815002038220108A4
:109718009C1C002034200020074A10B5137843F021
:1097280001031370FFF72CFFBDE81040034B012223
:109738000021022007F0F6BA981C0020751B0108CA
:10974800074A10B5137843F004031370FFF718FFA6
:10975800BDE81040034B01220021022007F0E2BAC5
:10976800981C0020851B01082DE9F0410F4616467C
:109778001D46804607F0C0FD0A4A0B4C1378278126
:1097880043F00803C4E90008137066812573FFF7E6
:10979800F7FEBDE8F041054B01220021022007F049
:1097A800C1BA00BF981C0020A4210020951B010805
:1097B80013B507F0A1FD0D4B6C461860204607F065
:1097C800EFFC94E803000A4A0A4B83E80300137885
:1097D80043F010031370FFF7D3FE074B012200215B
:1097E800022002B0BDE8104007F09CBAB421002066
:1097F800981C0020D41F0020A21B01082DE9F0416D
:1098080092B0064602F04DFC002840F05681AC4D5F
:1098180095F81831012B09D02B6BAA4C93B194F809
:109828000431BBB1042B6FD0032003E002F03BFCF2
:1098380018B10F2012B0BDE8F08102F036FC002804
:10984800EAD0F6E7B5F81E31D4F81424013B5343A7
:109858002B63E4E79C4803F0E4F9002840F02981F1
:1098680094F80C3123802B6B0C930DF1180895F8A4
:1098780039308DF83830404695F81C318DF83A303B
:1098880007F0B4FCD5F82431009302AF98E806003D
:10989800D5F82031384607F040FC97E803000FABB5
:1098A80083E80300EB6A0D9300238DF84430238886
:1098B800ADF8463095F82C3101228DF839201BB9C6
:1098C8008DF844208DF83930804B0093804B95F803
:1098D8004800A3F173020CA903F0E1FAC0B10B2808
:1098E800A8D1D4F8841499B1002EA3D0D4F8403369
:1098F800784843F02003C4F8403307F0C9FD7548A1
:1099080007F08CFD002095E76F4803F0BEF9A4E747
:1099180095F8487095F9693095F9392095F87D10D2
:109928006D4E384603F0CDFA009641B2EB6C95F8CF
:1099380050203846143603F063FA0096EB6C95F81D
:10994800502095F9701095F8480003F059FAD4F8AA
:10995800C413AB6DD4F8D8230B44C4F8B033EB6D03
:109968001344C4F8B43394F80431042B07D02B6E95
:109978000B44C4F8B0336B6E1344C4F8B4330023FB
:10998800089395F82C3183B108A802F061FC0028EF
:109998004AD195F9390094F837629DF82070FFF79D
:1099A80003FE3E4480B2B0423CD300238DF813300E
:1099B80095F839308DF8213095F838308DF8223007
:1099C800D5F880300993D5F884300A93238894F821
:1099D8001164ADF82C3095F84800404B8DF82060A4
:1099E8000DF1130208A903F01FFA012384F8353496
:1099F80095F8393084F836349DF8133084F83734C4
:109A0800D4F81434C4F84464C4F83C34C4F84C346E
:109A180002F04DFB50B1D4F8140402F05AFB28B1FF
:109A2800102007E7082005E7132003E795F8183109
:109A3800012B01D102F04FFB02F03CFB0023059300
:109A480094F8043195F9395094F81164BBB1042B9A
:109A58007FF4EAAE05A802F037FE60BB94F80C3438
:109A68001BB994F80E34012B02D9059B013B0593D1
:109A7800154B05983246E9B202F098FE02E012480A
:109A880002F06CFEA8B9D4F8403394F80C11218088
:109A980043F00203C4F8403394F8103423B994F81F
:109AA8000C34013384F80C340D4B0E489B6A9847EC
:109AB80028E71120BEE61220BCE60E20BAE600BF59
:109AC800281500209C1C0020A41D002058150020EB
:109AD800202100200420002054200020B020002055
:109AE800382201089E1C002073B5144C144D04F54F
:109AF8007876EB6C95F8502095F9781095F8480031
:109B0800009603F07DF940F2012395F84800A4F887
:109B1800F23304F21C42314603F07EF958B194F84E
:109B28001C3484F85E34074B00205B6B984794F82C
:109B3800F33384F8803402B070BD00BF9C1C002051
:109B48002815002038220108F8B5334D95F818413A
:109B5800012C06464BD0022C51D064B938B9D5E94E
:109B68001B0105F1740383E803002046F8BD0128B2
:109B78003DD0022801D00324F7E7284F85F81801C3
:109B880007F5737EBEE80F0007F5787CACE80F0098
:109B9800DEF80030CCF8003095F8E93087F8F36348
:109BA800E3B195F80031022B18D1D5F804316B6771
:109BB800C7F8E43395F87D3095F8082187F8F03335
:109BC80095F88C3085F8782087F8F13397F81124C8
:109BD80087F8E02340F20133A7F8F233002387F82F
:109BE80010340F4BDB6A9847FFF77EFFBDE702F0A2
:109BF80063FA04460028B8D185F81861B5E700284B
:109C0800B9D1064B85F81801062283F88024044B45
:109C1800DB6A98473446A8E7281500209C1C0020DA
:109C280038220108F0B5484C484EB4F8DC202287A9
:109C3800D4E92D0194F8B12084F8692004F16C026C
:109C480082E80300D4E92F0104F1740282E80300DA
:109C5800B4F8C420A4F87C20D4F8CC20C4F884201C
:109C68008FB0D4F8D020D4F8C810C4F888200025C4
:109C7800374AC4F880100123A4F81E31C6F80C2412
:109C8800C4E94E5584F82C51A56284F81B5184F818
:109C98003A50C4F83051A4F8345186F8105484F876
:109CA80041518DF8143004F5087394F84800A4F86D
:109CB8004251039303A904F52D73049303F088F824
:109CC800E36EC6F8D03394F87D3086F8DC3394F828
:109CD8008C3086F8DD334FF48073A6F8DE3386F8CF
:109CE800CC5306F573770FCF06F578740FC43B682D
:109CF800236040F20123A6F8F233D6F8483386F8F9
:109D08001154CDE901551BB15A685B690192029360
:109D1800104B0693A3F144020792A3F11402089290
:109D28000D4A0A9225330993A2F19C030B93A2F1E1
:109D380098030C9301A9131D06A802F274620D93EF
:109D480002F0A4F90FB0F0BD281500209C1C0020DB
:109D580000010100F82000200C160020F8B50D4F76
:109D68000D4C0E4E0D4607F00BFB3B6B984796F8D3
:109D7800480004F21C42294603F04EF848B194F812
:109D88001C3484F85E34706D7B6B9847EB7C84F8E8
:109D98008034F8BD382201089C1C002028150020BA
:109DA8000D4890F8113480F8B8330C4B93F86920BB
:109DB80080F8BB2393F87D2093F88C3080F8C93362
:109DC800002380F8C823A0F8CA3300F56E7100F5A7
:109DD8006070FFF7C3BF00BF9C1C0020281500203F
:109DE8000F4890F88034CBB190F8113480F8CC3318
:109DF8000C4BDA6EC0F8D02393F87D2093F88C30A2
:109E080080F8DD334FF4807380F8DC23A0F8DE336C
:109E180000F5737100F56670FFF7A0BF704700BFCB
:109E28009C1C00202815002070B5344C24212046A5
:109E380004F098FF636A984218BF60624FF01C01F3
:109E48002F4814BF0125002504F08CFF636C98424D
:109E580018BF60644FF0FC012A4818BF45F002059E
:109E680004F080FFD4F84431984218BFC4F8440184
:109E78004FF0D401244818BF45F0040504F072FFE0
:109E8800D4F81C32984218BFC4F81C024FF0900155
:109E98001E4818BF45F0080504F064FFD4F8B03236
:109EA800984218BFC4F8B0024FF49461184818BF1C
:109EB80045F0100504F056FFD4F85437984218BFFF
:109EC800C4F854074FF01401124818BF45F0200594
:109ED80004F048FFD4F86C3798420F4B18BFC4F809
:109EE8006C07D3F8483318BF45F040052BB11B6900
:109EF8001BB12846BDE87040184770BD28150020E2
:109F080050150020701500207016002048170020FA
:109F1800DC170020801C00209C1C00202DE9F04F3D
:109F280091B00026BD4F8DF81560054688469346CA
:109F3800ADF81860B146C14502D311B0BDE8F08F45
:109F480015F8090002F0C2F948444045F5DC15F857
:109F5800093009F10104023BE4B2112BEDD801A24A
:109F680052F823F0B59F0008E59F0008A5A0000857
:109F7800D1A0000861A1000885A10008F9A1000886
:109F88002DA20008ABA20008439F0008439F0008C9
:109F98000BA30008439F0008439F0008C1A30008C3
:109FA800E7A300082BA4000869A40008052002F014
:109FB80039FA88B10521002002F0F8F92B5D87F8FD
:109FC800503409F1030409F102095FFA89F9E4B28E
:109FD80015F8093087F85134A146ACE700238DF80D
:109FE80016308DF817308DF81C308DF82030002E83
:109FF80052D18B4E631E2B440D9396F81A318DF86F
:10A008003A3096F87C308DF8393096F839308DF83A
:10A018003B3096F838308DF83C3096F868308DF83B
:10A028003D30D6F828310C9308AB019307AB009369
:10A0380096F84800A8EB09090DF117030DF116026F
:10A048000CA98DF8389002F0FBFE8DF8150000F091
:10A05800070007280BD19DF8163086F839309DF88F
:10A06800173086F838309DF81C3086F8683000269E
:10A078004FF0050906E001220DF11501032002F059
:10A088003BF80136F2B29DF82030B3FBF9F191426A
:10A09800F1D8013B2344DCB201269DE72B5D6049E2
:10A0A80003F00F03012281F81B3109F1020902FABA
:10A0B80003F3A1F81E315FFA89F9002206A90420EA
:10A0C80002F01AF84C4687E707238DF815302B5D08
:10A0D800C3F3021203F00F038DF8303009F10303C4
:10A0E800DBB28DF83120EA5C09F10403DBB209F137
:10A0F8000504EB5C09F102095FFA89F91B0443EADC
:10A10800022315F80920DFF81891134364225343FA
:10A1180099F848000D930CA902F0A1FE00F007037E
:10A12800072BE4B28DF815000ED19DF8303089F870
:10A13800703089F878300D9BC9F86C30C9F87430E4
:10A148009DF8313089F869308DF81800012206A988
:10A15800052001F0D1FF3FE7D7F8483363B11B680A
:10A1680053B198470BF03F038DF818008DF819305C
:10A17800022206A90620ECE7FF20F3E703238DF867
:10A1880015302B5D8DF824300CAB089309F10303CF
:10A19800DBB209F10604EA5C09F10403DBB208A9A1
:10A1A800EB5C1B0443EA022309F10202D2B209F173
:10A1B8000509AA5C1343642253435FFA89F90C9397
:10A1C80000230D9315F809308DF83830144B93F8A7
:10A1D800480002F04AFEC3B20028E4B28DF81530F8
:10A1E800FFF6FAAE8DF81830012206A90720B0E76D
:10A1F8002B5D03F00F03012B4FF47A7238BF012354
:10A208005343074A09F10209936503F57A73D36545
:10A218005FFA89F9002206A9082051E79C1C002052
:10A22800281500202B5D9C4CC3F340128DF81D208F
:10A2380094F84800C3F3001207A903F00F038DF840
:10A248001C208DF81E3002F016FE09F102090130BB
:10A258005FFA89F93FF436AFBDF81C308F4AA4F88D
:10A268007C309DF81E309DF81CA0D05CF7F7CEFB23
:10A278000223C4F880000CA994F848008DF8303007
:10A288008DF832A002F096FD94F93930089040B26A
:10A298009842B8BF184684F83900002206A9092058
:10A2A8000EE703238DF815302B5D8DF8303009F15A
:10A2B8000303DBB209F10504EA5C09F10403DBB22C
:10A2C80009F10209EB5C5FFA89F91B0443EA0223EE
:10A2D80015F809201343642253430D936E4B0CA9C0
:10A2E80093F8480002F0CDFDC3B20028E4B28DF81F
:10A2F8001530FFF671AE8DF81830012206A90A2034
:10A3080027E70A2002F08EF800283FF465AE0A21FC
:10A31800002002F04BF80023ADF8263009F10203C3
:10A32800DBB24FF47A71EA5C09F10303DBB20DF199
:10A33800300AEB5C1B0443EA02232A5D134309F14C
:10A348000402D2B209F1060409F10509AA5C5FFA10
:10A3580089F943EA026315F8092003934A43121264
:10A368005046ADF8242006F01BFF039B03F19653DB
:10A3780003F5A91303F5EC530893D7F83C3300937E
:10A388000DF1200999E80600D7F838330AA806F035
:10A39800C4FE0B9B00939AE806000A9B484606F009
:10A3A800A1FE99E8030006F0D3FE01F08FFE012319
:10A3B800E4B287F830340FE60D2002F033F80028B5
:10A3C8003FF40AAE0D21002001F0F0FF97F8803429
:10A3D800043B012B7FF600AE01F074FEFCE509F1A9
:10A3E8000203DBB22A5DE95C09F10303DBB209F180
:10A3F8000504EB5C09F104095FFA89F91B0415F8F7
:10A40800090043EA012313436421594300F00F0074
:10A4180001F059FEE4B28DF81800012206A91120B6
:10A4280097E60E2001F0FEFF00283FF4D5AD0E217F
:10A43800002001F0BBFF09F10203DBB2184AE85C17
:10A448002B5D126809F1040409F103095FFA89F91F
:10A4580043EA002015F80910E4B201F036FEBBE526
:10A468002A5D09F1020309F1040409F10309DBB2C9
:10A478005FFA89F9E95C15F809301B0443EA0123FE
:10A4880013436420584301F022FEE4B28DF818000B
:10A49800012206A913205CE628150020AF1B01083D
:10A4A800A42100200E4B93F88124920703D593F83A
:10A4B8007F24012A06D90B4A92F81A1111B1916A20
:10A4C80001319162002283F80C2483F8102483F868
:10A4D8000F24D3F8402322F00202C3F84023704728
:10A4E8009C1C00202815002010B5124C04F55A7049
:10A4F80006F046FFD4F84033012023F02003C4F8C7
:10A508004033FFF77BF998B10B2811D00A4B93F829
:10A51800393084F83634092094F80E3484F8393404
:10A5280084F8350401F064FFBDE81040FFF7BABFB6
:10A5380010BD00BF9C1C002028150020074BD3F835
:10A548004023012A06D03AB993F88204013818BF8B
:10A558000120704700207047012070479C1C002094
:10A56800034BD3F84003431E58425841704700BF7D
:10A578009C1C00202DE9F04FA5B0EFF3108172B6B6
:10A58800C04A00201368106081F31088BE4C002B6D
:10A5980000F0DA80D9065FFA83FB6BD5BB4D95F8DE
:10A5A8001831022B02D0BA4BDB6A9847EFF31088B8
:10A5B80072B6B84F06F0A0FE3E68D4F8B013361A4B
:10A5C8003144B54806F064FFB34806F027FFD4F8D5
:10A5D800B413B248314406F05BFFB04806F01EFFE2
:10A5E80088F3108895F81831022B02D094F81034AB
:10A5F8008BB116230EA995F848008DF8383002F073
:10A60800D9FBD4F8B4130C900144A54806F040FFD8
:10A61800A34806F003FF3B6894F81124EB620AAFE5
:10A6280038468DF86020199306F0E0FDD5F82431FE
:10A63800009304AE97E80600D5F82031304606F0BE
:10A648006CFD96E803001BAB83E80300D4F81434D0
:10A658001A9395F82C3195F84800003B18BF012350
:10A6680018A98DF8613002F0AEFB94F810340BB9DC
:10A6780084F835341BF0080F3AD08A4B834D5F6855
:10A688001E89B3F90A8093F90C90D5F8E420039257
:10A698000023079384F83834A4F81A3484F81D3456
:10A6A800C4F82034A4F8243484F82634C4F82834B0
:10A6B80084F81834C4F82C3484F83034744B94F883
:10A6C8008024DB6A84F87F24A4F87C8484F87E9450
:10A6D8009847724806F054FE3146384601F0DFFCD0
:10A6E8008246002800F0E680A4F8728484F8749406
:10A6F8001BF0040F1AD0654B93F81831022B02D0C7
:10A70800634BDB6A98470220FEF72CFF84F8350478
:10A7180001F06EFE94F8103413B1012384F80F345D
:10A7280094F8813443F0100384F881341BF0020F4D
:10A7380003D006210520FEF78BFF1BF0010F03D085
:10A7480004210320FEF784FF01F0C6FC94F881245D
:10A75800D0065FD5002384F88234D4F84033190634
:10A7680044BF23F08203C4F8403312F0050F00F011
:10A77800C5820C2001F056FE002800F0BF8294F834
:10A788008134DF0700F1BA825E0740F1CB82D4F84A
:10A79800403323F00203C4F84033D4F8402382BB8B
:10A7A80094F8815415F001011EBF2B4662F3000393
:10A7B80084F8813494F881345E0744BF6FF38203D0
:10A7C80084F88134012384F8823421B1D4F84433E5
:10A7D80035481B6898476D070BD5344801F02EFEA5
:10A7E80001F05CFE28B194F8813443F0040384F846
:10A7F800813401F060FC94F881346FF3041384F819
:10A808008134012384F8823494F8813443F020039E
:10A8180084F8813494F8813418070AD56FF3C30398
:10A82800234984F88134D4F84433A1F12000DB684B
:10A83800984794F8813499070AD56FF341031C4966
:10A8480084F88134D4F84433A1F164005B689847F4
:10A8580094F88034022B01D1FFF746F994F881343B
:10A868009A0640F1EC826FF3451384F88134D4F8EA
:10A878004033002B40F0E38225B0BDE8F04FFFF7EE
:10A88800D3BA00BF981C00209C1C0020281500206B
:10A8980038220108B42100201C2000203420002088
:10A8A80090200020A4210020D0200020E4200020B7
:10A8B8001821002095F81831012B0CD101F0F3FB79
:10A8C800804668B1504601F0E3FB504601F0E5FBD5
:10A8D800042384F87F347EB9012384F819344AE1CB
:10A8E80001F0E3FB0028F6D0404601F0D2FB4046D9
:10A8F80001F0D4FB0523ECE73B7802935B09013BAD
:10A90800062B00F2ED81DFE813F00700EB0192005F
:10A91800EB018F00EB01DB01102EDDD995F82C310E
:10A928000E97F6B28DF83C60002BD5D118A804F02C
:10A938002DF90EAA18A9FF2002F04CF89DF848300E
:10A94800C3F3030307468DF8203095F8480095F8BF
:10A958007D308DF82130072208A902F03EFA002F39
:10A968005AD1002858D09DF843309DF842201199BB
:10A97800C5F8E4101B0443EA02239DF84120022095
:10A988001343C5F8E03004F00FF99DF8483095F806
:10A99800480085F82A71C3F30212C3F3030385F84C
:10A9A800703085F878309DF8493085F86920012B9A
:10A9B80038BF01234FF47A725343AB651344EB65F8
:10A9C8004FF001080DF14A03113E0CA90C9385F8CC
:10A9D80068808DF8346002F008FA0223404685F852
:10A9E8002C3101F01FFD18B14146384601F0DEFC5C
:10A9F80094F81034002B00F0798194F8383413B1AE
:10AA08000020FEF7E9FD94F8813443F0100384F840
:10AA18008134FEF7A7FD6BE6012001F003FD002855
:10AA2800E6D001210720E1E7012384F8183495F8DE
:10AA38007D308DF8223094F81C348DF8213095F84B
:10AA48008C3095F848000D3308A98DF8203002F0B5
:10AA5800B1F9A6F10D031BB2069023EAE37300B225
:10AA680083423FF739AF0B2E7FF636AFA24B2193C7
:10AA780018A8FF2318978DF864608DF8883002F0C5
:10AA880075F8804600287FF427AF9DF86C301A9936
:10AA9800C4F82C1413F00F0203D09DF8800000288E
:10AAA8006CD19DF8880000286AD0002A7FF414AF82
:10AAB8009DF88020002A0CBF022703270022079256
:10AAC800D5F8EC2091425DD195F8E910002959D0CC
:10AAD800D5F80C1195F8EAA00968079195F81811AE
:10AAE800022902D1032184F87F14032F7FF4F4AEE6
:10AAF80013F0600F7FF4F0AE03924FF001081523B6
:10AB080095F848008DF8203008A902F053F995F817
:10AB18002A310690BAF1000F37D0BAF1010F3ED1B1
:10AB2800012B34D16FF009063E4106F00106C6F14B
:10AB38000206F6B281B2BDF86E2007AB304601F0CE
:10AB4800CFFD70B3072824D1082384F8193495F869
:10AB58002A315BB9029B03F0E003A02B06D16A6B94
:10AB6800239B9A4202D1012385F83A30079BC4F807
:10AB78002834C4F86034FEF74FFDB9E547469DE731
:10AB880001279BE74FF0010AB9E70426D2E703261D
:10AB9800D0E7082803D10A2384F81934E6E701230B
:10ABA800FAE718AB00930399079B3246504601F029
:10ABB80063FE20B102280CBF0B230C238DE6079BF4
:10ABC800C4F82834C4F860349DF86C3084F819044B
:10ABD800C3F3401384F8263484F8383494F87F3467
:10ABE80084F81A84012B98BFA862B8F1010FC4F841
:10ABF800200484F8240484F8350433D1022284F82C
:10AC0800182495F83A20002A3BD19DF86C20D206EA
:10AC180037D4012B94F834149DF86C2005D80129F9
:10AC280001D1960601D501F001FB022F37D0032F81
:10AC380009D09DF86C10012F4A4601F00F011CA89D
:10AC480031D0FFF76BF99DF8803084F81B34219BD5
:10AC5800C4F820349DF8883084F82434012384F81B
:10AC6800253426E0029A02F0E002A02A11D195F8D4
:10AC78002A11012285F83A2009B92399696384F8D1
:10AC8800182495F81821002AC3D1012284F81D241C
:10AC9800BFE7002285F83A2084F81824B5E79DF824
:10ACA800881021984A46FFF739F99DF8803084F8D2
:10ACB8001B3494F8813443F0020384F8813497E616
:10ACC800DFF83480013EB2B2791C404604F034F813
:10ACD8000323A4F81834C4F8208484F82464E8E72B
:10ACE800012384F81934FEF797FC81E695F81831AA
:10ACF800022B7FF488AE83E6D41E002094F88134BA
:10AD08005D070FD5012001F08DFB88B3012001F00C
:10AD18005FFB08B984F80C04D4F8403323F002032D
:10AD2800C4F8403394F88114C8077FF536AD94F819
:10AD380034340BB1032B26D1424B94F80C0493F80E
:10AD48006820904208D28A0750D593F818311BB171
:10AD580094F87F34002B49D13B4806F011FBD4F816
:10AD6800403323F02003C4F84033FFF79BFB14E57E
:10AD7800062001F057FB0028CED1072001F052FB36
:10AD88000028C9D1CEE7012B30D194F80F24002A2E
:10AD98003FF403AD94F80E3494F80D04834204D2C2
:10ADA80011F0020218BF94F83824264D95F82A119C
:10ADB800002941D132BB834218D20133DBB2DF070D
:10ADC80084F80E3412D522238DF8603095F87C3043
:10ADD8008DF8623095F8480095F839308DF8613073
:10ADE80018A901F0E7FF0E9085F8390094F881342E
:10ADF80000206FF3041384F8813484F80F04FFF7FC
:10AE080073FBCAE494F838648EB902238DF868306D
:10AE180005F50873189395F8480005F52D7318A9DA
:10AE2800199301F0D5FF84F8106484F8386494F815
:10AE38000E3484F839348FE7002AD7D08CE725B050
:10AE4800BDE8F08F28150020042000202DE9F04FE0
:10AE58008A468BB091460746002800F08D8100296C
:10AE680000F08A810368002B00F086814368002B7C
:10AE780000F082818368002B00F07E81C368002B7C
:10AE880000F07A81104601F091FF002800F07681E9
:10AE9800BC4CBD4D384601F03FFA4FF4EE6200213C
:10AEA800204603F05DFF4FF4A1620021284603F01D
:10AEB80057FFB64BC4F8283100264FF001080F237E
:10AEC80005A948468DF8143084F8489084F818612C
:10AED80084F88C6085F80E8485F80D8401F06AFF8B
:10AEE800801B18BF01204FF00A0B84F81C0105A92C
:10AEF80094F848008DF814B001F05CFF4FF0060993
:10AF080084F8DC0005A994F848008DF8149001F045
:10AF180051FF102384F8DD0005A994F848008DF846
:10AF2800143001F047FF1123C4F89C0005A994F8D8
:10AF380048008DF8143001F03DFF1223C4F8A0003A
:10AF480005A994F848008DF8143001F033FF132355
:10AF5800C4F8A40005A994F848008DF8143001F04D
:10AF680029FF14230DEB0301C4F8A80094F8480046
:10AF78008DF8143001F01EFF1723C4F8AC0005A9A2
:10AF880094F848008DF8143001F014FF182384F861
:10AF9800B10005A994F848008DF8143001F00AFFB3
:10AFA8001923C4F8B400C4F8BC0005A994F84800F3
:10AFB8008DF8143001F0FEFEC0B21E2384F8B800EC
:10AFC80084F8C00005A994F848008DF8143001F001
:10AFD800F1FE1F2384F8C40005A994F848008DF8F1
:10AFE800143001F0E7FE202384F8C50005A994F881
:10AFF80048008DF8143001F0DDFE2123C4F8C800A4
:10B0080005A994F848008DF8143001F0D3FE0B23FD
:10B01800C4F8CC0005A994F848008DF8143001F064
:10B02800C9FE0C23A4F8D00005A994F848008DF8AF
:10B03800143001F0BFFED4F89C306365D4F8A0301A
:10B04800A365D4F8A430E365D4F8A8302366D4F80F
:10B05800AC30636604F5087307A90490A4F8D2001D
:10B06800079394F848008DF8246004F52D7308932D
:10B0780084F8B080C4F894B084F89890C4F84CB0C0
:10B0880084F8509084F8688001F0A2FEC5F848A3BF
:10B09800FEF7C8FD32463E4B00964FF0FF3105F5EE
:10B0A8005A70C4E90B66C5F8447385F8816484F85E
:10B0B8001981C5F8408306F005F93246354B0096EC
:10B0C8004FF0FF3105F5607006F0FCF83246324B60
:10B0D80000964FF0FF3105F5667006F0F3F832463A
:10B0E8002E4B00964FF0FF3102AE05F57D7006F04D
:10B0F800E9F8304606F07AF896E8030004F590730C
:10B1080083E80300264BC5F84C33264BC5F8543367
:10B11800254BC5F85C33254F254BC5F85033254BD7
:10B12800C5F8583305F553703B68984704F5A47083
:10B1380003F04AFB20B1112630460BB0BDE8F08F72
:10B14800204601F09DFA0028F5D100F0C7FFB8B9F4
:10B15800194801F0F7FA06460028ECD17B699847B0
:10B1680003F0C8FDBB6D94F819019847FB6A98472E
:10B17800012385F88234DFE70326DDE70926DBE7CC
:10B188001326D9E7281500209C1C00200003000185
:10B19800F1A40008A99D0008E99D0008E1950008B0
:10B1A800B9970008719700089D9500083822010892
:10B1B80049970008219700081016002008B5034B8E
:10B1C8000020C3F84003FEF7CDF908BD9C1C002001
:10B1D80010B5FFF7B3F90A4C60B90A4B93F8183168
:10B1E800022B02D1084BDB6A98470123C4F840338D
:10B1F800002010BDD4F84003013818BF0120F8E73B
:10B208009C1C0020281500203822010838B5134C52
:10B2180004F55A7006F0B4F804F5607006F0B0F85A
:10B2280004F5667006F0ACF804F57D7006F0A8F831
:10B2380000F040FF0A4B0025DB6A9847C4F84053EA
:10B24800FEF7F2FD074908484FF4EE6203F074FD7B
:10B258000123C4F84033284638BD00BF9C1C002099
:10B268003822010828150020B80D002030B52A4BD7
:10B2780089B0054693F8DD008DF8020093F8DC00EC
:10B288009A6A8DF803000020019202900C4600296A
:10B298003ED00592D3F8882006921A8FD3F8281149
:10B2A800039152BA93F81A11ADF81C2093F87C2038
:10B2B80093F848308DF810008DF811108DF81E2085
:10B2C8008DF81F300DF1030201AB0DF1020103A847
:10B2D80000F06EFE9DF90200FEF766F9607002A8A4
:10B2E80000F0B6FFB0B9029A0F2A0DD863789A42D7
:10B2F8000AD81544AB42A3EB02012CBF0020012061
:10B308002170C00009B030BD002323700820F9E780
:10B318000320F7E71320F5E7281500201FB504469A
:10B32800002800F0FD8000783F2800F2F380DFE875
:10B3380010F0400046004B005000540058005D00DB
:10B34800F100F100F100F100F100F100F100F1006D
:10B35800640068006C0077007E008100840089002A
:10B3680087008B008F009200950098009B009E003C
:10B37800A200AA00A600AE00B100B500BE00BA0047
:10B38800BC00F100C200F100F100F100F100F10091
:10B39800F100F100F100F100F100F100F100F1001D
:10B3A800F100F100CA00CE00D300D700DB00DF00B7
:10B3B800E8005D4B93F81831237104B010BD5A4B67
:10B3C80093F82C31237102E0606803F099FB0020A8
:10B3D800F3E7606803F0DAFBF9E7534B93F81A31A7
:10B3E800F0E7514BD3F8E0306360F0E74E4B211D96
:10B3F80093F82C0103F0E2FBE9E74B4B93F8193182
:10B40800E0E7494B93F88C30DCE71D238DF80830D2
:10B41800454B02A993F8480001F0CCFC6060D6E7E0
:10B42800424B043493E8030084E80300CFE7404B21
:10B438000434F7E73F4B0434F4E73F4B0434F1E7B7
:10B448001B23E3E71A23E1E7374B93F86830B9E7A2
:10B45800354B5B6DC8E7344B9B6DC5E7324BDB6DF5
:10B46800C2E7314B1B6EBFE72F4B5B6EBCE72E4B21
:10B4780093F8DD30A6E72C4B93F83930A2E72A4B36
:10B4880093F8DC309EE7284B93F838309AE7264B40
:10B49800DB6CA9E7244B93F8503093E7224BD3F8A1
:10B4A8008430636093E7204B9EE7244B9CE71E4B58
:10B4B800D3F8CC30F5E71C4BD3F82831636001F0A2
:10B4C8000DFDA06083E7184BD3F890308CE7164B3E
:10B4D800B3F88830A3807AE7134BB3F88A30F9E7DA
:10B4E800114BB3F8D030F5E70F4BB3F8D230F1E792
:10B4F8000D4B93F848200AB1062A13D1B3F84C37FC
:10B50800E8E7094B93F848200AB1062A0AD1D3F88C
:10B51800503769E7204604B0BDE8104000F0CEBDC2
:10B5280003204AE7182048E7281500209415002032
:10B53800DC1500209C150020E4150020B80D002023
:10B5480073B5044600285ED0A04DD5F840339A075D
:10B5580000F15F8202783F2A00F25682DFE812F09B
:10B56800400046004E0056005A005F00640070001C
:10B578007A007F00840089008E00930098009D0067
:10B58800A7005402AC00CC00DF0006012801190115
:10B598002C013C014001440148014C015001620169
:10B5A8008A0178019C01A201A901AE01B3015402EC
:10B5B800180254025402540254025402540254020F
:10B5C80054025402540254025402540254025402C3
:10B5D800540227022C02310236023B0240024A0280
:10B5E800007902B0BDE87040FEF7AEBA0379022BCD
:10B5F80009D0774A82F82C31002005E0406803F032
:10B6080071FA0028F8D0032002B070BD406803F03A
:10B61800ADFAF6E76E4B027983F81A21ECE76C4B2A
:10B628004268C3F8E020E7E7694D416895F82C01C6
:10B6380003F0BAFA0028E6D16368C5F8E430E3E716
:10B6480041680029DFD0002001F0A8F90028D3D0F4
:10B658001120D9E741680029D5D00120F4E74168D5
:10B668000029D0D00820EFE741680029CBD0092075
:10B67800EAE741680029C6D00C20E5E741680029BF
:10B68800C1D00D20E0E741680029BCD00E20DBE7DF
:10B6980041680029B7D00F20D6E74E4C4C4B0079B3
:10B6A80083F81901A36D9847E36A9847A4E7484BC4
:10B6B800027983F88C209FE7454D037A8DF8003096
:10B6C80095F8480095F87D308DF8013007226946D5
:10B6D80001F083FB002896D0636895F84800009332
:10B6E8000022694601F079FB00288CD06C35D4E93A
:10B6F800010185E803007FE7354D037A8DF80030B6
:10B7080095F8480095F87D308DF801300722694694
:10B7180001F063FB00283FF476AFB435E7E72C4D22
:10B72800037A8DF8003095F8480095F87D308DF84B
:10B7380001300722694601F050FB00283FF463AF4F
:10B74800D4E9010105F1740383E8030095F8183181
:10B75800022B7FF451AF95F82C31002B3FF44CAFFE
:10B768001C4BDB6A9847FEF7BFF945E7184D037A8B
:10B778008DF8003095F8480095F87D308DF8013047
:10B788000722694601F029FB00283FF43CAFBC358D
:10B79800ADE74368009301238DF804300C4B6946EC
:10B7A80093F8480001F026FB00287FF425AF2AE72C
:10B7B800436800930023EFE703795A1E0E2A3FF6E9
:10B7C80022AF034A82F8683016E700BF9C1C0020AD
:10B7D8002815002038220108904B42685A650BE76B
:10B7E8008E4B42689A6507E78C4B4268DA6503E737
:10B7F8008A4B42681A66FFE6884B42685A66FBE63F
:10B80800864C037994F848008DF800300622694682
:10B8180001F0E3FA00283FF4F6AE9DF8003084F812
:10B82800DD30E9E67D4C03798DF8003094F8480066
:10B8380094F87C308DF802300522694601F0CDFA83
:10B8480000283FF4E0AE9DF8003084F83930D3E6A4
:10B85800724C037994F848008DF800300A22694642
:10B8680001F0BBFA00283FF4CEAE9DF8003084F812
:10B87800DC30C1E6694C037994F848008DF8003053
:10B888000922694601F0A9FA00283FF4BCAE9DF8E8
:10B89800003084F83830AFE6604B4268C3F8942033
:10B8A800DA64A9E65D4B027983F8982083F8502082
:10B8B800A2E65A4B4268C3F884209DE6574B42687B
:10B8C800C3F8CC2098E6012B40F0A380544C2421E7
:10B8D800204603F047FA636A984201D0172093E69E
:10B8E8001C2104F1280003F03DFA636C9842F5D15D
:10B8F800FC2104F1480003F035FAD4F844319842A9
:10B90800ECD1D42104F5A47003F02CFAD4F81C323D
:10B918009842E3D1902104F5087003F023FAD4F893
:10B92800B0329842DAD14FF4946104F52D7003F0E7
:10B9380019FAD4F854379842D0D1142104F5EB60A1
:10B9480003F010FAD4F86C379842C7D1334E214629
:10B9580030464FF4EE6203F0EFF920464FF4EE6202
:10B96800002103F0FDF995F8113485F8E033736F81
:10B97800C5F8E43396F87D3085F8F03340F20123BA
:10B98800A5F8F233274B96F819019B6D984733E6D3
:10B998008379012B3FF637AE204B42684068C3F8E5
:10B9A800282100F089FE00283FF42EAE50E61B4BFC
:10B9B8004268C3F890201FE6184B8288A3F88820B5
:10B9C8001AE6164B8288A3F88A2015E6134B82885C
:10B9D800A3F8D02010E6114B8288A3F8D2200BE6FA
:10B9E8000E4B93F848200AB1062A14D1A288A3F86E
:10B9F8004C2701E6094B93F848200AB1062A0AD1D8
:10BA08006268C3F85027F7E502B0BDE8704000F05F
:10BA180057BB0120F8E51820F6E500BF28150020DF
:10BA2800B80D0020382201082DE9F04186B0002326
:10BA3800ADF800300646002800F0E280FEF77EFDF3
:10BA480020B10124204606B0BDE8F08100F02CFDAD
:10BA58000028F6D100F022FD014618B969481422E1
:10BA680003F07EF9684D95F88134012243F0040310
:10BA780085F8492485F8813433788DF8043000211D
:10BA8800013B8DF805208DF807100D2B00F2B080D2
:10BA9800DFE803F007AEAEAE525A7DAEAE85AEA279
:10BAA8008F9ED5F8404314F02004CAD1DFF85C819A
:10BAB800574FFEF7B7F8224696F9051098F8480050
:10BAC80001F0E5F988F83900B37988F8383020466C
:10BAD80007238DF80530FEF737F8FF2307F5867042
:10BAE800A5F80C3185F80441C5F8087103F04EF843
:10BAF80007F58A7003F004F82046FDF77FFE044638
:10BB080040B196F9051098F84800012201F0BFF9F4
:10BB180088F83900D5F884343361002C6CD000F0F3
:10BB2800BDFC00288ED195F8813485F8100460F3A7
:10BB3800820385F8813485E700226946022000F0F7
:10BB4800DBFA10B31324E5E795F811348DF80830C3
:10BB58002E4BB28893F839108DF8091093F83810E5
:10BB68008DF80A10D3F880100391D3F8841004914B
:10BB780093F84800ADF8142002A901F09DF9D5F812
:10BB8800403343F00203C5F840330024C2E7214B99
:10BB9800B28896F90C10B068DB6B9847EFE702A9FA
:10BBA8000D2000F027FB0028EFD0002269460D2069
:10BBB800C5E7164B93F81831D3B9347904F0070068
:10BBC80000F077FA8DF80040012269461020B6E7A8
:10BBD800002269461220B2E78DF8072000F05AFAD1
:10BBE800044638B900F053FA204600F055FA91E7B8
:10BBF80002248FE701248DE701A800F0A1FB21E7CB
:10BC080003241FE7E42000209C1C002028150020A6
:10BC18009E1C0020382201082DE9F04F91B0002623
:10BC28000391054618B9032011B0BDE8F08FFEF75F
:10BC380085FC8246002840F06481B84C14220146F5
:10BC4800074604F2344003F08BF8012384F83534B6
:10BC580084F80E342A789A4200F0B080032A00F063
:10BC6800BF80002A40F0C98084F80D34022295F87C
:10BC78000490D5F80880AE8995F90EB062F347179D
:10BC88009A46A74B022493F87C2093F848008DF835
:10BC9800244009A98DF8262001F08CF8BAF1000F8C
:10BCA80000F02D819E4B93F81A21B2B940B2584545
:10BCB800B8BF584693F87C208DF814008DF81620EC
:10BCC80093F84800052205A901F087F80028AAD0B2
:10BCD800934B9DF8142083F83920198F1A8F93F805
:10BCE8002C010291996A069152BA002800F0058148
:10BCF80093F81B0100B9186393F81801ADF83C20BC
:10BD0800013893F87C208DF83E20D0F1000B93F891
:10BD180048208DF83F204BEB000B824A93F83A00FD
:10BD280093F81A4101900D914FF00100D3F8881053
:10BD3800D3F828318DF830000E910B93511C06ABC7
:10BD48000BA88DF8314000F033F9019B4FEA0B1B2B
:10BD58004BEA431B4FF0000A4BEA801B4BEAC41323
:10BD6800D0456E4C019308BF56463246414604F50D
:10BD78009C709B46CDE907AAA4F800A084F810A4FB
:10BD880002F0DAFFF9B2A770C7F34217F2B2042F34
:10BD9800634E019B84F8372233D0072F00F09D8033
:10BDA800022F32D00220029B33875C4B002283F89B
:10BDB80010245A4BD3F884342B6135E7EB7B082BDE
:10BDC80028BF082384F80D34042395F80490D5F887
:10BDD8000880AE8995F90EB063F34717924650E78D
:10BDE80084F80D34D5F804802E8995F90AB067F0E7
:10BDF8001F079A464FF0000943E7D346D046D1467D
:10BE08003FE74FF0010084F81004474F84F80D1104
:10BE1800042084F80401FF20D6F8E41084F80C010B
:10BE280084F8143107A807F59B73C4F8087184F8DF
:10BE38002891C4F8101184F83021C4F82C3100F08E
:10BE480043FC002857D1079BA4F8380408A8A4F895
:10BE58001631C4F8403400F0FBF960BB089BABB165
:10BE680096F93900FDF7A0FB94F837322BB3089BFD
:10BE78000F2B19D807F58B7208A90F2000F0F4F9D9
:10BE8800C8B9089B63F3030B84F814B10398FDF752
:10BE9800B5FC002887D1069B86F83A00B36200F00B
:10BEA800B7F980B3132080E707F2864208A900F0AB
:10BEB800DBF90028EAD0132075E707F286473A46EF
:10BEC80008A900F0D1F90028F5D1089B84F82801C9
:10BED800C4F82C7184F83031D8E7B8F1000FD5D008
:10BEE800002AD3D04146E01C02F026FF94F83732EE
:10BEF80001332380CAE7122055E7072055E720467B
:10BF080057E7012090E62B7884F8343494F881348C
:10BF180043F0010384F881344BE700BF9C1C0020E8
:10BF280028150020601500209E1C002037B50B4DF9
:10BF38008DF8040004460F2295F8480001A900F086
:10BF48004CFF40B1064A85F81C4192F8813443F011
:10BF5800200382F8813403B030BD00BF28150020CB
:10BF68009C1C002010B5FFF733F90446A0B90B4814
:10BF780005F006FA0A4805F003FA0A4805F000FA3F
:10BF8800094805F0FDF900F095F8FDF74BFE074B61
:10BF9800DB6A9847204610BD0124FBE704200020F7
:10BFA8001C20002034200020902000203822010886
:10BFB8002DE9F04F90F802908BB004468A46019222
:10BFC800B9F1000F60D14579816890F9102090F996
:10BFD80011801960002D55D0817C8DF81610C07C19
:10BFE8004FF0020B05A9CDE902238DF814B000F03B
:10BFF800E1FE029A47B2BA421646B8BF3E46BA4276
:10C008000CDC039BC3F800904D46019B8AF8006046
:10C0180083F8008028460BB0BDE8F08FA268A1899C
:10C02800E3898A420B4434BF002501259A42ECD3A8
:10C03800082305A9E07C8DF8143000F0BBFEE289E6
:10C04800A368B3FBF2F102FB1133012B4FFA80F81E
:10C05800DBD122238DF81430E07CA37C8DF81560A9
:10C0680005A98DF8163000F0A5FE46B2B742CCD12E
:10C078002579002DC9D0E07C8DF824B007A900F0FF
:10C08800A7FEC1E71646C0E70025C3E7704770471B
:10C09800704770470020704770477047704700200E
:10C0A800704700207047002070470020704700202C
:10C0B80070477047704770470220704702207047EA
:10C0C8000220704770470020704770477047002073
:10C0D80070470020704770477047000010B5054C46
:10C0E800FC222046002102F03BFE0020C4E90000AB
:10C0F80010BD00BFB82100202DE9F041804615464B
:10C10800002942D0244B002403F1010C1A462001D7
:10C11800103312F8016F002E39D19A42F9D11F4F0E
:10C128003B680BB9C7F800C07B680BB1C3F800C007
:10C138003B18002201349A6083F80C800D302301EB
:10C14800AAB23844FD50C7F804C002F0F5FDB8F1B2
:10C15800050F17D0A8F10808B8F1020F8CBF4FF0EF
:10C1680000084FF0010807EB041400236371D7F8A7
:10C17800F83084F8048001332B44C7F8F83030468F
:10C18800BDE8F0814FF00108EDE70126F7E701343B
:10C198000F2CB9D10226F2E7BF210020B8210020D8
:10C1A80010B510B3124A1368984204D1036813609B
:10C1B800002304E00B4613B119688842FAD151688C
:10C1C800884208BF53600BB101681960D2F8F83093
:10C1D8008168013B00245B1A04602146C2F8F830EC
:10C1E800102202F0BDFD204610BD0120FCE700BF73
:10C1F800B8210020054B1B6813B11A798242FAD185
:10C20800002B0B600CBF032000207047B8210020D2
:10C2180010B5054B186800B910BD037B04680BB94D
:10C22800FFF7BEFF2046F6E7B821002010B5074B00
:10C23800186800B910BD03790468052B02D0083BC3
:10C24800022B01D8FFF7ACFF2046F2E7B821002007
:10C2580028B1044BD3F8F830036000207047012060
:10C26800704700BFB82100202DE9F04107460E466F
:10C2780015463AB331B3144B1C6800232CB9304629
:10C28800FFF7E6FF0020BDE8F081A268F91A013245
:10C29800914210D32279EA54581C22895FFA80F817
:10C2A800611D55FA80F002F047FDA36824689844A0
:10C2B8005FFA88F3E2E720462468FFF771FF002C55
:10C2C800F9D1DCE70120DEE7B82100200238C0B24E
:10C2D80011289ABF014B185C00207047BF1B01084A
:10C2E80030B50B4B93F820200446084672B1002164
:10C2F8001C330578A54208D001319842CDB20CBF55
:10C3080004480430AA42F4D8002030BD1046FCE7A7
:10C31800B4220020C022002010B5084C0023206061
:10C32800142204F10C00FF2184F82030C4E9010034
:10C3380002F016FD012384F8213010BDB42200203C
:10C3480010B50E4A92F82010042915D8936804787D
:10C358001C7044785C70C078D870013100209870E7
:10C3680082F8201002F11C018B4214BF043302F141
:10C378000C039360012010BD0020FCE7B4220020CC
:10C38800094B93F8200068B15A6803F11C018A42EE
:10C3980000F1FF3014BF043203F10C0283F82000CF
:10C3A8005A600120704700BFB422002010B5074B27
:10C3B80093F820200446084632B15968FFF790FFE9
:10C3C80010B101234470837010BD00BFB422002057
:10C3D80008B5064B93F820202AB15968FFF780FF6B
:10C3E80008B1407808BD0120FCE700BFB422002056
:10C3F80030B50A4A92F82010536882F8210061B1DA
:10C40800916801241C32DD78587005B99C709342FC
:10C418000CBF034B04339942F5D130BDB422002040
:10C42800C022002008B5044B5968FFF759FF0038AF
:10C4380018BF012008BD00BFB42200202DE9F34138
:10C448000422154E044600210DEB020096F82080C8
:10C4580002F086FC0025EBB2984502D802B0BDE890
:10C46800F0817368197821705A7862709F785FB18B
:10C47800336820469B689847FFF782FF17B901A8E1
:10C48800FFF75EFF0135E6E7DB788DF804108DF8DD
:10C4980005208DF80730EFE7B4220020014B93F810
:10C4A80020007047B4220020034B93F82000042892
:10C4B80094BF002001207047B42200201FB500243B
:10C4C800CDE90244C41F8DF800408DF801100C0A14
:10C4D800ADF80420090C120C8DF803108DF8062015
:10C4E8008DF8073002461B0A012168468DF8024084
:10C4F8008DF8083002F091FA002818BF0F2004B018
:10C5080010BD2DE9F04188B017460D460F9A064632
:10C5180000284DD000240121CDE904448DF81010E5
:10C528009DF838108DF81510ADF81630190CCDE9B6
:10C5380000441B0ECDE902448DF81930ADF81A20DD
:10C54800130C120E07948DF818108DF81C308DF806
:10C558001D20E3B24FEA0318002D5FFA88F803DCC8
:10C56800002008B0BDE8F081013310218DF81F309C
:10C578003A466B460DEB010002F0E5F90346C8B9EF
:10C58800102DAC46A8BF4FF0100CDAB2624503F18B
:10C59800010303DB103D2DB20134DAE708EB02009A
:10C5A80020326A44315C12F8202C4A403254ECE7BD
:10C5B8000A20D6E70F20D4E70138032815D8DFE88A
:10C5C80000F002080C100A4B1B681B690B60002066
:10C5D8007047074B1B685B69F8E7054B1B689B694D
:10C5E800F4E7034B1B68DB69F0E70520704700BFE1
:10C5F800D82200202DE9F041C4B00C464A9E1746C7
:10C608001D468046B8B3B1F5807F36D84FF488729E
:10C618000021684602F0A4FB492300934FF480737D
:10C62800ADF804302B0C8DF80830330CADF80650FB
:10C63800ADF80A608DF80C3022460023414604A864
:10C648002D0E360E8DF80E308DF809508DF80D60D0
:10C658008DF80F4002F070FB04F110014B9A3B4635
:10C6680089B2684602F059F910B1012818BF0F20A5
:10C6780044B0BDE8F0810A20FAE70E20F8E7000090
:10C6880010B590B10A4C28220021206002F068FB06
:10C698002368084A1A6000204FF0FF32C3E90302FA
:10C6A800C3E90522C3E9072210BD0920FCE700BF42
:10C6B800D822002000010101024B1B6818600020ED
:10C6C800704700BFD822002030B1044B1B68DB68DC
:10C6D80001330360002070470A207047D8220020E9
:10C6E80073B50E46002101911D4633B301A9FFF72A
:10C6F80063FFD0B9019C631C04D0A3B2D31A002BEA
:10C7080010DDE2180E4B2A601B689B786BB9121B70
:10C7180063EB0303B24273F10003ACBF01200020B6
:10C72800C00002E003D12C60072002B070BD230CCA
:10C738001B0403F580331A44E4E70A20F5E700BF39
:10C74800D822002028B1044B1B681C334362002008
:10C7580070470A20704700BFD82200201FB5044642
:10C76800F0B1002303A8039302F0AEF90E4ABDF816
:10C778000C30126820469380E38200F052FA60B9C8
:10C7880004F11803009321680123132202F0BCF876
:10C7980040B9204600F045FA00B1112004B010BDA0
:10C7A8000A20FBE70F20F9E7D8220020F0B505465C
:10C7B80087B01C463BB32F4E3368DB68834257D89B
:10C7C80094F82020002A14BF09220822834205D3A6
:10C7D800204600F05AFA70B111200AE000230190B7
:10C7E8000093A36894F82810606AFFF78AFE00286F
:10C7F800EED007B0F0BD23792168B4F808C0A76867
:10C80800043B9AB209B90A20F3E7B2F5807F2DD824
:10C81800ADF80EC08DF817304FEA174C04F12C0311
:10C828003F0E8DF8117000932F0C08234FF0490E1E
:10C83800ADF80C008DF814708DF816002F0E0DEB66
:10C848000300CDF808E08DF810C0ADF812508DF84F
:10C85800157002F059F808B10F20CAE7204600F019
:10C8680014FA0028B8D13368DD60C2E70E20C0E7AB
:10C878000620BEE7D82200202DE9FF410A9D804608
:10C888000F4616461C46002D5AD0002303A9104611
:10C898000393FFF791FE18B1062004B0BDE8F081BC
:10C8A800039B9C4201D80133F6D1284600F05EF97B
:10C8B800002847D1264B1A78424503D01A794245B9
:10C8C80042D10120AA68BA4240D103EB8002EB6A48
:10C8D80092F801802979CDE90043043992782868D3
:10C8E8003B4689B2FFF786FE0028D6D195F820305E
:10C8F8000194002B4FF00103009314BF4246082215
:10C9080095F82810686A3B46FFF7FBFD0028C4D15C
:10C91800013E032EC1D8DFE806F002070B0F0D4BCE
:10C928001B681C611C62B8E70A4B1B685C61F9E76D
:10C93800084B1B689C61F5E7064B1B68DC61ACE79C
:10C948000A20AAE71020A8E70C20A6E70220A4E7FF
:10C95800F4050020D82200201FB50A460B2A4FF004
:10C968000001CDE90011CDE9021107D00C2A13D03E
:10C978000A2A0FD00B2005B05DF804FB012802D16C
:10C9880020238DF80030684602F047F8002818BFC9
:10C998000F20F0E73023F4E70B21F4E738B505461C
:10C9A80002F036F8044678B97DB9094B1B680B21AB
:10C9B8009878FFF7D1FF38B90C21FFF7CDFF18B9E8
:10C9C8000A21FFF7C9FF00B10F24204638BD00BF78
:10C9D800D82200202DE9F04380468FB00C46174638
:10C9E800002A6BD0002969D0002529461D2206A8F7
:10C9F800059504F0D7FE8DF81350344D2B680DF1D2
:10CA080014099E88CDF804900DF1130302933B7925
:10CA180000933B6832462146404602F01AF8002847
:10CA28004ED138683A79494602F086F9384600F01E
:10CA38004FF8002846D13C7AFA79BB79240444EAB5
:10CA480002241C432B689A6894423DD99C609DF847
:10CA580013000B21FFF780FF034658BB0C21FFF79B
:10CA68007BFF034630BB0A21FFF776FF034608BB6E
:10CA78007B7ABA7AFF7A3F0447EA02271F433A468D
:10CA8800334621460920FFF719FD034690B933467E
:10CA98003A4621460820FFF711FD034650B92A6897
:10CAA8009DF8131091700021D1604FF0FF31C2E959
:10CAB8000411916118460FB0BDE8F0830A23F9E725
:10CAC8000F23F7E71023F5E70323F3E7D822002025
:10CAD80010B50446002845D00168002942D011F855
:10CAE800013B43710322063002F026F92046032257
:10CAF80050F8091B043102F01FF92168CB79E36073
:10CB08000A7A43EA0223E3604A7A43EA0243E3608B
:10CB18008A7A43EA0263E360CB7A23740B7B6374FB
:10CB28002379212B1AD110220D3104F1120002F0C1
:10CB380003F91D222168501C8B5C6362085C43EA80
:10CB48000023901C6362085C033243EA004363627B
:10CB58008A5C43EA02636362002010BD112B03DC88
:10CB68000D22E7E70220F8E70120F6E710B50446B2
:10CB7800002854D00168002951D00B7843714B78B4
:10CB880083608A7843EA02238360CA7843EA0243CF
:10CB980083600A7943EA026383604B7903738B7974
:10CBA800C381CA7943EA0223027BC38102F00F02E0
:10CBB8000831103002F0C0F8237B002203F00F0385
:10CBC80084F8202084F82820227903F10800111A1B
:10CBD80004290DDD21680933043AD21A085C84F867
:10CBE8002000D2B2606A84F82820194402F0A4F820
:10CBF800237922681A44002012F8043CE36212F8F0
:10CC0800031C43EA0123E36212F8021C43EA0143CE
:10CC1800E36212F8012C43EA0263E36210BD0220CA
:10CC2800FCE710B5044660B3036853B30279162ACB
:10CC380029D942791A700146082251F8060B0130A9
:10CC480002F084F82146082251F80E0B093002F050
:10CC58007DF82368E28A5A74E38A22681B0A93746F
:10CC68002368A269DA74A36922681B0A137523680A
:10CC7800628B5A752368E27E9A7517232371002008
:10CC880010BD0120FCE70220FAE738B50446002869
:10CC980063D00168002960D0037B90F8282003F056
:10CCA8000F03002A57D108332079043213449842DD
:10CCB80055D363790B702368A2685A70A3682268F9
:10CCC8001B0A937023686289DA702368E27A1A7102
:10CCD8002368227B5A712368E2899A71E389226862
:10CCE8001B0A2146D371227B51F8100B02F00F0268
:10CCF800083002F021F8237B94F8282003F00F0372
:10CD080003F108052AB1226894F82010515503F15F
:10CD18000905206894F82820616A284402F00CF874
:10CD280094F828302268E16A2B44D1545A1CE16AED
:10CD3800206892B2090A81549A1C2168E08D92B247
:10CD48008854DA1C216894F82F0092B2043388546E
:10CD58002371002038BD0933A6E70120FAE7022035
:10CD6800F8E70000024B1A8810431880704700BF8C
:10CD7800DC22002008B5074B1B883BB1FEF728FAD8
:10CD880000280CBF00206FF0020008BD6FF0010002
:10CD9800FBE700BFDC22002010B5034B00241C80F9
:10CDA800FEF70CFA204610BDDC220020B0FA80F015
:10CDB8004009704782B018B9084602B000F0D0B8F0
:10CDC800002002B0704710B9084600F081B97047DA
:10CDD80010B9084600F098B970470346084611464E
:10CDE8000BB900F0EFB90020704710B9084600F001
:10CDF80079BD704710B9084600F010BA0020704796
:10CE080010B40446084611461A46019B14B910BCD2
:10CE180000F022BA10BC70470346084611460BB909
:10CE280000F04CBA0020704710B40446084611467A
:10CE38001A4614B910BC00F0B9BA002010BC7047EB
:10CE480030B40546084611461A46DDE902341DB9D4
:10CE5800029430BC00F036BB002030BC704710B9DB
:10CE6800084600F0E7BB0020704710B9084600F0FC
:10CE780077BD0020704710B9084600F0F6BB0020C7
:10CE8800704710B9084600F0F3BB0020704703460E
:10CE9800084611460BB900F00DBC0020704710B4CD
:10CEA8000446084611461A46019B14B910BC00F006
:10CEB80003BC092010BC704710B9084600F070BDCB
:10CEC800704710B40446084611461A4614B910BCF7
:10CED80000F090BDC8B210BC704700000048704711
:10CEE80003000101064B10B51B6A0446984730B190
:10CEF8000448054B204498428CBF0020012010BDF7
:10CF08003822010840C220C980B92A00F0B5114B67
:10CF180085B00C4610491F56054601F079F80F4BAD
:10CF2800E4B25E6A072D4FF00103CDE902430146E2
:10CF38000AD105220023CDE900234FF47A727A43FF
:10CF48001846B04705B0F0BD08220020CDE9002002
:10CF58003A46F5E7FB1B0108D41B010838220108F3
:10CF68001FB5002300930378013B382B22D8DFE854
:10CF780003F01D252121211F212121214244464F53
:10CF88002156595C5F62656821701F72777C7E212B
:10CF980021818527212121212121212121212121AF
:10CFA8002187898E2121878E21909400C3780BB127
:10CFB80002230093009805B05DF804FB8378F6E738
:10CFC80043788DF8043005238DF805308378003BCD
:10CFD80018BF01235B008DF8063010238DF8073049
:10CFE800314B1B6801A803F59062CDE9022300F0DC
:10CFF800EFFF0090DEE74023DBE72023D9E78278C4
:10D0080090F9013012B9294AD35CD2E7284AFBE7E4
:10D01800827890F90130002AF8D1264AF4E740F6E0
:10D02800B833C6E74FF47A73C3E74FF4FA63C0E73F
:10D0380041F28833BDE741F27073BAE74FF4804399
:10D04800B7E71D484FF47A7101F05AFE00F5FA600F
:10D05800CFE71A4BADE7144B1B6803F59063A8E7BD
:10D06800114B1B6803F28C43A3E71023A1E70E4B77
:10D078001B689EE74FF0834300939BE7104BFBE749
:10D08800104B96E740F21123ADF8003092E70323E6
:10D098008FE790F901300C4AB6E70C4990F9010086
:10D0A80000F0B6FFA5E700BFE42200200B1C010832
:10D0B800131C01081B1C010818FCFFFF00EA0637B7
:10D0C8009A99094040F70937FB1B0108D41B01084E
:10D0D80037B50B4B02781B680C2101FB02335B7AD6
:10D0E80003EB4304074B1D6803690093C368427848
:10D0F800816805EBC40000F00BFD03B030BD00BF34
:10D10800E4220020E022002070B586B0027A642371
:10D11800ADF80030012A4FF00003CDE90133CDE925
:10D12800033301468DF802308DF814302FD0022ACF
:10D1380038D052BB006840B34B6833B31E4A1F4D0A
:10D148001060694618222B6001F0F6FD1C4B2C6814
:10D1580093E807000C3384E8070093E8070004F11C
:10D168000C06032386E80700A4F88C34012204F295
:10D178008C4104F5906000F0BCFC2B684FF6B0724F
:10D18800A3F898240522C3F89C2406B070BD0B4967
:10D1980008684360036100F28C4100F5906000F07C
:10D1A800A8FCF2E7054B1B68B3F88024B3F88C148D
:10D1B8000A43A3F88024E8E7E0220020E4220020C4
:10D1C8005C19010808B503460A2924D8DFE801F0EC
:10D1D80006232323230B161B23212100BDE8084027
:10D1E8000068FFF77FBE90F900009978052271B9B1
:10D1F80000F03FFC003818BF012008BD052293F954
:10D2080000000021F4E790F900005978EEE70221C8
:10D21800EEE70722F3E70020EFE7000010B50479F6
:10D228001CB1012C0BD0002010BD0A4B01681B68F3
:10D23800012203F5906000F05CFC0120F4E7054B47
:10D2480001681B68224603F28C4000F052FC20461D
:10D25800EAE700BFE4220020F7B50528144D1C4674
:10D26800A8BF052058700E462946174600F0D0FE84
:10D2780094F90130A070072B13D1322000F0C8FDBB
:10D288000C4BDB6D0546984704F10C020834034645
:10D29800019200943A463146284600F0BEFD03B09C
:10D2A800F0BD054A55F82310D05C00F0A9FDE7E76A
:10D2B800D41B010838220108FB1B01082DE9F04F97
:10D2C800344F90F901607B68D0F804908BB0044625
:10D2D800884698470546002859D1E37C73B92E4AF9
:10D2E8002378126803EB4303990002EB8303D3F816
:10D2F8000490B9F1000F01D152F80190274B48462C
:10D3080013F906B0FB689847A37CD7F818A02289C0
:10D318000993072E28D100230121CDE90223204AB1
:10D328000693CDE90431CDE907330521CDE9002184
:10D338004FF47A7202FB0BF24CF250311846D04788
:10D34800637C13B3174B995D7B6D0D31C9B22846C9
:10D358009847E07C3246494600F06CFE88F8006049
:10D3680001200BB0BDE8F08F002101250823CDE98D
:10D378000013CDE90715CDE90511CDE90311029296
:10D38800A1782B465A462846D9E7074BDBE7002009
:10D39800E7E700BF38220108E4220020FB1B010850
:10D3A800854501001B1C01080B1C01082DE9F04FE5
:10D3B8008DB090F90130DFF8F8A0DFF8F890CDE9EA
:10D3C8000A123D4A017812F903B0DAF800203B4B03
:10D3D8000C2505FB01221B68527A182101FB023338
:10D3E800044693F9021090F9020000F00CFE34494B
:10D3F800064694F9010000F00BFEA26861688046B9
:10D40800304600F032FD2178DAF80020D9F80C30E7
:10D418006943074650589847D9F81C309C4694F9F8
:10D4280001300025072B4FF47A63CDE90753CDE986
:10D4380005552DD10123CDE903530523CDE901532A
:10D448004FF47A7303FB0BF300933946434646F2D5
:10D45800A81228466746B8472378DAF800200C2136
:10D468004B4394F90110D05800F006FEA18994F9B5
:10D478000100FFF74BFD0B9B217B1860D9F8543056
:10D48800284698470A9B01201E700DB0BDE8F08F12
:10D4980001200823CDE90350CDE901032A46CDF840
:10D4A80000B0654643463946A84701200546D3E7FC
:10D4B800E422002038220108FB1B0108E02200209A
:10D4C800D41B01082DE9F04F8FB0002405468A4689
:10D4D800914698460494ADF81440ADF802400726EA
:10D4E8004FF0010B2B7AA34206D9686804A920449F
:10D4F80000F020FC00285ED102238DF8083002A835
:10D508006B7A8DF80A30FFF72BFDAB7A8DF81D305A
:10D518009DF811308DF81E309DF812308DF81F30AF
:10D528009DF810308DF82030EB7A8DF821302B7B68
:10D538008DF822306B7B8DF8233010238DF81C601A
:10D548008DF824303A4E8DF82C000DF102030A9321
:10D5580005238DF82D3033680C930723ADF834304C
:10D568002B6806930DF1120204AB0DF1110106A808
:10D5780000F0FAFB072805460BD130680C22002181
:10D5880000F5906001F0ECFB3368BDF80220A3F8C9
:10D5980080249DF811308AF800309DF8123089F8FF
:10D5A80000309DF8103088F80030189B28461C7011
:10D5B8000FB0BDE8F08F9DF81330BDF81470ADF8CA
:10D5C80002702044C4B2F3B917B3194A0020116895
:10D5D800072602464FF00C0C062B1BD10CFB00FE55
:10D5E80051F80EE0BEF1000F04D00BFA00F23A43F6
:10D5F80097B2012201301028EED1002A3FF472AF11
:10D60800ADF802706EE75A1E042A01D9062BDCD049
:10D61800062667E747FA00FE1EF0010FEAD00CFB6A
:10D6280000FE51F80EE0BEF1000F08BF0626E1E744
:10D63800E422002038B505464068FFF753FC052270
:10D64800841D002195F90000E4B200F012FA08B92F
:10D6580004F0FD0495F901000722002100F009FA01
:10D6680008B904F0FB04204638BD002070470000CC
:10D6780010B503780F2B044618D84068FFF732FC22
:10D6880022780B4902EB42020968831C01EB8200F5
:10D6980051F82220DBB21AB903F0FD0358B210BDCD
:10D6A800032B06BF626842600223F7E70020F6E713
:10D6B800E4220020022070472DE9F04FDFF838817E
:10D6C8000446D8F8000099B08946174600211E463E
:10D6D8000122032300F59060CDE90611CDE9081178
:10D6E8008DF814108DF81510ADF8163000F0E3F928
:10D6F80038B9D8F80020B2F8803443F00303A2F810
:10D708008034D8F80020637A8DF8283002F59061CB
:10D71800CDE90B12394A94F9083012680D920DF1CF
:10D7280016020F922268109262681192D4E90301DE
:10D73800A27A8DF8482001228DF8492013AA82E8A0
:10D7480003001025227DE18A8DF8293018468DF8CE
:10D758005420ADF83850FFF7D9FB0AAB17930DF1F9
:10D768001503169000933146019705AB06AA10A839
:10D7780000F0EAFB064698BB9DF81410204F0139CB
:10D7880001F0BEFA1F4B1B690393C4B24FF00C0B98
:10D7980004F160036B44D8F8000013F848AC9DF816
:10D7A80014300BFB0AFC01343946B4FBF3F203FBDB
:10D7B8001244D0F89C34B0F9982450F80C00DDF8E5
:10D7C8000CC0E4B2E04728B189F800A0304619B08F
:10D7D800BDE8F08F013D15F0FF05D9D10D26F5E71D
:10D7E8000C2801BFD8F80020B2F8803443F00303B6
:10D7F800A2F88034EAE700BFE4220020E0220020FB
:10D80800400D030038220108F8B50679012E0546B7
:10D8180001D80620F8BD0F2E2BD80368187A40F3DC
:10D8280003000522002140B200F023F92B680446CA
:10D83800187A40F303100522002140B200F019F9CC
:10D84800A8B1B4FA84F4640929680B7A086843F328
:10D85800030243F3031352B25BB29A42C8BF0124D6
:10D86800FFF740FB48B9002CD3D10420D2E70124AC
:10D87800EAE70320CEE70520CCE7002CFBD10C4FCC
:10D8880029683B6806EB460003EB80000C2201F098
:10D8980053FA3A680C2303FB062320465C72B2F85D
:10D8A80080140123B3400B43A2F88034B2E700BFD1
:10D8B800E422002010B4017801290ED9084B186819
:10D8C8000C234B43C4180022C250C4E9012200F5BE
:10D8D800906010BC102200F0D5B8002010BC704732
:10D8E800E42200202DE9F04186B050238DF8143051
:10D8F8000379102B074630D10368DD7B6DBB02240A
:10D90800A8466426062C14D83A68535D03932A4423
:10D91800517843EA01230393927843EA024373431D
:10D92800CDE9033863B968468DF80040FFF7C2FFB8
:10D938000DE0CDF80C808DF81480CDF81080F2E75A
:10D9480003AB01A801938DF80840FFF75DFF013490
:10D95800E4B2102C05F10305D4D106B0BDE8F0817E
:10D968001FB502680379116851B901A88DF8043010
:10D97800FFF7A0FF78B9002040B205B05DF804FBBE
:10D9880002A802928DF80C30FFF73EFF0628F2D865
:10D99800024B185CF0E70320EEE700BFF41B010818
:10D9A80070B5114E01783268104B0C2505FB012229
:10D9B8001B68527A182101FB0233044693F90210BE
:10D9C80090F9020000F01FFB2378326861686B430E
:10D9D800D558A26800F049FA054BA289DB6B0146CD
:10D9E8002846BDE870401847E4220020E0220020C5
:10D9F80038220108074B9B56C91A431E5842584102
:10DA080040008842B8BF08460528A8BF0520C0B214
:10DA1800704700BF031C0108F0B59A42069D03DB5E
:10DA28009DF914309A4220DD0020F0BD03EB43033A
:10DA380031F814C005EB830300264CFA06F7FF07FC
:10DA480007D51F7A07F00F0E724502DBB2EB171FDE
:10DA58000DDD0136102E03F10C03EED10134E4B2D2
:10DA68002301DBB29842E1D8DEE70024F8E7012081
:10DA7800DBE7884204DB9042CCBF002001207047DE
:10DA88000020704710B51409B4EB111F03464FEA84
:10DA980011100ED391420CD202B201F00F0133F8EB
:10DAA8001240012000FA01F124EA010123F81210C2
:10DAB80010BD0020FCE7F0B528B100EB41050127B7
:10DAC8000020914200D3F0BD002435F802CB234654
:10DAD80007FA04F636EA0C0608BF013304F101041C
:10DAE80008BFDBB2102CF3D118440131C0B2C9B25F
:10DAF800E7E710B500B149B910BD31F8134020F877
:10DB080013400133DCB2A242F7D8F5E70023F9E766
:10DB180082B030B5048804936AB9B3F5616F18D33D
:10DB280049F6AF2542F21072AB4298BF4FF47A72B1
:10DB3800944238BF1446012C38BF01246143BDE824
:10DB48003040C3688B428CBF5B1A0023C36002B0AD
:10DB580070476422ECE700002DE9F04F91B01546BC
:10DB6800DDF86C8004939DF8683009930C460646EE
:10DB780003F0C2FB684ADFF8A4B10590A8F5F633B4
:10DB8800303BB3FBF2F3534303F5F63203F5A83306
:10DB980003F5C0730393182313FB05433032069231
:10DBA800089300254FF0FF3A089BA34207D1002DA8
:10DBB80014BF50464FF0FF3011B0BDE8F08FBDF9EB
:10DBC8007030ADF82C300B99CDF86C804046CDF80C
:10DBD800288003F021FBB4F800906EB9B8F5616FA6
:10DBE8005BD349F6AF2242F21073904598BF4FF4C9
:10DBF8007A73994538BF99464B46012B38BF0123A4
:10DC08000793002E52D1B9F1640F48D1A0605F4646
:10DC1800A1680EA803F022FB0F9B0093DDE90A120E
:10DC28000E9B0CA803F079FA049B0C9A0BB9099B7C
:10DC38002BB12369BB4202D1394B9A420DD9394BDA
:10DC4800E760984509D90023ADF83430069B0D9953
:10DC58000C93184603F0E0FAA060606800B9E7602A
:10DC6800276126B103F052FBE3680344E360D4E97B
:10DC780003329342059B1D996360079B88BFE2604E
:10DC88004B43E168994202D20498A8B9A6B101238E
:10DC98001D442375EDB2183486E76423A9E7B9F566
:10DCA8007A7F0ABF204F214FA060B1E7049B0BB9D0
:10DCB800C4F80CB05F46D0E700209342207506D820
:10DCC8005B1A9A4505F1010528BF9A46EDB2002E68
:10DCD800E1D1B9F1640F164AADF8346019D049F6AC
:10DCE800B023B9F57A7F18BF1346904584BF039ACD
:10DCF8009B180C931C9B00930CAF97E806001B9B8A
:10DD0800384603F00AFA97E8030003F085FA8246DA
:10DD1800C1E74FF46163E8E78051010040771B00D9
:10DD28007F5101002FEC010080A81201002E930200
:10DD380030EC01000378032B14D1437803F00F0271
:10DD48001B098A704B7083788B80C27843EA022360
:10DD58008B800379C3F3021203F00F03CA700B70B0
:10DD680005207047002070472DE9F347984643790E
:10DD7800057990F907609146044690F906208A468D
:10DD880083B190F9087075B30F2A12D194F909205C
:10DD98000F2E1ED194F90A60072D24D1002F08BF39
:10DDA800012720E090F90B7090F9092090F90A609A
:10DDB800E9E7A369019394F915300093216994F96F
:10DDC8001430207BFFF728FE0028E1D105F0FD057F
:10DDD800DEE794F91D30B3420FDC94F91C30B342EE
:10DDE800DADA05F0FB0528468AF8002089F8006091
:10DDF80088F8007002B0BDE8F0871E46CCE7000046
:10DE0800024B03FA00F0B0FBF1F0704740420F00FC
:10DE18004FF4FA53B3FBF0F0704730B54FF47A750E
:10DE28000C1F6A4300FB042252001EBF00F1FF349E
:10DE38001219B2FBF0F2914238BF1146039A1160F1
:10DE4800820048431CBF013040084FF47A71121A0F
:10DE580001FB1323002BCABF03F2E73393FBF1F155
:10DE6800B3FBF1F1049B196030BD38B5400014468E
:10DE78000D46F3F7CBFD01462846F3F715FD21467D
:10DE8800F3F712FDF3F704FC03F0D2FCF3F7E0FC20
:10DE980040B238BD2DE9F74F019300231F469C4639
:10DEA8001C01058A5FFA84FE04F0F004A54206D836
:10DEB800019B82F800C01F7003B0BDE8F08F0EEB25
:10DEC8004E054FEA4309AD000024466836F809605C
:10DED8002641F60727D5866806EB050A765916B354
:10DEE800067836B9466926B136F809602641F6073C
:10DEF80019D59AF8086090F901B046F303084FFA6B
:10DF080088F8D8450FDC46F3031676B25E450ADB7F
:10DF18009AF8096006EB4608C66806EBC806367D1F
:10DF28004EB90137FFB20134102C05F10C05CCD1E4
:10DF38000133DBB2B4E70CF101060EEB040801F87B
:10DF48000C805FFA86FCEEE72DE9FF47044640683F
:10DF5800DDE90C671D468A46914603F0D7F9236828
:10DF68001B1A3B604FF000080123337085F80080CE
:10DF7800636813B12368834224D8CAF80080D4F8B0
:10DF88001CC0A3699CF800E00393D4E9030101AB2A
:10DF980083E80300237D0093DCF80C10237A627A6F
:10DFA8007046FFF7D9FD334638602A46E06949468E
:10DFB800FFF770FF2B782BB1C7F80080002004B062
:10DFC800BDE8F0873378002B14BF0B200C20F6E750
:10DFD80037B590F9002090F90250954204460FD0C9
:10DFE800013A52B295420BD0A368019394F90130DB
:10DFF80000936168E0782B46FFF70EFD0028EFD00C
:10E00800104603B030BD8842B8BF084670470000CC
:10E0180051F82000054B984205D0054BC31A5842C9
:10E028005841400070470120704700BF90D003005E
:10E0380020A1070005281FB50ED80C4B53F8203037
:10E048000093CDE901120A4B01220021022002F0BF
:10E0580069FE05B05DF804FBCDE90012054B01220D
:10E068000021022002F05EFEF3E700BF901C0108C9
:10E07800231C0108421C010807B5054BCDE9000126
:10E0880001220021022002F04DFE03B05DF804FBDE
:10E098005E1C010810B5102204460021F13000F082
:10E0A8005FFE0021C4F814112046F022BDE810409C
:10E0B80000F056BE02460846102100F0A5B92DE929
:10E0C800F0430446D0F8140185B00E46154604F214
:10E0D800011988B3C0F110089045474628BF174674
:10E0E800BAB2484400F028FED4F814313B440F2B50
:10E0F800C4F814312DD9A8452BD204F1F00304F546
:10E10800807113F8012F187C8B4282EA00021A7082
:10E11800F7D104F1F10810224146684600F00CFEE0
:10E1280022466946684600F0E9F9102269464046E9
:10E1380000F002FE3E44ED1B04F5807804F1F1077F
:10E14800102D09D8AAB23146484600F0F5FDC4F8AA
:10E15800145105B0BDE8F08304F1F003711E13F803
:10E16800012F11F8010F434582EA00021A70F6D117
:10E1780010223946684600F0DFFD224669466846A7
:10E1880000F0BCF910226946384600F0D5FD10367B
:10E19800103DD5E7F0B589B00C46102200210546A0
:10E1A800684600F0DDFD22466946684600F0A6F99B
:10E1B8009DF90030002B6A464FF0000143DA1378CE
:10E1C80012F8010F01315B0043EAD0130F2902F85E
:10E1D800013CF4D19DF80F305B0083F08703D4F83D
:10E1E8001401DBB210288DF80F303BD104F5807391
:10E1F800694604F5887013F8016F11F8012B9842ED
:10E2080082EA06021A70F6D104F1F00304F580716F
:10E2180013F8012F187C8B4282EA00021A70F7D19A
:10E2280010220DEB020004F1F10100F085FD2246F9
:10E23800294604A800F062F910220021684600F07F
:10E248008FFD09B0F0BD137812F8010F01315B00A2
:10E2580043EAD0130F2902F8013CF4D19DF80F309E
:10E268005B00BCE79DF90030002B6A464FF00001C7
:10E2780037DA137812F8016F01315B0043EAD613DD
:10E288000F2902F8013CF4D19DF80F305B0083F0B0
:10E298008703471CDBB28DF80F30102F04EB000307
:10E2A800C0F10F064FF0800288BF002600F581708C
:10E2B80083F801210021324620443E4403F072FADB
:10E2C800C4F8146104F58073694604F5887013F87E
:10E2D800016F11F8012B984282EA06021A70F6D1F2
:10E2E80092E7137812F8016F01315B0043EAD61305
:10E2F8000F2902F8013CF4D19DF80F305B00C8E704
:10E308000A780378534003704A784378534043703F
:10E318008A78837853408370CA78C3785340C3702F
:10E328000A790379534003714A7943795340437119
:10E338008A79837953408371CA79C3795340C37109
:10E348000A7A037A534003724A7A437A53404372F3
:10E358008A7A837A53408372CA7AC37A5340C372E3
:10E368000A7B037B534003734A7B437B53404373CD
:10E378008A7B837B53408373CA7BC37B5340C373BD
:10E38800704710B50B7814786340037054784B7855
:10E398006340437094788B7863408370D478CB78EB
:10E3A8006340C37014790B796340037154794B79D6
:10E3B8006340437194798B7963408371D479CB79C5
:10E3C8006340C371147A0B7A63400372547A4B7AB0
:10E3D800634043728B7A947A63408372D47ACB7A9F
:10E3E8006340C372147B0B7B63400373547B4B7B8A
:10E3F80063404373947B8B7B63408373CB7BD27B7B
:10E408005340C37310BD0000A1F11003DBB2102B01
:10E418002DE9F04704D8374C24FA03F3DB0705D479
:10E42800002382F8F030FF20BDE8F087531E44181F
:10E43800A0424ED101F11C039B005FFA83F9C3F39C
:10E448000313013B2C4D82F8F03001240B46D618FB
:10E45800B3FBF1F001FB103010F0FF0016F804AC2C
:10E4680016F803EC16F802CC16F8017C36D115F82C
:10E478000E8015F80CE015F807C015F80A70E009C9
:10E4880000EB400084EA080800EBC0006400C0B25A
:10E49800E4B24440C246581AC0B212F800808AEA70
:10E4A800080A02F803A01044043390F801808EEAA9
:10E4B800080E86F801E090F802E08CEA0E0C86F867
:10E4C80002C0C078DBB247409945F770BFD800203A
:10E4D800AAE710F8015B03F8015FA9E71829DAD960
:10E4E800102801BF15F80AA015F80EE015F80CC0A1
:10E4F800EF5DD0E701010100A81E01082DE9F04FEA
:10E50800A3B092F8F0301D911B920193002B00F0FC
:10E51800538101461EA8FFF734FF1B9BA74CA84D4B
:10E52800A84E10330293002303939DF87C000490B7
:10E538009DF886000590205C06909DF87B0007906A
:10E54800205C089004989DF881C0205C099014F81C
:10E558000C000A909DF880000B909DF885009DF8AE
:10E5680078809DF87DE09DF882A09DF887900C90BA
:10E578009DF87A00029B1C9314F80A2014F80930BD
:10E5880014F8081014F80E700D90205C0E909DF889
:10E598007F000F90205C10900B98205C11900C98D5
:10E5A800205C12909DF8840013909DF879001490D7
:10E5B8009DF87E001590205C16909DF883001790BA
:10E5C800205C18901398205C19901498205C1A907D
:10E5D8000398013003900298DDF804B010300290DF
:10E5E8009DF80C00834536D88DF878108DF87A2080
:10E5F80009990E9A8DF87C108DF882201199069A47
:10E608008DF880108DF87E201999169A8DF884104F
:10E618008DF886200A99189A8DF87D108DF8872034
:10E628001299109A8DF87B301B9B8DF881108DF80C
:10E6380083201A99089A1D988DF885108DF87F20E7
:10E648001EA903EB0B128DF87970FFF79AFE0020D4
:10E6580023B0BDE8F08F15F808B082EA03008BEA12
:10E66800000016F80EB080EA0B008DF8780015F857
:10E678000E004B40434016F80A0043408DF87930AD
:10E6880081EA070315F80A10594016F8093059406D
:10E6980016F808308DF87A107A40534015F809209A
:10E6A80053408DF87B30089A069B5340049AAA5C25
:10E6B800534016F80C2053408DF87C30DDE90832C1
:10E6C8005A4015F80C305340059AB25C53408DF807
:10E6D8007D30DDE909325A40059BEB5C5340079ACF
:10E6E800B25C53408DF87E30069B0A9A5340049AD8
:10E6F800B25C5A40079BEB5C5A408DF87F200E9B1A
:10E70800109A53400B9AAA5C53400C9AB25C53403F
:10E718008DF88030DDE910325A400C9BEB5C534099
:10E728000D9AB25C53408DF88130DDE911325A40C0
:10E738000D9BEB5C53400F9AB25C53408DF88230CE
:10E74800129A0E9B53400B9AB25C5A400F9BEB5C9B
:10E758001C995A408DF88320169B189A5340139A97
:10E76800AA5C5340149AB25C53408DF88430DDE9BA
:10E7780018325A40149BEB5C5340159AB25C5340D4
:10E788008DF88530DDE919325A40159BEB5C534012
:10E79800179AB25C53408DF886301A9A169B5340EC
:10E7A800139AB25C5340179AAA5C1EA853408DF87E
:10E7B8008730FFF7A5FDB8E6FF2049E7A81E010846
:10E7C800A81C0108A81D010808B538B1044A054964
:10E7D8001060D82200F0B0FA002008BD0220FCE743
:10E7E800E8220020D82301080A4B1A6870B50023D4
:10E7F80002F1180503EB03142E5D864204D1183488
:10E8080022440A60002070BD01330B2BF2D1032093
:10E81800F9E700BFE82200202DE9F041CCB0064618
:10E82800DDF8488117461C460D4631B3B8F1000F94
:10E8380023D006A8FFF72EFC204601A9FFF7D4FF36
:10E848000446B0B9019906A80131FFF733FC26B197
:10E858001022314606A8FFF732FC3A46294606A898
:10E86800FFF72DFC06A902A8FFF794FC029BC8F845
:10E87800003020464CB0BDE8F0810224F9E70000E2
:10E8880030B595B013A90446FFF7AEFF002830D184
:10E898001B490C2303FB00F2555CA5422BD1139BAB
:10E8A800187C1090D87B0F90987B0E90587B0D9019
:10E8B800187B0C90D87A0B90987A0A90587A09901D
:10E8C800187A0890D8790790987906905879059021
:10E8D80018790490D8780390987802900A445B7865
:10E8E8000193936800930022064B1146022002F020
:10E8F80019FA15B030BD01300B28CBD1F9E700BFAC
:10E9080020210108A81F01080B2B10B402D810BC45
:10E91800FFF782BF032010BC704730B50D4685B0A5
:10E928001446014668B103AA002000922A460390C3
:10E93800FFF772FF18B90398001B18BF012005B034
:10E9480030BD0220FBE72DE9F0430D46BFB0144669
:10E958009946804620B31BB311F00F0122D1F02253
:10E9680001A800F0FDF920466946FFF73DFF04467F
:10E9780048B9009801AA10210130FFF745FD2E463D
:10E98800AF1BFFB21EB920463FB0BDE8F08301AA15
:10E9980009EB070108EB0700FFF7B0FD103EEFE7B2
:10E9A8000224F0E70524EEE7F0B5184E3468024675
:10E9B80085B00846002304F1180103EB03154F5DE9
:10E9C80097421ED10D2A05F1190513D10023CDE96F
:10E9D8000033CDE902330C2210216B46FFF7B3FF59
:10E9E8000446306810226946284400F0A5F92046FC
:10E9F80005B0F0BD01461022601900F09DF9002411
:10EA0800F5E701330B2BD8D10324F0E7E8220020E7
:10EA180009B1FFF7C9BF022070471FB51446A0B15E
:10EA28000C2A01D10B2912D10023CDE90033CDE9FD
:10EA380002330A466B461021FFF785FF18B969466D
:10EA48002046FFF7B1FF04B010BD0220FBE703200A
:10EA5800F9E7F8B51E46DDE907479DF818505BB39E
:10EA680054B34FB3212D29D819462A46204600F021
:10EA780063F90122631C691EB018FFF764FFF8B937
:10EA8800E37ADB093B70EBB96319204613F8012CD4
:10EA980013F8021C120642EA014213F8041C0A4346
:10EAA80013F8031C012342EA0122291FFFF735FF4F
:10EAB800003818BF0120F8BD0220FCE70520FAE75E
:10EAC8000720F8E70420F6E710B5044628B1044B00
:10EAD8005B6998472060002010BD0220FCE700BF5A
:10EAE8003822010808B5014630B1044B08221868DD
:10EAF80000F022F9002008BD0220FCE7E8220020EF
:10EB080008B530B1044B0822196800F015F9002047
:10EB180008BD0220FCE700BFE82200207FB5124EA6
:10EB28000023044602A801930D46FFF7E9FF336866
:10EB38005B6901936CB102AA082312F8011B41B961
:10EB4800013B13F0FF03F8D102A8A04702A8FFF782
:10EB5800C9FF35B1019B23B901A8A8473368019AB9
:10EB68005A61002004B070BDE822002008B50146B3
:10EB780038B1054B18680822104400F0DDF8002071
:10EB880008BD0220FCE700BFE822002008B538B124
:10EB9800044B19680822114400F0CEF8002008BD83
:10EBA8000220FCE7E8220020034B1B6802280CBF68
:10EBB8001961596100207047E822002041B1054BD6
:10EBC8001B6802280CBF1B695B690B60002070473B
:10EBD80002207047E822002030B58FB00024054697
:10EBE8000CA80994FFF78CFF9DF8373007939DF820
:10EBF800363006939DF8353005939DF834300493EC
:10EC08009DF8333003939DF8323002939DF83130EC
:10EC180001939DF830300093224621461E4B022076
:10EC280002F080F80AA8FFF7B1FF9DF82F3007938C
:10EC38009DF82E3006939DF82D3005939DF82C30C5
:10EC480004939DF82B3003939DF82A3002939DF886
:10EC5800293001939DF82830009322460F4B214616
:10EC6800022002F05FF809A92846FFF7A7FF9DF8E0
:10EC7800243003939DF8253002939DF826300193A4
:10EC88009DF8273000932246054B2146022002F0CA
:10EC980049F80FB030BD00BF042001084220010828
:10ECA8008020010808B50020FFF7EAFD0120FFF7E2
:10ECB800E7FD0920FFF7E4FD0820FFF7E1FD00204C
:10ECC800FFF78AFF002008BD10B504460B20FFF7A8
:10ECD800D7FD0C20FFF7D4FD0920FFF7D1FD082050
:10ECE800FFF7CEFD0A20FFF7CBFD2046FFF774FFA4
:10ECF800002010BD014B1860704700BFFC050020C4
:10ED08000B4A30B514680B4D43F2390305FB043345
:10ED18001360091A6FF00042B3FBF2F2C2EBC27241
:10ED280001319B1A93FBF1F201FB1233184430BDF9
:10ED3800FC0500206D4EC64101380A44914200D1BD
:10ED4800704711F8013B00F8013FF7E710440A4407
:10ED5800914200D1704711F8013B00F8013DF7E7F7
:10ED680002F020BD30B530B10A4D01444FF0FF33F9
:10ED7800814201D1D84330BD10F8012B53400822FD
:10ED880043F30004013A2C4092B284EA5303002A68
:10ED9800F6D1EDE72083B8ED01207047054B4FF41D
:10EDA80000529A62044B1B6813B15B6803B11847A1
:10EDB800704700BF00040048EC230020054B4FF4C7
:10EDC80080529A62044B1B6813B1DB6803B1184781
:10EDD800704700BF00040048EC2300200120704762
:10EDE8000120704701F048B901F036B910B501F0BB
:10EDF80019FE0E21044640F61F1001F02DF9204699
:10EE0800012101F0F9FDBDE8104001F0D7BA00007A
:10EE180070B50C4E01EB40030D46B3654FF6FF711C
:10EE2800002304461A46084601F05EFB96F8560091
:10EE3800002101F0E1FD29462046BDE8704001F0BF
:10EE480095BA00BF0824002010B5044601F0AAFEB8
:10EE580001281CD101F0AEFE34B11248214602F05F
:10EE680017FB104802F0DAFA0F4C104B00214FF450
:10EE78008052A1659A6194F8560001F0BDFD63784F
:10EE88006BB16FF07F40BDE8104001F053BA00232A
:10EE980040F262211A46084601F026FBDCE7A0682A
:10EEA8008001F0E7F0230020082400200004004837
:10EEB800002001F0BFB9000008B501F0C7F8043818
:10EEC800C0B2032896BF024B0020185C08BD00BFE3
:10EED8003422010808B501F0BAFD033008BD01F07D
:10EEE80049B901F009B908B501F000FD00B208BD43
:10EEF80038B50D46144601F05DFB284601F092FD39
:10EF08000E21054640F61F1001F0A6F828460121FB
:10EF1800074D01F071FD01F051FA4FF47A71614328
:10EF2800284602F0B5FA2846BDE8384002F076BA1D
:10EF38006424002001F03EBB08B5084B002193F87B
:10EF4800560001F059FD00234FF4C0711A460846D7
:10EF580001F0CAFABDE8084001F024BA08240020EC
:10EF680010B5044601F01EFE01281CD101F022FE56
:10EF780034B11248214602F08BFA104802F04EFADA
:10EF88000F4C104B00214FF48052A1659A6194F800
:10EF9800560001F031FD63786BB16FF07F40BDE83A
:10EFA800104001F07DB9002340F262211A4608465C
:10EFB80001F09AFADCE7A0688001F0E7F02300206E
:10EFC800082400200004004808B54FF0040001F0B0
:10EFD80017F9BDE808400220F3F76ABD08B5002319
:10EFE8001A461946184601F07FFABDE8084001F0B4
:10EFF8006DB900001D4B73B51D4D186000241D48E8
:10F008006C70C5E90144AC6501F098FAAC8101F077
:10F0180003FA2146204601F04BFC21460422012038
:10F0280001F0FCFA144E154D4FF6FF7123462246A7
:10F03800084601F059FAFFF7C7FF2246104B009423
:10F048004FF0FF31304602F03DF90E4B0094224656
:10F058004FF0FF31284602F035F9304602F090F9BA
:10F06800284602B0BDE8704002F08AB9EC230020BF
:10F07800082400204500010864240020F023002013
:10F08800A5ED0008C5ED00080128084805D1084B82
:10F09800C17719700E3001F0A7BB437D012B03D156
:10F0A800034B81751970F5E7704700BF08240020ED
:10F0B800000600200D4B10B5044618735873012044
:10F0C80000F016F85CB134214FF4E86000F0C4FF9A
:10F0D8004421BDE8104040F2417000F0BDBF14214A
:10F0E8004FF4E86000F0B8FF2421F2E7082400207C
:10F0F80038B5114C0546207001F061FD052D04D886
:10F10800DFE805F0090B03171709032001F070FA6F
:10F118000023637338BD0020F8E7012001F068FA86
:10F12800207B637B8342F5D06073BDE83840FFF7EE
:10F13800C1BF0220EAE700BF082400202DE9F04300
:10F148001E4687B000230546CDE901330C46174615
:10F1580001F027FD032D61D8DFE815F07B00C3001F
:10F168000E010400A27C082A04D94FF0FF3007B032
:10F17800BDE8F083A16801A801F0DCFE2168002940
:10F18800F3D042F210729142E37C864D51D80322AB
:10F19800AA7385F83820E96385F844304FF00208EF
:10F1A8006368A17DDB002B820423AB74A37CDB00A6
:10F1B800EB7402294FF000032B75637D02D0227D8A
:10F1C800022A42D103F10F02D2B2012A01D9012B3E
:10F1D800CBD1754B754A196803944FF0010903A800
:10F1E8008DF8149001F0DAFC0028BED1287685F855
:10F1F80017906875FFF75CFE4046FFF779FF6C488B
:10F2080001F086FA6B4801F0EFFA01A800F084FFDC
:10F21800208A00F055FFA08900F09AFF384601F0D7
:10F2280001FC604C84F8560001F0C0FC66600020C8
:10F238009DE74FF00008E963890885F80E8085F896
:10F24800388085F844302964AAE7EB7529766A7511
:10F25800D0E72368002B88D0A27C082A85D8514D96
:10F26800A16801A801F066FE002385F838302268FD
:10F27800EA63E27C85F84420A269AB732A64626879
:10F28800A17DD2002A820422AA74A27C2B75D20006
:10F298000229637DEA7402D0227D022A1DD103F17E
:10F2A8000F02D2B2012A02D9012B7FF45EAF3E4B86
:10F2B8003E4A196803944FF0010803A88DF814809A
:10F2C80001F06CFC00287FF450AF287685F8178091
:10F2D8006875FFF7EDFD00208FE7EB7529766A75F5
:10F2E800F7E7304D012185F83810227885F850204D
:10F2F800637885F85130A37885F85230E3788B42EB
:10F3080002D0022B03D03BB985F8533004E00B3A06
:10F31800012A29D885F853104FF0010885F80E8086
:10F32800A388AB83A379AB77E37985F82030237A78
:10F3380085F82130FFF7BCFD4046FFF7D9FE1C4891
:10F3480001F0E6F91B4801F04FFA95F85130062B09
:10F3580040F689000AD100F08FFE00F0FB0140F66C
:10F36800890000F079FE59E70023CDE700F084FE1C
:10F3780040F00401C9B2F2E72368013BB3F57A7F94
:10F38800BFF4F3AE0320FFF7B3FE0648022380F86C
:10F39800383023688364162380F84C30383001F005
:10F3A800B7F93BE708240020EC2300206424002060
:10F3B80040240020162400202DE9F041002686B0C4
:10F3C8001F461446CDE9016680460D4601F0E9FB6B
:10F3D800B442764C16BF0123334637466370B8F102
:10F3E800000F06D0B8F1010F7CD0002006B0BDE8B0
:10F3F800F081AB68002B00F0D680EB68002B00F0A2
:10F40800D280AA7F082A00F2CE80296901A801F0DB
:10F4180091FD2868003818BF012000F0D9FF84F852
:10F428003880AB68E36395F8203084F84430686826
:10F4380001F05AFB84F80E8084F84500EB68DB0085
:10F448002382EB7FA374AB7FDB00E37495F8213054
:10F45800237595F82230002B3ED12A7D95F824108B
:10F46800A275022995F8232001D0022B36D102F18A
:10F478000F03DBB2012B02D9012A40F0948000234C
:10F488008DF814304A4B4B4A1968049503A801F0CB
:10F4980085FB002840F0878001232076E37560759E
:10F4A800FFF706FD0020FFF723FE434801F030F97F
:10F4B800424801F099F901A800F02EFEA88B00F04F
:10F4C800FFFD288B00F044FE4FF4FA53AA687B43F3
:10F4D800B3FBF2F3A36088E7FF22BFE7E27521766A
:10F4E8006375DDE72B8E002B5DD095F83230A86A66
:10F4F800012B0CBF95F814804FF0FF08003818BF97
:10F50800012000F065FFF8B200F06EFF012184F8D9
:10F51800381095F82C2084F8502095F82D3084F870
:10F52800513095F82E3084F8523095F82F308B42B0
:10F5380002D0022B03D03BB984F8533004E00B3AD5
:10F54800012A28D884F853102B8EA38395F83230DB
:10F55800A377AB8E23840126A67384F81F80FFF758
:10F56800A7FC3046FFF7C4FD134801F0D1F8134853
:10F5780001F03AF994F82130B34240F236700CD1D8
:10F5880000F07AFD00F0FB0140F2367000F064FDF7
:10F598004FF6FF739EE70023CEE700F06DFD40F0C5
:10F5A8000401C9B2F0E74FF0FF301FE7082400203C
:10F5B800EC230020F0230020402400201624002003
:10F5C8002DE9F04F85B082460E9DBDF840B09DF8FC
:10F5D80044709DF84890019288461E4601F0E1FA71
:10F5E800BAF1010F524C54D0BAF1040F00F09180D7
:10F5F800BAF1000F3AD10B22304684F8442084F83F
:10F6080038A0E56301F070FA019B23644FEACB034D
:10F61800B9F1000F238241F60403638214BFF22379
:10F628000123E37587F001070123237684F8450059
:10F6380084F80EA084F814A06775FFF739FC5046CB
:10F64800FFF756FD04F1380001F062F804F10E00EE
:10F6580001F0CAF8374A1068516802AB03C302A820
:10F6680000F05AFD40F2FF1000F02AFD404601F07C
:10F67800D9F90E2184F8560040F61F1000F0ECFC72
:10F6880094F8560001F092FA169B636005B0BDE845
:10F69800F08F294984F838A0EAB2895D84F85020AF
:10F6A80076BB0B3D012D8CBF00250125053A012AAB
:10F6B80004D8BBF10C0F38BF4FF00C0B1F4B9DF853
:10F6C8003C201B7884F85350E37701259DF854308B
:10F6D80084F8511084F8522084F82130A573A4F8D6
:10F6E8001CB0A77784F82090FFF7E2FB2846FFF7C5
:10F6F800FFFC134801F00CF8124801F075F8B5E763
:10F70800012E04D1A5F10C035D425D41CEE7002531
:10F71800CCE75046FFF7ECFC022384F8383004F1BC
:10F7280038001623A56484F84C3000F0F1FF9DE7FB
:10F73800082400207419010802220108000600208C
:10F7480040240020162400202DE9F04F87B0DFF870
:10F75800B4B29DF864A09DF84C90029314469DF8AD
:10F7680054309DF85020BDF84880039205468BF828
:10F7780001A0BDF8446001930F4601F012FABAF1F6
:10F78800000F18BF4FF00008DFF87CA2039AB9F108
:10F79800000F08BFFF22012D8AF8002000F0C88062
:10F7A800052D48D0002D40F0C080284600F010FEFE
:10F7B8000B2238468BF844208BF83850CBF83C4065
:10F7C80001F092F9019B8BF8450041F60402002BE9
:10F7D800ABF812209AF800208BF8162014BFF222FA
:10F7E80001228BF81720F600012289F001098BF815
:10F7F80018208BF80E50ABF810608BF814508BF86B
:10F808001590FFF755FB2846FFF772FC0BF13800FF
:10F8180000F07EFF0BF10E0000F0E6FF7B49086860
:10F82800496804AA03C204A800F076FC40F2FF105D
:10F8380000F046FC71E0012000F0CAFD09224FF0FB
:10F8480000098BF8442038464FF44872CBF8402022
:10F858008BF83890CBF83C4001F046F94FF48052D1
:10F86800ABF812209AF800208BF845008BF8162088
:10F8780028460122F6008BF817208BF80E90ABF87B
:10F888001060ABF814908BF81890FFF731FC0BF16F
:10F89800380000F03DFF0BF10E0000F0A5FF5B49BA
:10F8A8008868C96804AA03C204A800F035FC40F2BD
:10F8B800FF1000F005FC40F6B80000F0DDFB00F09A
:10F8C800EF0140F6B80000F0C7FB042140F6B9008C
:10F8D80000F0C2FB40F69B0000F0CEFB00F0E30115
:10F8E80041F0080140F69B0000F0B6FB40F2D16001
:10F8F80000F0C2FB40F01801C9B240F2D16000F03C
:10F90800ABFB40F2AC6000F0B7FB00F08F0141F0B8
:10F91800500140F2AC6000F09FFB4FF4FA5202FB3A
:10F9280008F2B2FBF4F2CBF8082007B0BDE8F08F7C
:10F93800002000F04DFD36498BF83850E2B2C95D21
:10F948008BF85020002F4DD10B3C012C8CBF00248C
:10F958000124053A012A02D80C2E38BF0C26029B36
:10F968009AF800208BF852308BF85340019B8BF8A3
:10F978001F2001249DF860208BF821208BF851105E
:10F988008BF820308BF80E40ABF81C608BF81E907B
:10F99800FFF78EFA2046FFF7ABFB1E4800F0B8FED3
:10F9A8001D4800F021FF5FFA88F000F01DFD40F6C9
:10F9B800A30000F061FB00EA040140F6A30000F098
:10F9C8004BFB9BF82120A24240F2367013D100F085
:10F9D80053FB00F0FB0140F2367000F03DFB4FF6A0
:10F9E800FF72A0E7012F04D1A4F10C035C425C4133
:10F9F800AFE70024ADE700F03FFB40F00401C9B2D7
:10FA0800E9E700BF08240020000600207419010857
:10FA1800022201084024002016240020F0B58BB0F3
:10FA28000D46044617461E46FFF742FA0020FFF728
:10FA38005FFB204600F0BEFD00240123CDE908430A
:10FA480003234FF4167229462046CDE90644CDE932
:10FA58000444CDE90244CDE900532346FFF774FE80
:10FA68002046FFF77DFAFFF735FAF3F721F801F0A2
:10FA780043FC0446204601F049FCB04205D301246A
:10FA8800FFF716FA20460BB0F0BD00F02FFF00B2CA
:10FA98008742EFDA0024F3E7F7B500230C4640F27B
:10FAA80001211A460646084600F01EFD644B654DC6
:10FAB8004FF400529A6195F85600012100F09CFF1E
:10FAC8002B78012B40F6890013D195F85130062B7D
:10FAD8000FD100F0D1FA00F0FB0140F6890000F0E8
:10FAE800BBFA2B78042B6CD8DFE803F0524B527F1B
:10FAF800090000F0C1FA40F00401C9B2EDE7524A2A
:10FB0800731E1046C6F101074FF0000CF9188C421D
:10FB18006FDC0022E7001346BA4271D19A0142EA2B
:10FB2800C3125B0183F020031343661C0355F6B22E
:10FB380002234648AB73AE7600F056FE0021F12052
:10FB480000F08AFA0021F02000F086FAAB6C642BF2
:10FB580070D17021F32000F07FFA1D21F22000F00F
:10FB68007BFAE1008C1CF420090A00F075FA04F015
:10FB7800FE01F52000F070FA33486FF07F423146FD
:10FB88001DE0EC77314800F02FFE0022214615E0F9
:10FB980001F008F80128074625D121460DF1070292
:10FBA800304601F004F80446A0B99DF8073027480C
:10FBB800AB7500F019FE9DF807102246304600F09C
:10FBC80065FB6968224801F063FC214801F026FCC6
:10FBD800002006E01F4B3A460021022001F0A2F85F
:10FBE800032003B0F0BDAC75CCE70223AB73AC7651
:10FBF800C8E713F8011FC943197002F801CB85E75C
:10FC0800D1106FEA020C715C0CF0070C013241FA5A
:10FC18000CF101F001014FEAE20C4B40D14310F81E
:10FC28000CE001F0070103FA01F141EA0E0100F8C6
:10FC38000C1071E7E121F32000F00EFA04218DE7A2
:10FC48000004004808240020EC220020162400208C
:10FC580064240020A4210108F0B5BDF814409DF8E3
:10FC680018709DF81CE09DF8205040B1012814D070
:10FC78000122002398180138B0FBF2F0F0BD87F09C
:10FC88000107E30003EBC70318330EEB450503EB4D
:10FC9800C5034FF47A714B43ECE7501F012803F179
:10FCA800040302D80C2C38BF0C24D1B9A2F10B0CD8
:10FCB800BCF1010F8CBF4FF0000C4FF0010C280174
:10FCC800002F00EBCE0014BF00251425A0EB820006
:10FCD800062A4FEA82062844A2F102070DD83546C3
:10FCE80010E0012906D1A2F10C00D0F1000C4CEB78
:10FCF800000CE4E74FF0000CE1E70830BCF1000F1E
:10FD0800EDD0BD000028ACBF2E182E1C701E90FB35
:10FD1800F5F003FB0044094B062A5A5C8CBF0C34EF
:10FD28000E340A2A09D8A30001334FF47A71BB4074
:10FD38004B43034951F822209CE7FFDE02220108C9
:10FD48000822010808B5094B012193F8560000F074
:10FD580053FE4FF4D7602D2100F07EF900F033FBFD
:10FD6800BDE80840024800F07BBA00BF0824002024
:10FD7800FFFF0F0073B5A44CB4F854300025202BB6
:10FD88008DF80350019500F01B8114D8082B0DD86D
:10FD98007BB1013B072B0CD8DFE813F042005B0076
:10FDA8000B00CD000B000B000B00FD00102B00F02A
:10FDB800008102B070BDB3F5807F00F0988011D843
:10FDC800402B00F01081802BF3D1284600F032FA46
:10FDD8008E4B1B68002BECD09B69002BE9D0284682
:10FDE8009847E6E7B3F5007FE3D1894B012229461E
:10FDF800022000F097FF00F029F9042840F08580E0
:10FE0800844B85484FF400529A6201F0B9FA2846AB
:10FE180000F010FA7D4B1B68002BCAD05B6814E019
:10FE28007C4B7D484FF400529A6201F0A9FA0020F9
:10FE380000F000FA00F0B8FE012801D100F0BDFE84
:10FE4800724B1B68002BB4D01B68002BB1D09847AD
:10FE5800AFE7704B71484FF480529A6201F090FA04
:10FE6800657895B9284600F0E5F9294640F602106C
:10FE780000F0F2F840F6441000F0FEF840F00201FD
:10FE8800C9B240F6441000F0E7F8FF220DF1030173
:10FE980063485E4D00F05AFD624800F071FD2B6822
:10FEA800002B86D09E68002E83D094F82430012B36
:10FEB80008D194F9313094F930209DF8031058484E
:10FEC800B04776E7E06B01A900F022FE019B9DF8A0
:10FED800031053484FF47A7203F5FA7393FBF2F365
:10FEE8002A685BB2956894F92920A84761E72846F3
:10FEF80000F0A0F9454B1B68002B3FF45AAF9B69F3
:10FF0800002B3FF456AF01206AE700F09FF8052860
:10FF18007FF44FAF3F4B41484FF480529A6201F053
:10FF28002FFA284600F086F9384B1B68002B3FF45F
:10FF380040AFDB6889E700213B4B0122022000F03B
:10FF4800F1FEA16D00293FF434AFC1F3074140F63B
:10FF5800031000F081F894F8591040F6041000F0EE
:10FF68007BF894F8581040F6051000F075F840F644
:10FF7800021000F081F840F00101C9B240F6021009
:10FF880000F06AF8002340F262211A460846A36589
:10FF980000F0AAFA0DE7254B01220021022000F00B
:10FFA800C1FE00F0FFFD01287FF403AF00F006FE5C
:10FFB800FFE61F4B01220021022000F0B3FEF8E605
:10FFC800164801F0DDF9607808B900F033F90F4BF5
:10FFD8001B68002B3FF4EDAEDB68002B3FF4E9AE65
:10FFE8009847144BE6E7144B01222946022000F0FB
:08FFF80099FE607808B900F0E1
:020000040801F1
:100000001DF9044B1B68002B3FF4D7AE1B6920E79A
:1000100008240020EC230020B92101080004004836
:1000200064240020F0230020EC2200202C24002057
:10003000CD210108D6210108E0210108E9210108AC
:10004000F2210108024BA3F85400FFF797BE00BF4E
:1000500008240020014B1878704700BF822400203C
:1000600007B501238DF807100DF10702014603487B
:10007000F7F7D2F903B05DF804FB00BF0C080020CD
:1000800007B5012301460DF107020448F7F7FDF912
:100090009DF8070003B05DF804FB00BF0C080020CA
:1000A00010B50446F3F79EFF01280CD140F623104B
:1000B000FFF7E6FF00F0F901214340F62310BDE809
:1000C0001040FFF7CDBF10BD10B50C4B1B78044698
:1000D0009BB94FF4D760FFF7D3FFC4F3002100F0C2
:1000E000FE0001434FF4D760FFF7BAFFE1B240F2E0
:1000F000B960BDE81040FFF7B3BF10BD83240020F6
:1001000010B51346EFF3108472B60A460146034851
:10011000F7F782F984F3108810BD00BF0C080020A7
:1001200008B5014608224FF4D860FFF7E9FF002028
:1001300008BD000007B5074B1B7840BAADF80400B6
:100140002BB9022201A940F2BC60FFF7D9FF03B02E
:100150005DF804FB8324002007B5074B1B7840BAE9
:10016000ADF804002BB9022201A940F2BE60FFF7EE
:10017000C7FF03B05DF804FB8324002010B51346CD
:10018000EFF3108472B60A4601460348F7F77DF98B
:1001900084F3108810BD00BF0C08002010B5134672
:1001A000EFF3108472B60A4601460348F7F75FFA88
:1001B00084F3108810BD00BF0C0800200A460146D9
:1001C0000020FFF7EBBF000010B51346EFF31084DB
:1001D00072B60A4601460348F7F77CFA84F31088A2
:1001E00010BD00BF0C08002010B51346EFF31084BB
:1001F00072B60A4601460348F7F782F984F310887D
:1002000010BD00BF0C08002013B504460020F3F712
:10021000C3FE0220FFF744FF04F0070401220DF1A2
:10022000070184208DF80740FFF7DEFF024B002214
:100230001A7002B010BD00BF8224002007B5012251
:100240008DF807000DF107018020FFF7CDFF9DF825
:100250000730002B034B0CBF012202221A7003B09F
:100260005DF804FB8224002007B5094B8DF80600D9
:1002700004221A70030C8DF804300322030A01A92A
:1002800083208DF80530FFF7AFFF03B05DF804FB66
:100290008224002010B51446FFF790FF2046BDE8E9
:1002A0001040FFF7E1BF000007B5094B8DF80600CD
:1002B00005221A70030C8DF804300322030A01A9E9
:1002C00082208DF80530FFF78FFF03B05DF804FB47
:1002D0008224002073B5002640F6E2000196FFF765
:1002E000CFFE00F0FE01054640F6E200FFF7B8FE43
:1002F00040F6E500FFF7C4FE00F07F01044640F63B
:10030000E500FFF7ADFE6FF07F40FFF7CDFF042261
:100310000DEB020140F61900FFF730FF3046FFF702
:100320008DFF294640F6E200FFF79AFE214640F68F
:10033000E500FFF795FE019802B070BD13B50C4BB8
:1003400004460522972140F6AC001A70FFF788FE9C
:10035000230C8DF804300322230A01A982208DF892
:1003600005308DF80640FFF73FFF02B010BD00BF1B
:100370008224002007B5030C8DF80030030A8DF8A5
:1003800001300B0C49BA8DF80200ADF804100622BA
:10039000694694208DF80330FFF726FF024B0622B2
:1003A0001A7003B05DF804FB82240020002208B517
:1003B0001146C520FFF718FF014B07221A7008BD30
:1003C0008224002000221146D120FFF70DBF002219
:1003D0001146D220FFF708BF07B501228DF80700AC
:1003E0000DF107019F20FFF7FFFE03B05DF804FB4E
:1003F00007B501228DF807000DF10701A020FFF7D6
:10040000F3FE9DF807103F2907D901F0F8010131EB
:10041000C9B240F20670FFF723FE03B05DF804FB9B
:1004200007B5F3F7DFFD431E584258418DF807002A
:1004300001220DF107019620FFF7D6FE03B05DF80B
:1004400004FB07B500F07F008DF8070001220DF1D5
:1004500007018920FFF7C8FE03B05DF804FB000028
:10046000154B984207B51BD8144B98421BD8144B18
:1004700098421BD8134B98421BD8134B984295BFF8
:1004800029226B222B236F238DF8042001A902223D
:1004900098208DF80530FFF7A7FE03B05DF804FB48
:1004A000E122E923F0E7D722DB23EDE7C122C523D0
:1004B000EAE775228123E7E700E9A43580F8A9324D
:1004C0008044E52D000B6B1B40FC541907B58DF8DB
:1004D000062004228DF804008DF8051095200DEB00
:1004E00002018DF80730FFF77FFE03B05DF804FBD3
:1004F00007B552BAADF8042040BA082249BAADF89F
:100500000000ADF802105BBA69461046ADF806303F
:10051000FFF76AFE03B05DF804FB07B50B0C04227D
:1005200000F0070049BA8DF80400ADF806109720D6
:100530000DEB02018DF80530FFF756FE03B05DF8B4
:1005400004FB000010B508B1194B1860F2F7B6F9BA
:100550000220FFF7A5FD0024164B20461C70FFF774
:100560006DFEF3F73DFD012817D14FF42071FFF721
:10057000D4FF40F611102146FFF772FD4FF07F00C7
:10058000FFF75FFF0E2140F61F10FFF769FDF3F73D
:10059000CFFC094B01221A7010BD102140F611103A
:1005A000FFF75EFD102140F61210FFF759FDE9E755
:1005B00084240020802400208224002037B50C4DA4
:1005C0002B7804461BB9FFF74BFF01232B70002348
:1005D000084A6006E109F1F79BFA042200BA01908B
:1005E0000DEB02018620FFF7FFFD03B030BD00BF19
:1005F000802400200048E80107B5094B8DF807006A
:100600000146187018B940F2AC60FFF729FD0122CD
:100610000DF107018A20FFF7E7FD03B05DF804FB49
:1006200083240020012873B50C46164637D10020DC
:10063000F3F7DAFCA042B8BF44B20E2805461AD13F
:1006400001231A4600210420FFF740FF6FF010033A
:100650009C42B8BF1C46182140F6E700FFF700FD9A
:10066000022201A98E208DF804408DF80560FFF765
:10067000BBFD02B070BD01230A28E4B21A464FF058
:10068000000105D11846FFF721FF033464B2DDE70E
:100690000720C5F10E05FFF719FF2C44F6E740F6D9
:1006A000D800FFF7EDFC40F01E01C9B240F6D800BB
:1006B000FFF7D6FC0120F3F797FCA042B8BF44B285
:1006C000142805464FF001034FF000020CD105211C
:1006D0000320FFF7FBFE023464B26FF008039C4274
:1006E000B8BF1C463821B7E7112805D103210220E5
:1006F000FFF7ECFE0534EFE70E2804D1022108468F
:10070000FFF7E4FEE9E7C5F11605072104202544BB
:10071000FFF7DCFE6CB2E0E713B5314A04465168DE
:1007200010686B4603C32F4B20781B78834201D09F
:10073000FFF762FF2378032B27D8DFE803F00239A5
:10074000283C6268284BB3FBF2F31A0CA1688DF8C1
:1007500000208DF802301A0A237B8DF80330637B6A
:100760008DF801208DF80430204A00234806C9097D
:10077000F1F7CEF9030C40BA8DF80530ADF806005C
:10078000082269468B20FFF72FFD02B010BD2269B9
:10079000154BB3FBF2F31A0C8DF800208DF80230E4
:1007A0001A0A237D8DF801208DF803300422E8E732
:1007B000A3690093FAE762680B4BB3FBF2F31A0CE0
:1007C0008DF800208DF802301A0A237B8DF8033053
:1007D000637B8DF801208DF804300522D1E700BF3E
:1007E00084190108832400200000093D0048E80125
:1007F0001FB52E4A0446D1689068127C01AB03C332
:100800001A702B4B20781B78834201D0FFF7F4FE3F
:100810002378032B26D8DFE803F002383302637A0B
:10082000F12B21D14FF6FF70FFF784FC48F2050051
:10083000FFF792FC02236288A188ADF8061052BA35
:10084000E188ADF804208DF80B30227AA37A8DF878
:100850000A20ADF808108DF80C30092201A98C206F
:10086000FFF7C2FC04B010BDF22BE4D141F60F50EB
:10087000FFF760FC41F22100FFF76EFC0623DAE788
:10088000237B8DF804300122E8E7E389094A5BBA4B
:10089000ADF80430237C13708DF80630637C8DF83E
:1008A0000730638AADF808300622D7E784190108BB
:1008B000832400208124002007B502228DF8040043
:1008C0008DF805108F2001A9FFF78EFC03B05DF8AD
:1008D00004FB000010B51346EFF3108472B60A460D
:1008E00001460348F6F744FE84F3108810BD00BFAC
:1008F0000C08002007B5012201A91520FFF7EAFF27
:100900009DF804004042401003B05DF804FB000075
:1009100037B505460C46022201A91320FFF7DAFF7E
:100920000A4B1B78012B0DD1094B1B78012B09D1E8
:1009300040F20270FFF7A4FB9DF805302870237089
:1009400003B030BD9DF80400F6E700BF832400200B
:1009500081240020F7B50D46064600240DF107015D
:10096000284617468DF80740FFF7D2FF2A78BA428B
:1009700007D89DF807003146FFF726FC204603B054
:10098000F0BD0120FBE7000013B50322044601A9D6
:100990001420FFF79FFF184B1A7822704AB1012AE2
:1009A00017D014220021204600F0D2FA0F23237022
:1009B0000DE09DF8043023719DF80530A2605B4284
:1009C0005B10A3719DF806305B425B10637102B04F
:1009D00010BD9DF804305B425B1023739DF9053018
:1009E00002339B1063739DF806305B425B10A37368
:1009F000024B1B682361EAE7832400207C2400204B
:100A0000012908B5034608460ED1012B07D1042061
:100A1000FFF746FB0220BDE80840F3F7BDBA022B02
:100A200014BF08460320F6E70120F4E738B5044672
:100A3000F3F7D4FA50B1022814BF01250225284645
:100A400002222146FFF7EEFD284638BD0F2CCCBF11
:100A500002250125F3E70A2070470000014B012021
:100A60001B68184784240020014B02201B6818478C
:100A700084240020014B40201B6818478424002058
:100A800011B1012904D07047044B1B68802018471E
:100A9000024B4FF480701B68F9E700BF84240020EC
:100AA000024B4FF400701B68184700BF84240020DD
:100AB000014B20201B68184784240020014B042090
:100AC0001B68184784240020014B08201B68184726
:100AD00084240020014B10201B6818478424002028
:100AE000024B4FF480401B68184700BF842400204D
:100AF00068B1084A002352F83310814203D902EB4F
:100B0000C302107970470133162BF4D1FEE71F2082
:100B1000704700BFC422010873B51D4B0193044602
:100B200040F607000D46FFF7ABFAC0F3C1030833E8
:100B30006B4413F8042C00F00703013302FA03F3AB
:100B4000144AB2FBF3F2B2FBF4F007281ED84000BF
:100B500003288CBF022304234FF4D66002FB03F466
:100B6000FFF78EFA060240F2B160FFF789FA06F449
:100B700070663043030544BF6FEA00506FEA1050BF
:100B800063094343DB112B6002B070BD0123E3E72F
:100B900004080A0C0048E8014FF0FF3070474FF09E
:100BA000FF3070474FF0FF307047704700207047AC
:100BB0000020704770474FF0FF3070474FF0FF3014
:100BC000704770477047704770B5EFF3108672B684
:100BD000144B5C8A1A8A944213D1C4F5806292B293
:100BE000904206D3844218D901229A7000221C80B8
:100BF0005A825A8A0A800244C2F309025A820020A9
:100C00000DE006D9C4F58065ADB28542F1D88242C7
:100C1000E9E7121B92B28242EBD84FF0FF3086F325
:100C2000108870BD88280020EFF3108172B6034A47
:100C3000D38A0133D38281F310887047882800203B
:100C4000EFF3108172B6034AD38A013BD38281F35A
:100C5000108870478828002010B508481822002105
:100C600000F076F906484FF48062002100F070F938
:100C7000044B05481B68BDE8104018478828002031
:100C800088240020241A0108F90D0108014B58603E
:100C9000704700BF88280020014B1872704700BFC2
:100CA0008828002073B5EFF3108572B61C4CE08ADB
:100CB00000282FD1FFF7B8FF218A628A914227D0FE
:100CC000A378012B12D1238820805B1A9BB20221CA
:100CD000A382A17063B9A3702382238A9A428BBF37
:100CE000D21AC3F58063A282A38201E0002BF4D064
:100CF000238A0C4E1E4485F31088F1F7CBFE0A4B75
:100D0000A18ADB680193304602B0BDE87040184705
:100D1000FFF796FF85F31088002002B070BD00BF7A
:100D20008828002088240020241A010808B4F0B57F
:100D300086B00023ADF800302C4B0B9C1D7A854209
:100D40004DD3D86881434DD15B681BB112B1694660
:100D500002A898470CAB22464FF400712448019337
:100D600000F0F6FBFFF760FFBDF8003018440DF10E
:100D7000020180B2FFF728FF01302BD00022BDF81E
:100D80000030BDF802701B480DF1080C164691B2F8
:100D900017FA82F58B42ADB216D83B449BB20EB126
:100DA000ADF80230BDF80250019B22464FF40071AD
:100DB000284400F0CDFBFFF743FFFFF773FF06B0B9
:100DC000BDE8F04001B070471CF8011B41550132ED
:100DD0000126DCE7FFF734FF6FF00200EFE76FF06A
:100DE0000400ECE76FF00500E9E700BF8828002069
:100DF000A02800208824002013B5EFF3108472B6D9
:100E0000204B9A78588A022A1DBF1A8A998A52184A
:100E1000002214BFC2F309029A7090421A8228D0AD
:100E2000D98A012925D19978012913D119888A1ADB
:100E3000022192B2997000219A82198062B99A7047
:100E40001A821A8A90428BBF801AC2F580629882F9
:100E50009A8201E00029F4D01A8A0B48104484F3E6
:100E600010880A4A998AD368019302B0BDE81040FD
:100E7000184784F31088F1F711FE02B0BDE8104066
:100E8000FFF7DEBE8828002088240020241A0108ED
:100E9000024A00231360024A13607047A42A00200C
:100EA000A02A002010B5EFF3108472B641B10129D9
:100EB00003D1064A13680343136084F3108810BDFE
:100EC000024A136823EA0003F6E700BFA42A0020C1
:100ED00010B5EFF3108472B641B1012903D1064A6F
:100EE00013680343136084F3108810BD024A13682B
:100EF00023EA0003F6E700BFA02A002038B5EFF38D
:100F0000108572B60A4B0B4C1B6833B123689847A7
:100F10006368984785F3108838BD074B1B681BB181
:100F2000A3689847E368F4E7236998476369F0E7A3
:100F3000A42A0020B0190108A02A002001380A4480
:100F4000914200D1704711F8013B00F8013FF7E7EB
:100F500000F02CBC10B5EFF3108472B6064A13688B
:100F600003431360054A52F83130034342F83130ED
:100F700084F3108810BD00BFF42A0020EC2A002062
:100F800070477047030C1B04C3B90004102310F012
:100F90007F4F02BF08330002DBB210F0704F08BF72
:100FA00000014FEA1070064A08BF0433125C08BF04
:100FB000DBB2C3F11F03981AC0B270470023E6E703
:100FC000742301082DE9F84F384D394ED5F80080CB
:100FD000DFF8E0B0DFF8E0A0DFF8E090D6F800C07E
:100FE000374FDBF80010374CDAF80020D9F8003022
:100FF00008EA00002860286800EA020E1EEA0C0FCA
:1010000001D019421ED04FF0FF333B60FFF7B8FF0D
:10101000EFF3108472B63368DBF80020DAF80010C2
:101020000B4029680B4205D1D9F80030134201D199
:10103000F1F7BEFC84F31088FFF7A3FFC5F800802A
:10104000BDE8F88F236823680340134062681A42A2
:1010500004BF4FF0FF32626060681840FFF792FFF4
:1010600062683860012303FA00F022EA000262603D
:10107000EFF3108172B63A689340326822EA0302B5
:101080003260226822EA0303236081F310880E4A4B
:101090003B6852F823309847D6F800C0DBF80010C0
:1010A000DAF80020D9F80030A5E700BF04060020D8
:1010B000F42A0020AC2A002008060020B02A0020D4
:1010C000A82A0020EC2A0020B42A002010B51146DE
:1010D000EFF3108472B6FFF755FF034B43F820106F
:1010E00084F3108810BD00BFB42A002082B082B003
:1010F0000DF1080C0CE90600BDF8042003930B4425
:10110000BDF810100A4491B212B2B2F57A7FA2BFB4
:10111000A1F57A72013312B20360828002B002B08C
:10112000704782B082B00DF1080C0CE90600BDF8E2
:1011300004200393CB1ABDF81010521A91B212B2C8
:10114000002ABEBF01F57A7203F1FF3312B20360C9
:10115000828002B002B0704730B585B0114D6B4649
:1011600083E8030000230293ADF80C3003A82B6939
:101170009847009BBDF804400290181ABDF80C3047
:10118000E41AA3B224B2002CBEBF03F57A731CB2DA
:1011900000F1FF302B689847AB682046984705B0B0
:1011A00030BD00BFE419010873B5114E0023054698
:1011B0000093ADF8043001A833699847F3680090B4
:1011C0009847736804469847009B1844BDF804305C
:1011D00023449AB21BB2B3F57A7FA2BF0130A2F5C5
:1011E0007A731BB228602846AB8002B070BD00BF86
:1011F000E419010837B500230093ADF80430074B1C
:1012000004461B6901A898476D46009095E80300C5
:1012100084E80300204603B030BD00BFE419010894
:1012200037B50F4D02AB03E90300EB6898476B68D5
:1012300004469847BDF80430009A1B1B99B21BB2B4
:10124000002BA2EB0002BEBF01F57A7102F1FF3262
:101250000BB24FF47A7000FB023003B030BD00BF18
:10126000E41901082DE9F0414FF47A75B1FBF5F569
:10127000C5EB4513DFF83C8005EB8303A1EBC3030B
:101280009CB2D8F80C3006469847D8F80430074688
:101290009847E31999B21BB2B3F57A7F2844A2BFED
:1012A000A1F57A7301301BB23060B3803046BDE8DF
:1012B000F08100BFE4190108024B00221A60024BC2
:1012C0001B681847F82A0020F8190108F8B50446E9
:1012D000174608461E467CB173B1084B00255B6A71
:1012E00025609847069B60602581A572E6602361B2
:1012F000E77265612846F8BD0120FCE7F81901088E
:1013000010B5034CE3699847A36ABDE8104018473D
:10131000F819010870B5064DEB69064698476B6AE7
:10132000044630469847AB6A201ABDE8704018471B
:10133000F8190108054B1B680BB918467047834222
:1013400001D05B69F8E70120704700BFF82A002050
:101350002DE9F3410B4E336A044698470123B769E0
:101360002372D4F800800546B8472844804502D24D
:10137000B84728442060B3682068019302B0BDE8F4
:10138000F0411847F819010870B520B3EFF3108643
:1013900072B6124D2B680122827253B10022427242
:1013A00098425C690ED102723CB120462C60FFF776
:1013B000CFFF86F31088002070BD094BDB6898478B
:1013C0002C60F6E71A465B69002BF2D09842F9D1FF
:1013D00043695361EDE70120EEE700BFF82A0020E2
:1013E000F8190108084B10B51A685369516911B909
:1013F0005061416110BD046819688C4202D91A46D7
:101400005B69F3E71946F3E7F82A0020044A1368FA
:101410000BB10021197243611060FFF799BF00BF43
:10142000F82A00202DE9F041044600282DD0FFF7CE
:1014300081FF50BB657A45BBEFF3108872B6144E3E
:101440006768336A984787422CBF27602060114F36
:10145000A5724FF4807323813B684BB93369984779
:101460002046FFF7D3FF88F310882846BDE8F081B7
:10147000B3699847236818443B6820601B6898420A
:101480002046EED3FFF7AEFFEDE70125EDE700BF05
:10149000F8190108F82A002010B5044608467CB166
:1014A000084B5B6A984760602046FFF743FF40B1F6
:1014B0002046FFF769FF2046BDE81040FFF7B2BFA6
:1014C000012010BDF81901082DE9F041EFF3108754
:1014D00072B61D4E1D4D736998473369044698478F
:1014E0002B684BB94FF000082B688BB9286828BBD4
:1014F00087F31088BDE8F081011B241A1A688A421C
:101500008CBF121900221A605B69002BF6D1E9E743
:101510001C681CB1B36998478442E7D22C686369A0
:101520002B60A4F80880D4E9033098476389B3F5A9
:10153000807FD9D12046FFF775FFD5E7037A002BCE
:10154000D6D1FFF705FFD3E7F8190108F82A0020E4
:101550002DE9F04F97B000298046039140F30E81AA
:101560009A46044603991378A4EB0800013923B97D
:101570000023237017B0BDE8F08F8842F8DA252BDE
:1015800004D004F8013B1646721CEBE792F801C048
:10159000ACF13003D3F1000E4EEB030EACF130038F
:1015A000092B02F1010629D8324600254FF00A091D
:1015B000164612F8013BA3F13000092819D93378F7
:1015C000692B00F09C801CD8632B28D0642B00F082
:1015D0009680582B5BD0252B19D13378002B00F047
:1015E000928004F8013BA4EB08038B4280F28980CF
:1015F000CAE709FB0533A3F13005D9E74FF0FF3502
:10160000DDE7752B7DD0782B43D0732B1ED025239F
:1016100004F8013BA4EB08038B4272DADDE7002DEE
:1016200005F1FF39D8BF4FF000094A462046202176
:1016300000F0BCF85346A144002D53F8042B89F860
:101640000020D8BF01252C449A469DE74C4B5AF800
:10165000047B002F08BF1F463846EFF7B1FEA5EB0D
:10166000000B8542B8BF4FF0000B5A46814620213F
:10167000204600F09BF8A34400234B4502DB0BEB14
:10168000090481E7FA5C0BF803200133F5E74EF01B
:10169000400E1020DFF8EC903B4F1EF0400F08BFCB
:1016A0004F465346BCF1300F0197A4EB08020CBF24
:1016B000302720271EF0020FA1EB0202029753F8F9
:1016C000041B22D0002920DA4942013D4FF02D0EA3
:1016D00005AF009700278946DDF804A0B1FBF0F1C3
:1016E00000FB119B48451AF80BB0DDF800A00AF882
:1016F00001BB07F10107CDF800A0ECD90EE04EF0D8
:10170000020E0A20C6E7013E6DE711B14FF0000E50
:10171000DEE730208DF814008E460127BCF1300F33
:10172000A5EB070504D02020002D05F1FF3509DCCD
:10173000BEF1000F04D02D21013A04F8011B83D023
:1017400025440AE0013A04F8010BEDD17CE7029947
:1017500004F8011B013A3FF477AF291B0029F6DC9E
:1017600005A9394422442744A7423FF46DAF11F83C
:10177000010D04F8010B9442F6D165E70020F9E66B
:10178000842301088B230108B023010810B5013917
:101790000244904201D1002005E0037811F8014F86
:1017A000A34201D0181B10BD0130F2E702440346EA
:1017B000934200D1704703F8011BF9E770B50D4D56
:1017C0000D4C641BA4100026A64209D10B4D0C4CF5
:1017D00000F0B2F8641BA4100026A64205D170BD2B
:1017E00055F8043B98470136EEE755F8043B984717
:1017F0000136F2E7B8240108B8240108B82401082A
:10180000BC24010800F003B8002200F00EB80A441E
:10181000914200F1FF3300D1704710B511F8014B30
:1018200003F8014F9142F9D110BD13460A461946FB
:10183000FFF7BCBF00000000C1F30A522DE9F843D6
:10184000A2F2FF36132E0B4607460C46054632DC45
:10185000002E14DA34A3D3E90023EFF7BFFD0022F2
:101860000023EFF7EFFF38B1002C56DA24F00044E4
:10187000254355D02E4C002523462F4625E02D4AE2
:1018800042FA06F801EA080202431ED026A3D3E971
:101890000023EFF7A3FD00220023EFF7D3FF00287A
:1018A000EAD0002CBEBF4FF480133341E41824EA81
:1018B00008040025E0E7332E0BDDB6F5806F04D178
:1018C0000246EFF78BFD07460B4638461946BDE842
:1018D000F883A2F213424FF0FF3828FA02F810EA18
:1018E000080FF2D010A3D3E90023EFF777FD002211
:1018F0000023EFF7A7FF0028BED0002C0ADA142E31
:1019000001D1013406E0C6F134060123B3401D4481
:10191000AF42F6D825EA0805AEE700252C46ABE72E
:101920004FF00044A8E700BF9C7500883CE4377E78
:101930000000F0BFFFFF0F00F8B500BFF8BC08BC07
:101940009E467047F8B500BFF8BC08BC9E4670477D
:1019500000000000010000000200000000EA06375D
:10196000000000005000000040F7093700000000B0
:1019700050000000C194C10000000000B227000028
:101980000000000000000000000000000000000057
:101990000000000000000000B5010008F10100088F
:1019A00098190108FC7F003F00350113C41200089C
:1019B0007327000855270008392700085927000811
:1019C00035270008852700085975336E3148344F94
:1019D0003152354E395332543653256473253033E2
:1019E000643A0000612C0008012D0008712C0008E9
:1019F0000D2D0008D12C0008192D00080000000052
:101A0000812C0008392C0008052C0008BD2B00088B
:101A1000152C0008292C0008C92B0008CD2B000824
:101A2000E12B0008C12F0008E92F00086D2F0008E6
:101A3000592F00085246414300505658585800212B
:101A400059756E486F726E205354532052657669F3
:101A50007665210001000000030000000500000081
:101A60000100000001000000060000000A00000064
:101A70002000000002000000040000000800000038
:101A80001000000040000000800000000001000085
:101A90000002000000000000000000000000000044
:101AA0000000000001000000020000000300000030
:101AB00004000000A0860100400D0300801A06000B
:101AC00000350C0040420F0080841E0000093D00DC
:101AD00000127A000024F40000366E010048E8018C
:101AE000006CDC02000000000000000000000000AC
:101AF0000000000004020800101010041010100272
:101B000010101008010002000400060008000A007E
:101B10000C001000200040008000000108040204B6
:101B20000801010101010103070100006572726FE4
:101B3000723A20526567696F6E206973206E6F7408
:101B400020646566696E656420696E20746865202E
:101B50004D573A20736574206C6F726177616E5FC8
:101B6000636F6E662E68206163636F7264696E676F
:101B70006C790D0A004D414320727854696D654FB0
:101B800075740D0A004D414320747854696D654F9A
:101B900075740D0A004D4143207278446F6E650DD7
:101BA0000A004D4143207478446F6E650D0A0008A9
:101BB0000A0C0D0E10121415181A1B1D1E212403D9
:101BC00005020501060202050000060000010504E9
:101BD0000400000048E8010048E8010048E801006E
:101BE00048E8010048E8010048E8010090D00300FF
:101BF00000000000030000000201000C0B0A0908AD
